:1000000000400020457200008572000087720000E9
:1000100000000000000000000000000000000000E0
:1000200000000000000000000000000089720000D5
:1000300000000000000000008B7200008D720000C4
:100040008F72000041530000C17600008F720000E3
:100050008F720000000000008F7200008F7200009D
:100060008F720000997A0000393200008F72000010
:100070008F7200008F7200008F7200008F7200007C
:100080008F720000457700008F7200008F720000B1
:100090008F7200008F7200008F7200008F7200005C
:1000A0008F7200008F72000000000000000000004E
:1000B0000000000000000000000000000000000040
:1000C00010B5064C2378002B07D1054B002B02D02E
:1000D000044800E000BF0123237010BD640200202B
:1000E0000000000030E60000044B10B5002B03D0E8
:1000F0000349044800E000BF10BDC04600000000F6
:100100006802002030E60000164B002B00D1144B93
:100110009D46402292029A1A924600218B460F4633
:100120001348144A121A0BF003FB0F4B002B00D09C
:1001300098470E4B002B00D0984700200021040068
:100140000D000D48002802D00C4800E000BF0BF065
:10015000AFFA2000290007F005FB0BF083FAC04638
:100160000000080000400020000000000000000027
:1001700064020020C42F00200000000000000000E6
:1001800002000120104011D1042A0ED91368180969
:1001900080B2002809D001388000031D11180979A8
:1001A000002902D001309842F8D170470020FCE7C6
:1001B0000378002B03D05AB2002A01DB01307047CC
:1001C0003F229343C03B59424B41C01803789343AD
:1001D000802BF4D10130F9E710B500240378002B0F
:1001E00001D1200010BDFFF7E3FF0134F6E770B541
:1001F000002204000D00411C092003F047FB0028E9
:1002000006D001236200134343600023A34200DBB6
:1002100070BD9A00A958821891600133F6E770B555
:10022000012803DC1C2001F073F870BD01230D6868
:1002300011201D42F7D04868184206D1042804D97D
:100240000F2302681340042B01D00E20EBE703F0CC
:100250007BF96D100400002D03DDFFF7BDFFA84200
:1002600006DA1220DFE72000FFF7A2FF0400013DBD
:10027000012DF8D120787F2809DDDF280BDCF82359
:100280003F22DB00800118406378134018430123AC
:1002900040001843C9E7EF280BDCFC226378120109
:1002A0009B0113403F220007000C0343A07810403D
:1002B000ECE7F72812DCFC22637892021B03134060
:1002C000E0228004520310403F221843E378134099
:1002D000FC220343A07812018001E8E7012040429C
:1002E000D5E7F8B54D680F00EB0706D4042D04D907
:1002F0000F232E683340092B03D00B2001F008F8A0
:10030000F8BD6B683609B6B25C10731EA3420FD8F5
:100310000321200009F0C8F86421642803DC0100EF
:10032000032800DA03212800891903F0E1FA050007
:100330002B6800201B099BB2013B9C42E0D23A682B
:10034000A31C9B005A510123013464001C436C60C0
:10035000D6E7F0B585B0012803DC1C2000F0D8FFFB
:1003600012E001274B683A000093022806D08B6800
:100370003B4203D05F10002F00DC17000125009BDB
:100380002B4203D00120404205B0F0BD009B042B5E
:10039000F8D91B680C680F261900314004292AD1AE
:1003A0002C4205D1042C03D923681E40042E01D011
:1003B0000E20D3E70098FFF7E3FEB842E2DB009897
:1003C00003F0C2F80600200003F0BEF80100781E1A
:1003D00030180BF063FD041ED4D03378002B01D00D
:1003E000A64202D36800012521E03000FFF7E0FEBD
:1003F00001350600F1E709293ED1009B5B685B10DF
:1004000001939F42BEDC2C422ED1042C2CD92368B0
:100410003340042B28D1200003F096F80396029075
:100420007E1C009AB300D058844202D17800284341
:10043000AAE728420ED104280CD90368039A134076
:10044000042B07D103F080F8010002980BF0F0FCB8
:100450000028EBD0019B37009E42E1DD92E71F00B0
:10046000019B9F4200DD8DE77B1C00999A008A5812
:10047000A242F4D17800B6E7032900D082E71A0936
:1004800092B25B0F92000B40D31A01939F4200DDA2
:1004900078E72C4229D1042C27D922681640032E54
:1004A00019D1100980B2520F80003240251D801AE8
:1004B000019B2E181B1A0193009B781E0433019A8E
:1004C000904200DD5EE72A001918B2420FD316D120
:1004D0000130400087E7042E07D1200003F034F8F4
:1004E00005002000FFF74CFEE2E70F2036E70C780E
:1004F000A4461478A44502D101310132E5E7013068
:10050000DDE710B503F004F843000120184310BDE7
:10051000C30711D404280FD90F2302681340032BFB
:100520000AD119400133591AC0234907DB05194084
:10053000024B1A40114301607047C046FFFFFF9F06
:10054000F7B507000E001C20012F06DD4C680123C3
:1005500022001A40009203D10D2000F0D9FE53E092
:10056000022F02D08A681A42F6D0012335681D4254
:1005700000D0A9E0042D00D8A6E01C41002C00DC2E
:100580001C000F2029680840092828D16B685B10DF
:100590000093022F05D0B368009A5B109A4200DDE9
:1005A0000093009B01221D1B0135EB43DB171D400F
:1005B000691C092003F06AF9071E09D001236D00A8
:1005C0001D4303003268083345600099A14201DAF7
:1005D0003800FEBD0134A100515802C3F5E70428DC
:1005E00045D1280002F0B0FFFFF7F6FD0190022F81
:1005F00004D0B3685B10984200DD0193019BA342D5
:1006000004DA002003F0B4F90700E1E7280002F063
:100610009BFF0700009BA34221DB2800009702F00C
:1006200093FF05003800FFF7C3FD019B013407006D
:10063000A342F7DA009BC41A200003F099F9071EC1
:10064000C6D002F081FF0190306802F07DFF2200E9
:10065000009B591B411801980BF04EF8B8E7380081
:10066000FFF7A6FD009B070001330093D2E70328A4
:100670002AD10B099BB2490F9B000140591A022F46
:1006800004D0B2685210914200DD1100A14205DA97
:1006900000220320110003F0F9F8B5E703200E1B38
:1006A000331DD9170140C9188910002203F0EEF854
:1006B000071E00D18CE7013631000334FFF728FF15
:1006C000381D29193200C7E7212046E7F8B5002870
:1006D00005DC1C2000F01CFE05002800F8BD0126EA
:1006E0000C6826400FD06410E343DB171C40E11C6C
:1006F00089100022032003F0C9F8051EEDD0210067
:10070000FFF706FFE9E7042C01D80025E5E70F23F2
:1007100022681340042B1BD12000FFF731FDC31CBE
:1007200007000320D9170140C9188910320003F0CF
:10073000ADF8051ED1D03900FFF7EAFE200002F027
:1007400003FF2B1D01003A0018000AF0D5FFC4E793
:10075000092BDAD10320636832005F10FB1CD91724
:100760000140C918891003F091F8051ECDD0390059
:10077000FFF7CEFEFF20BE42AFDA0122B300E3183E
:100780009B68134208D01341FF2B00DD0300D943BF
:10079000C917AA190B4013710136ECE710B57F2970
:1007A00002DC0170013010BD1A4B99420CDC402371
:1007B0008A115B42134303703F230B40802149425F
:1007C000194341700230EEE7134B994210DC2023AD
:1007D0000A135B4213433F24802203708B11524261
:1007E0002340214013430A43437082700330DAE709
:1007F0000A4B9942D7DCF0230370603B4370113BF6
:100800008A11FF3B1A4382703F2211401943C17085
:100810000430C8E7FF070000FFFF0000FF0F0100E2
:10082000F0B50D0085B0002803DC1C2000F070FD41
:100830000DE009680122080010400AD002AC114105
:100840002000FFF7ABFF011B200003F09DF8040020
:100850001AE004293FD90F230C682340092B3AD111
:100860004B685B10019303239C46019B9A420EDD6B
:1008700003F07EF8041E07D02E68012502F064FE06
:100880002F00019B9D421DDD200005B0F0BD01320F
:100890009300CC580123234001D10D20C6E76410FA
:1008A0007F2C0DDD0D4E0223B44209DD0C4E634654
:1008B000B44205DD00270B4EE30FA6427B419B00AF
:1008C000C018D2E70135AB00F1583942E5D04910E4
:1008D000FFF764FFD5E72120A8E7C046FF07000027
:1008E000FFFF0000FF0F010010B5040001200840C9
:1008F00010D104290DD90F230A681340042B08D105
:10090000080002F021FE010020000BF091FA4342A2
:10091000584110BD0020FCE7F7B50F00012803DCAB
:100920001C2000F0F5FCFEBD01264D682E4006D1CE
:10093000042D04D90F222B681A40092A01D00B205C
:10094000EFE76A681B099BB25410A34200D85C1EF3
:1009500039681E48FFF7C8FF01230190002813D112
:1009600039681B48FFF7C0FF002811D0002C0DD0BC
:100970000123621C013C9C409200535123436B6055
:1009800004E00136B200AB50B442FADA0020CAE704
:100990003B680D20DA07C4D55B10002B11DD9C42AB
:1009A0000FDB9B00A200291DEB1889180433994224
:1009B00009D10123013C9C40AA181C4353606C6080
:1009C000E4E71220ADE758681860EFE7C3CD0000F8
:1009D000C7CD0000002310B50C000B70C30705D570
:1009E0000D49421020000BF0E7F908E00B49002800
:1009F00002D0042804D10A4920000BF0FDF910BDF3
:100A00000428FCD90F2302681340042BF7D102F00D
:100A10009BFD04490200E5E7C8D70000CCCD0000EB
:100A2000D2CD0000D7CD0000F0B593B00600029102
:100A30001C20012E1DDD029B01251B681C002C4083
:100A400000D0ADE0042B00D8E6E01A680F231A406E
:100A5000092A4AD10394039A029992008A581700EE
:100A60002F4005D1042A03D910681840092806D060
:100A7000222000F04DFC0190019813B0F0BD5268A7
:100A80005210A418039A013203929642E3D1611CDA
:100A9000012202F0FBFE0190002802D10023019305
:100AA000EAE7019B6400190025435D600831029A62
:100AB000BB00D05802684368120992B25B109A4298
:100AC00000D8531E0022934209DCDA43D2171340A8
:100AD0009B00C918039B01379F42E8DBCCE79400D9
:100AE0000519AD6801320D51EDE72700032A59D1F0
:100AF0000193029ABB00D3582B42B9D1042BB7D92A
:100B0000186801990140032939D1020992B2430FB3
:100B100092000B40D31A1C190137BE42E9D10320C1
:100B2000E31CD9170140C9188910002202F0AEFE5B
:100B300001900028B2D000252100FFF7E9FC019BBD
:100B40001E1D029AAB00D45801231C421FD1042C55
:100B50001DD90F2123681940032918D1180980B223
:100B60005B0F80000B40C01A0023834213DBC3439A
:100B7000DB17184001353618BD42E2DB7CE704295B
:100B800000D075E71800FFF7FBFA2418C4E720002F
:100B9000FFF7F6FAE8E7E2181279F2540133E4E7D6
:100BA00000273C000F25029ABB00D35801221342B4
:100BB00034D1042B32D9186801002940042935D1D9
:100BC0001800FFF7DDFA24180137BE42EBD12000F0
:100BD00002F0CEFE0190002800D15FE7029FB60030
:100BE000BB19041D029301233D681D4229D1042D28
:100BF00027D90F262B681E40042E37D12800FFF777
:100C0000BFFA0600280002F09FFC0100200032001D
:100C10000AF072FDA41922E02700C3E7180005A915
:100C2000FFF7D8FE05A80BF00DF9CCE7032900D09B
:100C30001EE7020992B2430F92000B40D31A1C190F
:100C4000C2E705A92800FFF7C5FE05A80BF0FAF8D2
:100C500005A90500020020000AF04EFD6419029B60
:100C60000437BB42BFD10023237005E7032EF6D122
:100C70001A0992B25B0F92001E40961B291DC5E710
:100C8000F0B50D0097B0002806DC1C2000F040FBFA
:100C90000700380017B0F0BD0C68012123000B409D
:100CA000009306D1042C04D922680F331A40092A74
:100CB00001D00B20EAE7626852100392002A03DC9D
:100CC000009802F055FEE3E7504A019201280BD04C
:100CD0006868084208D1042806D902681340042B2A
:100CE00002D102F031FC019001980BF0ABF8060044
:100CF0000F27039B0834013B05935E43039B02903F
:100D00009B00E318049301232068184273D1042840
:100D100071D901680B003B409C46042B03D1FFF7BF
:100D20002FFA861909E0032B6CD162460B099BB29E
:100D3000490F9B0011405A1A9619049B0434A34290
:100D4000E1D1300002F014FE071EA2D02B680793F9
:100D5000029B002B03D0686802F0F6FB019038007C
:100D600002F0F2FB0400009B079A9B00D3189E68D8
:100D7000300002F0E9FB0123334005000693002B0D
:100D800001D1042E04D809A93000FFF723FE09ADD4
:100D900028000BF057F8069B0490002B0ED1042E70
:100DA0000CD90F2133681940032907D11A0992B2CF
:100DB0005B0F92000B40D31A351D04932000049A58
:100DC00029000AF099FC049BE418029B002B0AD02E
:100DD000059B009A934206DD2000029A01990AF0D1
:100DE0008BFC029BE418009B01330093009A039B49
:100DF0009342B8D14DE709A9FFF7ECFD09A80BF024
:100E000021F88EE702F0A0FBF9E7C0466BD20000A4
:100E100010B50024A04207DD0B6801341C4003D04C
:100E20005C10E343DB171C40611C0122092002F027
:100E30002DFD002803D0012364001C43446010BD35
:100E40000A6870B510000125284034D1042A32D92F
:100E50000F24136849681C40092C17D154681B09DA
:100E60009BB22C41A34200D85C1E844205DC0220C8
:100E70000133984206DB00200FE085005519A96078
:100E80000130F2E7840011510130F2E7032C12D156
:100E9000294203D1132000F03BFA70BD4910FF290D
:100EA000F8D81B099BB204329B00D3189342E2D9B5
:100EB00011700132FAE70B2000F02AFADBE700009C
:100EC0000123F7B500254E680F0033400093AB4275
:100ED0000ED11D00042E0BD90F2233681A40092AA7
:100EE00010D172681B099BB25510AB4200D85D1E31
:100EF0003968CB0717D54C10002C01DDA5421DDA4F
:100F0000122032E0042A04D13000FFF739F905003D
:100F1000EEE7009D032AEBD11D09ADB25B0FAD00DA
:100F20001340ED1AE4E72E48FFF7DEFC002814D04A
:100F30000AF0DEFE290008F09DFB4C1C009B002BF4
:100F40004CD1042E4AD932680F331340092B10D1EB
:100F50000134A400A4592000FEBD39682148FFF7E0
:100F6000C3FC2C000028E9D1113000F0D1F90400B5
:100F7000F1E7042B2AD1300002F0E6FA0500FFF772
:100F80002BF9A042BCDB012C1ADC300002F0DCFAA9
:100F900000902800FFF70CF9461B300002F0E8FC37
:100FA000041ED8D002F0D0FA0190786802F0CCFA92
:100FB000009B3200E91A411801980AF09DFBCAE72C
:100FC0002800FFF7F5F8013C0500DCE7032B05D10D
:100FD0003419E478023B64001C43BCE70B20C4E7EF
:100FE000BCCD0000C7CD0000F7B54D680F002A004A
:100FF00001210A402FD1042D2DD90F242B68BE6862
:101000001C40092C14D169681B099BB24C10019239
:10101000A34200D85C1E39682A48FFF765FC002807
:101020002DD00F232A681340092B1DD1012317E06F
:10103000032C10D10E4203D1132000F069F9FEBD3C
:1010400072100192FF2AF7D81A0992B25B0F920030
:101050001C40141BDFE70B20EFE701339A00AE5072
:101060009C42FADA0020EAE7032BFBD12B00013384
:101070005A1BA242F6DC6A461279DA70F7E7396841
:10108000CB0706D54910002901DD8C4209DA122070
:10109000D3E70D48FFF728FC2100002801D11130CB
:1010A000CBE70F232A681340092B03D101318900B4
:1010B0004E51D7E7032BD5D16B461B796D18EB70DA
:1010C000D0E7C046C3CD0000C7CD000010B5012455
:1010D000086820421AD1042818D90F21026811404B
:1010E000092901D1406810BD032908D113099BB219
:1010F000500F9B000840181A40002043F3E70429D2
:1011000004D102F021FAFFF767F8F5E70B2000F0B1
:10111000FFF8E8E710B5034A0B21034804F0D2F9C1
:1011200010BDC04664CD00005CCD000000207047BB
:10113000042070470120704710B5002002F018FC11
:1011400010BD00207047002070470020704700202D
:101150007047002070470020704700207047002033
:101160007047000010B5034A0C21034804F0AAF9A7
:1011700010BDC0464CCE0000ACCE00007047000051
:1011800010B50124044002D04410200010BD0428F2
:1011900010D90F2302681340042B07D102F0D4F9B1
:1011A00021000A220AF016FF0400EEE7032B01D10A
:1011B0000430F5E70D22014B1A70E6E7A402002087
:1011C000012210B5024018D1042802D903681A0977
:1011D00092B201230B4012D1042902D90B681B09DA
:1011E0009BB20024934206D104309B000431C31803
:1011F000984206D30124200010BD0022E9E7002315
:10120000EFE704780A78002C01D1002AF2D00130EF
:1012100001319442ECD00024EDE70000F7B507005F
:10122000009101933049314B002A02D002220A700A
:10123000013A00261A601B68CE54BE4200DBF7BD9F
:10124000009AB300D058294B274D1C68C8239B0037
:1012500065191C1B0123184206D0254A43102100A2
:1012600028000AF077FD09E0224A002802D004286D
:101270001BD1214A210028000AF06CFD1A4C2000E5
:101280000AF0E0FD194A019B1060002B0BD07B1E79
:10129000B34208DD194B984205D8431C1360202245
:1012A00022540022E2540136C7E7042819D90F233B
:1012B00001680B40042B04D102F046F9104A0300E8
:1012C000CDE7092B03D143680E4A5B10C7E7032B18
:1012D00008D10A0992B2490F92000B40D31A0A4A68
:1012E000BDE70123094ABAE7A5020020C80500208E
:1012F000C8D70000CCCD0000D2CD00001F030000F5
:10130000F3DD00001CD100002BD1000036D100001D
:10131000014B187000207047A402002070B501F046
:101320006FFE094C0100251D1F2228000AF0A2FDB6
:1013300028000AF087FD04230430800800011843C8
:101340002060200070BDC04680020020C368F0B558
:101350009D00836889B05D19030018330693036903
:10136000069A9F00069B0290DF19436901939B0038
:10137000D3180393CD4B1B78002B26D17F222B68EB
:10138000CB491C1213409B005B58043501929F46C9
:10139000029B587804F0D0FC0023029A137027E0D7
:1013A000C24B1B78002B10D12B68019A1C121340E2
:1013B000BF4A9B009B580435E9E7069B3A1DD11AAA
:1013C000BA4BD82928DD1A221A70029BB74C9B68A9
:1013D00021780193EA1A029B92109B7812021A4319
:1013E000029B587804F0B0FC0023029A237013701B
:1013F000029B069A9B680193ED1A029BAD10DD607B
:10140000069BFE1A029BB6101E61039B9B1A029A52
:101410009B10536109B0F0BD1B783C60002B01D0DC
:101420001700D2E72B6801991C120B40A0499B00C2
:101430005B5817000435AAE7069B3A1DD11A9B4B4F
:10144000D82902DD1A221A70BFE728681B78291DE7
:101450003860002B02D017000D00B6E76B680199C9
:101460001C120B4092499B005B58170008358EE711
:10147000069B3A1DD11A8D4BD82902DD1A221A700B
:10148000A3E7A4001B782C193C60002B01D01700A7
:101490009BE72B6801991C120B4085499B005B5808
:1014A0001700043573E7069B3A1DD11A7F4BD829E4
:1014B00002DD1A221A7088E77E49A40061581B7861
:1014C0003960002B01D017007FE72B6801991C12AF
:1014D0000B4077499B005B581700043557E7043FE2
:1014E000744B3A68A400E250704B1B78002B00D07C
:1014F0006BE72B68019A1C1213406D4A9B009B58A6
:10150000043544E76B4BA400E058FFF739FE043F75
:1015100006003868FFF734FE36180120654B760068
:101520000643E650614B1B78002B00D04DE72B683B
:10153000019A1C1213405E4A9B009B58043526E713
:10154000069B3A1DD11A594BD82902DD1A221A706E
:101550003BE70698039C0121A04202D221000C39EE
:1015600009681B783960002B01D017002DE72B6824
:1015700001991C120B404E499B005B581700043523
:1015800005E7069B3A1DD11A484BD82902DD1A22DD
:101590001A701AE70699039881420FD203000C3B98
:1015A0001B6845495B106418E41AA40023583B608B
:1015B0003E4B1B78002B05D0170006E71821197049
:1015C0000023F4E72B6801991C120B4038499B005B
:1015D0005B5817000435DAE6069B039A934219D24A
:1015E00013000C3B1B68344A043FA4185B10E31A39
:1015F000039A39689B0099502C4B1B78002B00D024
:10160000E3E62B68019A1C121340294A9B009B5861
:101610000435BCE61822254B1A70EDE7069B039AA9
:1016200093422DD2244B3E1FE31814000C3C04932C
:101630002368049A5B10D31A039A9B009858FFF70B
:101640009FFD07903068FFF79BFD2468049B6410A2
:101650001C1B079BA4001F1801207F00039B07434E
:10166000E7503700114B1B78002B00D0ADE62B68FC
:10167000019A1C1213400E4A9B009B58043586E6C3
:1016800018220A4B1A70EDE7069B3A1DD11A074B38
:10169000D82902DD1A221A7097E60399A40061582E
:1016A0001B783960002B09D017008EE6A4020020B9
:1016B0001CCF0000902D0020FDFFFF3F2B680199FB
:1016C0001C120B40CF499B005B58170004355EE6A7
:1016D000043F039B3A68A400E250CB4B1B78002BDD
:1016E00000D072E62B68019A1C121340C54A9B0079
:1016F0009B5804354BE6039BA4001C192368043F48
:1017000038685E10FFF73CFD36180120BE4B7600AE
:101710001B7806432660002B00D056E62B68019A02
:101720001C121340B74A9B009B5804352FE6069BBA
:10173000A4003F1BB44CBB420CD82378002B00D034
:1017400043E62B68019A1C121340AE4A9B009B583B
:1017500004351CE6AD4801F0E7FE2378002B00D0ED
:1017600033E62B68019A1C121340A64A9B009B5833
:1017700004350CE6A300ED18002C00DA38E6A24B85
:101780001B78002B00D020E62B68019A1C12134016
:101790009C4A9B009B580435F9E5043F3B68042BA9
:1017A00004D1A300ED18002C00DA21E6964B1B783B
:1017B000002B00D009E62B68019A1C121340914AB5
:1017C0009B009B580435E2E5043F3B68042B04D0A2
:1017D000A300ED18002C00DA0AE68B4B1B78002BD7
:1017E00000D0F2E52B68019A1C121340854A9B0039
:1017F0009B580435CBE53E1F3068C3070AD540101F
:101800000138002809DB01234000A40018432D19EA
:101810003060EDE5FFF7B4FCF2E77B4B37001B7857
:10182000002B00D0D1E52B68019A1C121340754A99
:101830009B009B580435AAE53A00069B0C32D31A4C
:10184000D82B03DD1A22704B1A70BEE5FF2361000E
:101850005B001940FE3BFF3B194339600299069833
:101860008968241204916D1A0299AD1089782D02AD
:101870000D4303999D40091A891099401D430B435C
:10188000BB60029B7D609C70E4B2614BE4000392FC
:10189000E358029A93605C4A1278002A03D0083316
:1018A0001D00039F91E51D00019A9B680C351C12D9
:1018B0001340544A9B009B58039F68E53B1F1C68DC
:1018C000039A069B934232D10A20E30711D4042CD9
:1018D00018D90F2322681340042B16D1200001F0E1
:1018E00033FE0AF0AFFAC8239B00984200D91800D3
:1018F0000630643003F020FE00280FD1043D069B23
:10190000039375E50720042CF3D02000431E984173
:10191000FA234042FF3318400730EAE7029B2100D8
:10192000587804F023FA0023029A1370E7E7039B28
:10193000039A0C3B1B6802995B109B00D31A0C3B6B
:101940001C601F1D1300083B1B685A108A70D2B21E
:101950002F49D2005B0055589B0A029A9B00956064
:10196000ED18039B069A043B1B685B109B00D31881
:101970000393254B1B78002B00D026E52B68019A9A
:101980001C1213401F4A9B009B580435FFE43B1F69
:101990001868FFF7F5FBA40006003F1B1E2827DC94
:1019A00000280DDC184B1B78002B00D00DE52B68B0
:1019B000019A1C121340134A9B009B580435E6E41D
:1019C00001F00CFB033E361801F008FB114B801BA5
:1019D0009842F9D80C4B1B78002B00D0F5E42B680B
:1019E000019A1C121340074A9B009B580435CEE411
:1019F0000123029A137001F0F1FA029B0A3886194A
:101A00005E60F5E41CCF0000A402002048D1000075
:101A1000982500203F420F003B1F1868FFF7B0FBDE
:101A2000A40006003F1B00280DDCCF4B1B78002BC9
:101A300000D0CAE42B68019A1C121340CB4A9B00C9
:101A40009B580435A3E4CA4B984203DD1D22C64BC4
:101A50001A70BAE40123029A137001F0BFFAFA2354
:101A60009B005E43029B0A3E30185860C0E4A3000E
:101A7000FF1A002320001A003900FFF7CFFBBD4EEC
:101A8000BD4C3168200001F07FFFBC4B316818600D
:101A9000200004F00DF83168200004F06EF9B24B1C
:101AA0001B78002B00D090E42B68019A1C12134085
:101AB000AE4A9B009B58043569E4AB4BA4001B78ED
:101AC0003F1B002B00D080E42B68019A1C121340AE
:101AD000A64A9B009B58043559E4029803F090FDF8
:101AE000A14B1B78002B00D06FE42B68019A1C12CD
:101AF00013409E4A9B009B58043548E43B1F1B68DB
:101B0000002B3ED13B000C3B1B68DA072CD539007B
:101B100001225B105800083902430A60002B44DDA3
:101B2000012259001143381F016039000839096842
:101B30001141CB1A39000C390968114224D09B1885
:101B40009340A4001343039AA350874B1B78002BA8
:101B500000D03AE42B68019A1C121340834A9B0080
:101B60009B580435FFF713FC042B06D90F211A6884
:101B70000A40092A01D15B68C9E719227A4B1A7019
:101B800023E45B10013BC9E7042909D90F200A6847
:101B90000240092A04D102339B005B58A400D2E71B
:101BA0001922714B1A70FFF710FC0435CDE7A30022
:101BB000069AFB189B1AD82B13DC0122631E002CFB
:101BC00014DC694B1B78002B01D0FFF7FEFB2B6860
:101BD000019A1C121340654A9B009B580435FFF77D
:101BE000D6FB1A22604B1A70FFF7EFFB3A601C001D
:101BF0000437E3E7069A3B1D9B1A5B4ED82B03DDA7
:101C00001A233370FFF7E1FB069B039AA40093426B
:101C10002AD23B1F1868FFF7B3FA011E21DD039B90
:101C20000C3B1A68521082421BDB9007801A544BFF
:101C30004018C018039B8000C2583B1B1A604A4BD7
:101C40003F1B1B780437002B01D0FFF7BEFB2B682E
:101C5000019A1C121340454A9B009B580435FFF71C
:101C600096FB20233370EAE71823FBE7434BA400DD
:101C70001A683B1B1F001A603B4B04371B78002B74
:101C800001D0FFF7A2FB2B68019A1C121340374AC0
:101C90009B009B580435FFF77AFB3B1F1A68042A08
:101CA00011D1A4002D19304B1B78002B01D0FFF768
:101CB0008CFB2B68019A1C1213402C4A9B009B58EA
:101CC0000435FFF764FB1F00EDE73A1F1368042B90
:101CD00004D0002313603A00A4002D19224B1B7876
:101CE000002B02D01700FFF770FB2B6801991C1224
:101CF0000B401E499B005B5817000435FFF747FB5C
:101D0000A3009C46FE1A002C17DC1C22164B1A70EE
:101D1000002333606346FF1A134B04371B78002BF4
:101D200001D0FFF752FB2B68019A1C1213400F4A97
:101D30009B009B580435FFF72AFB002033685A109C
:101D40008300F15801230B4003D10D21064A117085
:101D5000DFE749108A4200DD0A0001308442EFDCEF
:101D6000012352001343D4E7A40200201CCF00003B
:101D700080EE3600C8050020A502002008000020E3
:101D8000FCFFFF3FA3009C46FE1A002C17DC1C2220
:101D9000DB4B1A70002333606346FF1AD84B0437BD
:101DA0001B78002B01D0FFF710FB2B68019A1C1247
:101DB0001340D44A9B009B580435FFF7E8FA0020F3
:101DC00033685A108300F15801230B4003D10D21D1
:101DD000CB4A1170DFE749108A4200DA0A0001306D
:101DE0008442EFDC012352001343D4E73B00083B5D
:101DF0001868FFF7C5F93B1F06001868FFF7C0F920
:101E00000023864200DA0433A4003A1B1700136053
:101E1000BB4B04371B78002B01D0FFF7D6FA2B6899
:101E2000019A1C121340B74A9B009B580435FFF7D8
:101E3000AEFA3B00083B1868FFF7A2F93B1F06000B
:101E40001868FFF79DF9F30FC217B0425341A40081
:101E50003A1B17009B001360A94B04371B78002B1B
:101E600001D0FFF7B2FA2B68019A1C121340A54A61
:101E70009B009B580435FFF78AFA3B00083B186823
:101E80003B1F1968A600BE1B0423814202D0042810
:101E900002D80023336018E001239C461842F8D191
:101EA0000F2302681A40042AF3D163461942F0D185
:101EB0000429EED90B680B321340042BE9D1FFF74C
:101EC0007FF9431E9841800030608D4BA4001B7841
:101ED0003F1B0437002B01D0FFF777FA2B68019ADC
:101EE0001C121340874A9B009B580435FFF74FFA9A
:101EF0003B00083B18683B1F1968A600BE1B002367
:101F0000814202D0042802D80423336018E0012360
:101F10009C461842F8D10F2302681A40042AF3D1D4
:101F200063461942F0D10429EED90B680B321340F5
:101F3000042BE9D1FFF744F9434258418000306057
:101F40006F4BA4001B783F1B0437002B01D0FFF719
:101F50003CFA2B68019A1C1213406A4A9B009B585A
:101F60000435FFF714FA3B00083B1868FFF708F93F
:101F70003B1F06001868FFF703F9F317C20F8642EC
:101F80005341A4003A1B17009B0013605C4B0437BD
:101F90001B78002B01D0FFF718FA2B68019A1C124E
:101FA0001340584A9B009B580435FFF7F0F93B005B
:101FB000083B1868FFF7E4F83B1F06001868FFF7B6
:101FC000DFF80023864200DD0433A4003A1B17002B
:101FD00013604B4B04371B78002B01D0FFF7F5F94A
:101FE0002B68019A1C121340464A9B009B580435EB
:101FF000FFF7CDF93B1F1B68A400043B5A1E934119
:102000003A1B17009B0013603D4B04371B78002BD5
:1020100001D0FFF7DAF92B68019A1C121340394AF4
:102020009B009B580435FFF7B2F93B00083B18684A
:10203000FFF7A6F83B1F06001868FFF7A1F8321853
:102040000120A4003B1B1F00520002431A602C4BCE
:1020500004371B78002B01D0FFF7B7F92B68019AE2
:102060001C121340274A9B009B580435FFF78FF939
:102070003B00083B1868FFF783F83B1F0600186811
:10208000FFF77EF8321A0120A4003B1B1F0052000C
:1020900002431A601A4B04371B78002B01D0FFF75C
:1020A00094F92B68019A1C121340164A9B009B5806
:1020B0000435FFF76CF93B00083B1868FFF760F840
:1020C0003B1F06001868FFF75BF802000120A40020
:1020D0003B1B1F007243520002431A60084B043737
:1020E0001B78002B01D0FFF770F92B68019A1C12A6
:1020F0001340044A9B009B580435FFF748F9C0463B
:10210000A40200201CCF00003B1F1868FFF738F81E
:10211000061E17D11F23EE4A1370A4003B1B1F009D
:102120001E60EB4B04371B78002B01D0FFF74DF9F5
:102130002B68019A1C121340E64A9B009B580435F9
:10214000FFF725F93B00083B1868FFF719F8310045
:1021500007F0AAF9012640000643DEE73B1F186896
:10216000FFF70EF8061E17D11F23D94A1370A400DB
:102170003B1B1F001E60D64B04371B78002B01D081
:10218000FFF723F92B68019A1C121340D14A9B00D8
:102190009B580435FFF7FBF83B00083B1868FEF737
:1021A000EFFF310007F066FA012649000E43DEE733
:1021B0003B1F1868FEF7E4FFC21780185040012249
:1021C000A4003B1B1F00400010431860C04B0437A5
:1021D0001B78002B01D0FFF7F8F82B68019A1C122E
:1021E0001340BC4A9B009B580435FFF7D0F8A3006E
:1021F000FE1A3068012C24D1FEF7C2FF0494079028
:1022000009F076FD0799002900DC012107F032FA78
:10221000049BA400C918012349001943AC4B3F1B80
:102220001B7831600437002B01D0FFF7CEF82B6804
:10223000019A1C121340A74A9B009B580435FFF7D4
:10224000A6F8FEF79DFF04907068FEF799FF049BC7
:102250000130C31A0793D3E7A300FE1A3100200010
:10226000049301F017FD049B3060FF1A984B04376C
:102270001B78002B01D0FFF7A8F82B68019A1C12DD
:102280001340944A9B009B580435FFF780F83B00AD
:10229000083B1868FEF774FF3B1F06001868FEF73E
:1022A0006FFF02000120A4003B1B1F0032405200C0
:1022B00002431A60864B04371B78002B01D0FFF7CE
:1022C00084F82B68019A1C121340824A9B009B5889
:1022D0000435FFF75CF83B00083B1868FEF750FF39
:1022E00006003B1F1868FEF74BFF32000243012037
:1022F000A4003B1B1F00520002431A60744B0437BA
:102300001B78002B01D0FFF760F82B68019A1C1294
:102310001340704A9B009B580435FFF738F83B0088
:10232000083B1868FEF72CFF06003B1F1868FEF7F5
:1023300027FF320042400120A4003B1B1F00520037
:1023400002431A60624B04371B78002B01D0FFF761
:102350003CF82B68019A1C1213405E4A9B009B5864
:102360000435FFF714F83B1F1868FEF709FFC04358
:102370000122A4003B1B1F00400010431860544B77
:1023800004371B78002B01D0FFF71FF82B68019A48
:102390001C1213404F4A9B009B580435FEF7F7FF71
:1023A0003B00083B1868FEF7EBFE06003B1F186871
:1023B000FEF7E6FE3200824051000122A4003B1BE2
:1023C0001F000A431A60424B04371B78002B01D0D0
:1023D000FEF7FBFF2B68019A1C1213403D4A9B003D
:1023E0009B580435FEF7D3FF3B00083B1868FEF707
:1023F000C7FE06003B1F1868FEF7C2FE320002410E
:1024000051000122A4003B1B1F000A431A60304BFD
:1024100004371B78002B01D0FEF7D7FF2B68019AF9
:102420001C1213402B4A9B009B580435FEF7AFFF4C
:102430003B000C3B1868FEF7A3FE3B00083B060080
:102440001868FEF79DFEF1170200C317300007F071
:1024500063F93B1F049005911868FEF791FE020096
:102460000498059907F00CF943000120A4003E1BD5
:1024700037001843164B30601B780437002B01D00F
:10248000FEF7A3FF2B68019A1C121340114A9B0010
:102490009B580435FEF77BFFA300FE1A3100200095
:1024A0000493FEF7B5FC049B3060FF1A084B043719
:1024B0001B78002B01D0FEF788FF2B68019A1C12B5
:1024C0001340044A9B009B580435FEF760FFC0464A
:1024D000A40200201CCF0000A300FF1A3900200036
:1024E000FEF7AEFCE44B1B78002B01D0FEF76DFF2E
:1024F0002B68019A1C121340E04A9B009B5804353C
:10250000FEF745FFA300FE1A310020000493FEF7FA
:10251000D7FC049B3060FF1AD74B04371B78002B85
:1025200001D0FEF752FF2B68019A1C121340D34AC8
:102530009B009B580435FEF72AFFA300FF1A3900C1
:102540002000FEF751FDCC4B1B78002B01D0FEF78D
:102550003CFF2B68019A1C121340C84A9B009B58F1
:102560000435FEF714FFA300FE1A31002000049387
:10257000FEF7ACFD049B3060FF1ABF4B04371B789D
:10258000002B01D0FEF721FF2B68019A1C1213408B
:10259000BA4A9B009B580435FEF7F9FE3B1F1868AA
:1025A00000F0D2FF3A00083A12680300A400D107F5
:1025B00029D4042A0CD910680F22104001380828A9
:1025C0000FD806F0DDFE052026220E0E0E0E24008A
:1025D000AB49180009F02CFC434258413B1B8000DA
:1025E0001860A54B3F1B1B780437002B01D0FEF76A
:1025F000ECFE2B68019A1C121340A04A9B009B58CA
:102600000435FEF7C4FE9F49E3E79F49E1E79F4990
:10261000DFE79F49DDE7069B3E1DF31A964CD82B5A
:1026200003DD1A232370FEF7D0FE00F0E1FC430027
:102630000120184323783860002B02D03700FEF7C2
:10264000C4FE2B68019A1C1213408C4A9B009B58B5
:1026500037000435FEF79BFE069B3E1DF31A864CA1
:10266000D82B03DD1A232370FEF7AFFE00F0B6FC73
:10267000884B400018400123184323783860002B12
:1026800002D03700FEF7A1FE2B68019A1C121340FE
:102690007A4A9B009B5837000435FEF778FE069B6C
:1026A0003E1DF31A744CD82B03DD1A232370FEF75A
:1026B0008CFE00F09DFC784B1A68831A904201D280
:1026C000764A9B1801205B0003433B602378002B74
:1026D00002D03700FEF779FE2B68019A1C121340D6
:1026E000664A9B009B5837000435FEF750FE00F009
:1026F0007FFC694BA40018605F4B3F1B1B78002BCD
:1027000001D0FEF762FE2B68019A1C1213405B4A4F
:102710009B009B580435FEF73AFE0123A600BE1B22
:1027200020001A003100FEF779FD5D4C206864300E
:1027300002F002FF002802D1043DFEF759FE029B81
:1027400021685A78574803F026FB0123029A370084
:10275000137000F043FC544B22681B68063253434D
:102760001818029B5860FEF743FEA600BE1B20000F
:10277000012300223100FEF751FD494C20686430EE
:1027800002F0DAFE0028D7D0464803F081F8DCE7F3
:10279000A4003E1BFEF7C2FD3700374B30601B78AC
:1027A0000437002B01D0FEF710FE2B68019A1C1293
:1027B0001340324A9B009B580435FEF7E8FD2E4B30
:1027C000A4001B783F1B002B01D0FEF7FEFD2B68F9
:1027D000019A1C121340294A9B009B580435FEF7AE
:1027E000D6FDA4003E1B300000F035FC3700224B24
:1027F00030601B780437002B01D0FEF7E6FD2B6814
:10280000019A1C1213401D4A9B009B580435FEF789
:10281000BEFDA4003E1B300000F01FFC3700164B2D
:1028200030601B780437002B01D0FEF7CEFD2B68FB
:10283000019A1C121340114A9B009B580435FEF765
:10284000A6FDA300FE1A31002000049300F008FC4E
:10285000049B3060FF1A084B04371B78002B01D013
:10286000FEF7B3FD2B68019A1C121340034A9B002C
:102870009B580435FEF78BFDA40200201CCF0000FE
:1028800058D1000060D1000067D100006ED1000077
:1028900073D10000FEFFFF7FD00500203789410083
:1028A000C8050020A502002004000020A4003F1B52
:1028B000380000F00BFCFB4B1B78002B01D0FEF71F
:1028C00084FD2B68019A1C121340F74A9B009B5809
:1028D0000435FEF75CFDA300FE1A310020000493CE
:1028E00000F01CFC049B3060FF1AEE4B04371B7891
:1028F000002B01D0FEF769FD2B68019A1C121340D2
:10290000E94A9B009B580435FEF741FDA4003F1B9C
:10291000380000F045FCE34B1B78002B01D0FEF79C
:1029200054FD2B68019A1C121340DF4A9B009B58F0
:102930000435FEF72CFD0121200000F019FCD94BD5
:102940001B78002B01D0FEF740FD2B68019A1C126A
:102950001340D54A9B009B580435FEF718FD002113
:10296000200000F005FCCF4B1B78002B01D0FEF7B8
:102970002CFD2B68019A1C121340CB4A9B009B58DC
:102980000435FEF704FDA4003E1B300000F02AFCD5
:102990003700C44B30601B780437002B01D0FEF7A2
:1029A00014FD2B68019A1C121340BF4A9B009B58D0
:1029B0000435FEF7ECFCA4003E1B300000F026FCC2
:1029C0003700B84B30601B780437002B01D0FEF77E
:1029D000FCFC2B68019A1C121340B34A9B009B58C5
:1029E0000435FEF7D4FCA4003F1B380000F0E8FBE0
:1029F000AC4B1B78002B01D0FEF7E7FC2B68019A4B
:102A00001C121340A84A9B009B580435FEF7BFFCDC
:102A1000A4003F1B380003F009FDA24B1B78002BDC
:102A200001D0FEF7D2FC2B68019A1C1213409E4A7B
:102A30009B009B580435FEF7AAFCA4003E1B300007
:102A400003F0A4FD3700974B30601B780437002B50
:102A500001D0FEF7BAFC2B68019A1C121340924A6F
:102A60009B009B580435FEF792FCA4003F1B3800E6
:102A700003F080FC8B4B1B78002B01D0FEF7A5FCEC
:102A80002B68019A1C121340874A9B009B580435FF
:102A9000FEF77DFCA4003E1B300003F081FC3700F4
:102AA000804B30601B780437002B01D0FEF78DFC83
:102AB0002B68019A1C1213407B4A9B009B580435DB
:102AC000FEF765FCA300FF1A3900200001F026FC88
:102AD000744B1B78002B01D0FEF777FC2B68019A12
:102AE0001C121340704A9B009B580435FEF74FFCA4
:102AF000A300FF1A3900200001F024FA694B1B786B
:102B0000002B01D0FEF761FC2B68019A1C121340C8
:102B1000654A9B009B580435FEF739FCA300FF1A59
:102B20003900200001F032FB5E4B1B78002B01D0F6
:102B3000FEF74BFC2B68019A1C1213405A4A9B006B
:102B40009B580435FEF723FCA300FF1A3900200030
:102B500001F044FB534B1B78002B01D0FEF735FCF2
:102B60002B68019A1C1213404F4A9B009B58043556
:102B7000FEF70DFCA300FE1A31002000049303F0C1
:102B800065FD049B3060FF1A464B04371B78002B11
:102B900001D0FEF71AFC2B68019A1C121340424A1E
:102BA0009B009B580435FEF7F2FBA300FE1A310090
:102BB0002000049303F052FD049B3060FF1A394B50
:102BC00004371B78002B01D0FEF7FFFB2B68019A1E
:102BD0001C121340344A9B009B580435FEF7D7FB68
:102BE000A300FE1A31002000049303F03FFD049B74
:102BF0003060FF1A2B4B04371B78002B01D0FEF7F7
:102C0000E4FB2B68019A1C121340274A9B009B5837
:102C10000435FEF7BCFBA300FE1A3100200004932C
:102C200003F02CFD049B3060FF1A1E4B04371B7809
:102C3000002B01D0FEF7C9FB2B68019A1C12134030
:102C4000194A9B009B580435FEF7A1FBA300FF1A0D
:102C50003900200001F0AEF9124B1B78002B01D097
:102C6000FEF7B3FB2B68019A1C1213400E4A9B001F
:102C70009B580435FEF78BFBA300FF1A3900200098
:102C800001F0D4FA074B1B78002B01D0FEF79DFB17
:102C90002B68019A1C121340034A9B009B58043571
:102CA000FEF775FBA40200201CCF0000A300FE1A53
:102CB00031002000049301F035FA049B3060FF1AC4
:102CC000304B04371B78002B01D0FEF77EFB2B68BE
:102CD000019A1C1213402C4A9B009B580435FEF7A6
:102CE00056FBA300FF1A3900200001F0E3F9254B41
:102CF0001B78002B01D0FEF768FB2B68019A1C1291
:102D00001340214A9B009B580435FEF740FB069B6D
:102D1000029AFB1A9B101361A300FF1A39002000CE
:102D200002F0F4FD174B1B78002B01D0FEF74DFB92
:102D30002B68019A1C121340134A9B009B580435C0
:102D4000FEF725FB069B029AFB1A9B101361A3005A
:102D5000FE1A31002000049302F0D8FD049B30607D
:102D6000FF1A084B04371B78002B01D0FEF72DFB10
:102D70002B68019A1C121340034A9B009B58043590
:102D8000FEF705FBA40200201CCF00000023F7B5CE
:102D90005A1E0192002B07DA01F0D6FA02F0E6FE85
:102DA00003F058F81923019300263000194B1968D5
:102DB000B14212DD184B1A6801328A420FDAF02450
:102DC0001A601D68154F6C43E35D002B1FD0E4199A
:102DD000022B06D12000FEF7B9FA019BD8E70022AA
:102DE000EDE7012B0DD1002801D100F0F7F8F0221A
:102DF0006A43BB185B680A49C31A8B4201D8022395
:102E0000BB54F0235D43054BEB5C022BE2D0013653
:102E1000CCE7C046CC05002000000020381C002074
:102E20003F420F00012200210A4B0B481A61195042
:102E300004301950A2210420C9005850C121C020DB
:102E40008900800258501A60044BFC311960044B11
:102E50001A70704700A000400405000000E100E087
:102E6000F505002004207047F8B550C90123220061
:102E70001A40101E2DD03340181E2AD06410002096
:102E80001A2C26D81D4B761035009E4200DD1D0001
:102E90001B4F3B5D012B05D00121200004F048FEB3
:102EA00001233B55174B1B78002B01D1FFF7BAFFCD
:102EB0000023154A9E420DDCFF2514491448D65CB8
:102EC000B44202D15E007052D5540133042BF6D1C6
:102ED0000420F8BDD15C8C4203D10C4A5B009D52AA
:102EE000F6E70133042BF5D10023D15CFF2901D192
:102EF000D454F2E70133042BF7D1E9E7881300003B
:102F0000D8050020F50500201C0000200E00002040
:102F1000DC05000070B530C9012322001A40101EE4
:102F20001BD02B40181E18D064101A2C00D919245D
:102F3000174E335D012B05D00121200004F0F8FD70
:102F40000123335569100800124A1038124B904281
:102F500004D9012252421A60042070BD1C600F483F
:102F600006F0A2FA0E4B18800E4B1B78002B02D1F4
:102F7000FFF758FFF0E701220B4B9A64A922D20019
:102F80009A588018A82280B2D2009850E4E7C04630
:102F9000D8050020908601001800002020A107001D
:102FA0000C000020F505002000A00040030010B533
:102FB0000120002B02DC1B30FEF7AAF910BD042013
:102FC000704710B5002803DC1C20FEF7A1F910BDE6
:102FD0000B680020DB07FAD40D30F6E70122034B23
:102FE0001A64A822D20098587047C046008000405A
:102FF00010B5FFF7F3FFFA21890006F0CBF910BDF9
:1030000000487047D8D100001B20704770B5054EAE
:103010000400335C0D008B4202D004F089FD35556D
:1030200070BDC046D805002070B50024084D635D12
:10303000012B09D10021200004F0A0FD0021200077
:1030400004F076FD0023635501341B2CEED170BDD6
:10305000D8050020704711207047372070470000C6
:10306000F8B501240B6806000D00234204D10D20A1
:10307000FEF74EF92000F8BD5B1004D103F09EF975
:1030800040002043F7E72000072BF4D80D4A9B00AF
:103090009C580D4F3B5D002B05D00021200004F013
:1030A00047FD00233B55012E06DD6B68042B03D141
:1030B0000221200004F03CFD200004F0E7FB012485
:1030C0004000DEE7B8D10000D8050020F8B50126A1
:1030D0000568354202D04468344203D10D20FEF722
:1030E00017F9F8BD6D101A2DFBD80A4F7B5D012B27
:1030F00004D03100280004F01BFD7E550649641001
:103100008C4202DCE143C9172140280004F044FC52
:10311000E7E7C046D8050020FF03000070B5012492
:103120000D68254204D10D20FEF7F2F8200070BD95
:103130006D101A2D17D80024012804DD4C68043CBA
:1031400063425C416400094E735DA34204D02100D8
:10315000280004F0EDFC7455280004F02DFD030058
:103160000420012BE3D00020E1E7C046D805002071
:1031700070B504000D001A280ED8084E335C012BE0
:1031800004D0012104F0D4FC012333552900200090
:103190004D1EA94104F0F2FC70BDC046D8050020C8
:1031A000036810B5DA0703D40D20FEF7B1F810BD9F
:1031B0004168581004394A425141FFF7D9FFF6E7F8
:1031C00037B569460A00064B30CB30C2036802208F
:1031D000042B02D100F0DAFF37BD00F0FFFFFBE760
:1031E00080D1000010B5084C237D002B05D00021B4
:1031F000142004F09DFC00232375142004F0DCFC53
:1032000043425841800010BDD805002010B5084C3D
:10321000A37D002B05D00021162004F089FC00239B
:10322000A375162004F0C8FC43425841800010BD2D
:10323000D805002070470000F7B5304D304E6B6C5C
:10324000002B15D0A8240023E40037596B642D4BC4
:10325000186800280CDB2C4B19784A425141C9B23E
:10326000197004F08BFC294B1B88DF19BFB2375152
:10327000AB6C002B39D00021254B264FF458A964A4
:103280003A780C340193244D8A4206D02B68032BE4
:1032900003D8224AD05C04F071FC2B68204A013329
:1032A000134004D50422013B5242134301331B490E
:1032B00000228C462B60042B18D06046C05C591C41
:1032C000FF2802D10B000122F5E7002A00D02B6075
:1032D000012104F053FC01233B702B68114A5B0071
:1032E0009B5AE418019BA4B2F450F7BD01235B4242
:1032F0002B6000233B700C4BF3E7C046FCA0004062
:1033000000A0004018000020F40500200C00002060
:1033100044050000F3050020D40500201C00002017
:10332000030000800E00002050460000084B094AB0
:10333000FF201A805A809A80DA800023064A0749C3
:103340001370074A087048708870C870136070471F
:103350000E000020DC050000F30500201C0000200A
:10336000D40500200122024B52421A607047C04629
:103370001800002010B5034A0621034802F0A2F805
:1033800010BDC04688D10000FAD80000E12170B518
:103390004902194803F0EEFF002401220320174BD5
:1033A00017491A615C500431585080180831585040
:1033B0001A60063004F064FAFF21124AA154013465
:1033C0001B2CFBD1012200200F4B01001A600423AB
:1033D0000E4A0F4D1468002CFCD02C680002013BF3
:1033E00020431160002BF5D101220A4B1A6004F032
:1033F0007DF901F0F5F870BDC01B00200080004091
:1034000004050000D805002000D0004000D1004095
:1034100008D5004004D00040F8B50B4E070030003E
:103420000D0003F0EFFF0400A84200DD2C003D007A
:10343000EB1B9C4205DD300003F0EEFF28700135E8
:10344000F6E72000F8BDC046C01B002010B5010003
:10345000014803F097FF10BDC01B002010B5054CBC
:10346000200003F09DFFE1212000490203F082FFCC
:1034700010BDC046C01B0020C3070CD4064B1B6800
:10348000834208D8054B1B68984204D8031F1B6869
:10349000002B00D01800704700060020FC0500201B
:1034A0000023012210B50A48990001334250642BD1
:1034B000FAD1084C084B00211A602000074A08F096
:1034C00037F9074B074A6360074B1A6010BDC046C7
:1034D000902D00200406002008000020D4090000E0
:1034E0003027000008060020F805002010B5044B26
:1034F000044A1A60044B054A1A60FFF7D1FF10BD59
:103500000006002004060020FC050020D80F002043
:10351000044B1B681868000980B20238C343DB17EC
:1035200018407047F805002000B59BB0020005491F
:1035300001A808F041FC01A802F0C6F902F08AFCDB
:10354000FCE7C0465BD200000B4BC20704D4042842
:1035500004D80A4B00D00A4B180070470F220368AA
:103560001A40031D042AF7D0064B092AF4D0064B53
:10357000032AF1D0054BEFE735D20000D2CD000091
:10358000CCCD00003FD200004FD2000046D2000058
:103590000020064A0649131F186013681B099BB2D6
:1035A00002339B00D2188A42F5D3704708060020E8
:1035B000D80F0020F7B50F240126314B314A196886
:1035C000314B324D186813681F002740072F26D84B
:1035D00013681B099BB202339B00D218AA42F2D394
:1035E00000242B4EA500AD192868FFF745FF0134D4
:1035F0002860642CF6D1274C2068FFF73DFF20603F
:10360000254C2068002802D0FFF736FF20600025F7
:10361000224B1B680093009B9D4214DBF7BD1B09E6
:103620009BB29B00D3189A42D2D01F68374208D170
:10363000B94206D2B84204D3043F3F68002F00D0FD
:103640001F60043BEFE7F0236B43154A9B181A7881
:10365000002A01D10135DEE71F693C2300266B43B8
:10366000DB199B0001930136BB1BF3D4019BB40013
:103670001C1B0B4B1C19A069FFF7FEFEA061F2E7B3
:103680000006002008060020FC050020D80F0020BE
:10369000902D002008000020D80F0020CC0500202D
:1036A000381C0020F7B50124204246D1234B1B686B
:1036B0009C46984241D3224B1B68019398423CD8C8
:1036C000031F1B68002B38D10200036800941B09FC
:1036D0009BB2002B0FD10099131F196090422CD080
:1036E00015682B1F1B68990069180C68013B146052
:1036F0000A602A00EDE79D0055192968009C2142C7
:1037000019D18C4517D8019C8C4214D30E1F3468F4
:10371000002C10D10F680F343C40072C08D92F60C3
:10372000151F2B600B680A601B099BB20A00D0E7CB
:1037300000993160CDE7013BCBE7F7BD00060020E3
:10374000FC0500200D4970B50A000D4D1368141FCB
:103750001B0926689BB2981C002E0BD000238A42BE
:1037600000D00B0023608300C91880001218AA4201
:10377000ECD370BD1B011360F7E7C04608060020BC
:10378000D80F0020F8B5124C27000F223B681D0906
:10379000ADB213420DD06E1CB600A74204D0320069
:1037A0003900200007F0B1FF0022A3190436A41944
:1037B0001A600235AD00074B7F199F42E5D31B1BF2
:1037C0009B10013B1B012360034B1C60F8BDC046EE
:1037D00008060020D80F0020F8050020F0B59BB0A7
:1037E000FFF7FCFB00240700214AA300D058013456
:1037F000FFF758FF642CF7D11E4B1868FFF752FFF4
:103800001D4B1868002801D0FFF74CFF00261B4B0A
:103810001B689E4217DBFFF795FFFFF7CBFEFFF714
:10382000B1FFFFF7DBFB164BC21B1B6815491B687A
:1038300001A81B099BB2023B08F0BEFA01A802F0E6
:1038400043F81BB0F0BDF02575430F4BED182B78F6
:10385000002B01D10136DAE72B695C1E002CF9DB65
:10386000A300EB189869FFF71DFF013CF6E7C0467F
:10387000902D002008000020D80F0020CC0500204B
:10388000F805002015D20000381C0020F7B5174DB0
:103890004F1C2B6806001B680C001B099BB2019291
:1038A0009F420BDBFFF79AFF2B681B681B099BB23B
:1038B0009F4203DB0A20FDF72BFDFEBD2868A71CF5
:1038C000BA00DB1B81181B010B6029600021031F5C
:1038D00019600F231E4003002401264340C3083A09
:1038E0009A189A42E9D9019902C3FAE7F80500202B
:1038F000F7B503000122134004000D000193002BD3
:103900002BD1174B1B68834227D8164B1B68834269
:1039100023D90F23144F386000681840FFF7B6FF13
:10392000019B3C68061E3B6017D0236804301B09CE
:103930009BB29D4200DD1D00AA00211D251F07F03E
:10394000DBFEFFF725FE2E60FFF734FE00232B6021
:103950002268064B1340236034002000FEBDC046A1
:1039600000060020FC050020D80F0020F0FF0F000B
:103970000323043010B5C11719400918891000221B
:103980000420FFF783FF10BD70B5050008000C0090
:10399000FFF7EEFF0023002804D170BDE95CC218D8
:1039A00011710133A342F9DBE343DB171C40002311
:1039B00004192371F1E7F0B50C009BB0022804DC78
:1039C0001C20FDF7A5FC1BB0F0BD012308681842C0
:1039D00006D1042804D90F2601683140042901D0FA
:1039E0000E20EEE761680D001D40F9D10429F7D9DA
:1039F0000A683240042AF3D1A2681A4201D10D208C
:103A0000DFE7FFF7A1FD06006068FFF79DFDA768EF
:103A1000010001AC7F103000257003F042F839003E
:103A20006423220003F0A2F8200008F00BFA010042
:103A30002000FFF7A9FFC6E710B51C4CA544041EE3
:103A400002D1FFF795FF0BE002F044FF0138062892
:103A500028D805F095FC0909111829042400002034
:103A60008023DB009D4410BD200002F0AFFF011B4E
:103A70002000FFF789FFF3E7200002F055FF430025
:103A800001201843ECE780226946D200200002F0B2
:103A900062FF684608F0D6F901006846E9E70421AC
:103AA0000348E6E70020CCE70420D9E700FCFFFF4D
:103AB000A4D2000070B50C00022803DC1C20FDF726
:103AC00027FC70BD01230868184206D1042804D9D8
:103AD0000F2501682940042901D00E20EFE7616815
:103AE0001942FAD10429F8D90A682A40042AF4D1E3
:103AF000A2681A4201D10D20E1E7FFF725FD05007C
:103B00006068FFF721FDA46801006410280002F03E
:103B1000C8FF210003F005F8FFF78EFFD1E770B56D
:103B20000D00012803DC1C20FDF7F2FB70BD012411
:103B30000868204206D1042804D90F2102680A40EF
:103B4000042A01D00E20EFE76A682242FAD1042A43
:103B5000F8D913680B40042BF4D1FFF7F5FC0600ED
:103B60006868FFF7F1FC0100300002F09AFF03F0F3
:103B70001CF840002043D9E7F8B507000C001C20D2
:103B8000012F0BDD01250868284206D1042804D93D
:103B90000F2102680A40042A03D00E20FDF7B8FB6B
:103BA000F8BD62682A42F8D1042AF6D913680B409E
:103BB000042BF2D1FFF7C8FC06006068FFF7C4FCD5
:103BC0000100022F14D0A4682C4211D064103000E0
:103BD00002F067FF050002F07DFE012811D1002CE4
:103BE00002DD0135012C06D12800FFF725FFD7E7BC
:103BF00001246442EBE7280002F0F4FE013C0500DA
:103C0000F0E70228F0D1002CEEDD0135012CEBD0DD
:103C100000222800110002F017FF02F0E3FE013C31
:103C20000500F3E710B501240868044016D04410DD
:103C3000200005F0CDFE154905F098FD07F07EFC4B
:103C400004F0D0F80022124B06F032FE04F072F8B5
:103C500007F004FC43000120184310BD042810D9CC
:103C60000F2302681340042B07D1FFF76DFC2100DE
:103C70000A2208F0AFF90400DAE7032B01D104307F
:103C8000F5E70D20FDF744FBD2E7C046D3023739F4
:103C90000000D040086870B501240500254006D119
:103CA000042804D90F2302681340042B03D00E20EC
:103CB000FDF72EFB70BDFFF747FC03782900233B7F
:103CC0005A4253411022C01808F084F980239B0502
:103CD000C218044B9A4201D91420E9E7400020435E
:103CE000E8E7C046FFFFFF3F10B5034A062103483F
:103CF00001F0E8FB10BDC04674D200006CD2000099
:103D00000020704710B51E20FDF702FB10BD10B556
:103D10001E20FDF7FDFA10BD10B51E20FDF7F8FAC4
:103D200010BD10B51E20FDF7F3FA10BD10B51E2012
:103D3000FDF7EEFA10BD10B51E20FDF7E9FA10BD33
:103D400010B51E20FDF7E4FA10BD10B51E20FDF7DA
:103D5000DFFA10BD10B51E20FDF7DAFA10BD10B560
:103D60001E20FDF7D5FA10BD10B5034A0B210348FC
:103D700001F0A8FB10BDC046E0D2000038D300001F
:103D80000120034B1860034B1B68834018437047A6
:103D9000FC0F0020DC0F0020F0B5EFF310810123B1
:103DA000194083F31088134C134AA4461268134E2B
:103DB000013A9340124F134A002B17D01468034264
:103DC0000FD03D682C60C046C046C046C046C046C5
:103DD000C046C046C0460C4C1568246825605B0888
:103DE000EAE765462C6014683460F8E781F31088D0
:103DF000F0BDC04608050050200000200C05005012
:103E0000E80F0020F00F0020E40F002030B585B04F
:103E100001AD0C220649280007F06EFC0024285D45
:103E200001210134FFF7F2F80C2CF8D105B030BDB8
:103E3000CDD30000F7B56A463B4B01AE1380062395
:103E400093703A4B33800F23B370FFF7C7F8384BAA
:103E5000384DC0182B68984201D200232B602C6883
:103E6000002C41D1375D01213800FFF7CFF8013434
:103E70000021380003F082FE032CF3D10024012737
:103E80006B461E5D39003000FFF7C0F80134390081
:103E9000300003F073FE032CF2D1C8200138C04675
:103EA000C046C046C046C046C046C046C046C046E2
:103EB000C046C046C046F1D16B4600211878FFF7D6
:103EC000A5F86B4600215878FFF7A0F86B46002153
:103ED0009878FFF79BF8FFF781F8FA2300241B017D
:103EE000C01828602000FEBDFFF778F82B6800247A
:103EF0009842F7D3042003F0C9FC0600052003F024
:103F0000C5FC3618062003F0C1FC0B4B9B1B181A8E
:103F10000A4BA04206DB18600023094A2B6013609D
:103F20000124DFE71C60F7E7040500000D0E000028
:103F300010270000F40F002043030000DC0F0020D6
:103F4000FC0F00200022054B10B51A60044B1B68C3
:103F5000934201D002F05EFC002010BDF80F00205B
:103F6000E41A002010B5041E10DA1A240A4BA4002B
:103F7000E25801239340094A09491360094A116034
:103F8000094A0A4911600A4A136010BDFFF73CF85C
:103F9000A042EADDEAE7C046F4E00000F00F0020AE
:103FA00008050050E80F0020E40F00200C05005029
:103FB00018050050F0B53B4B85B01B680C00002B7A
:103FC00003D101204042FFF7CDFF246801222700E2
:103FD000174028D0FF236012184033496714661039
:103FE00040431F401E4005F05FFA050438002E498B
:103FF000784305F059FA0002054330002A4970431E
:1040000005F052FA294B28431B68202B06D1640087
:10401000A40E274BA400E35800021843FFF7BCFE90
:10402000002005B0F0BD042CFAD90F2321680B4005
:10403000092BF5D1636803925B100193019B9F42AA
:10404000EEDABB00E3189E68039B1E4228D0FF23D4
:104050007012184072101A401349751440431D40E5
:10406000009205F021FA030428000F4968430293E7
:1040700005F01AFA029D0002054300980A494043E0
:1040800005F012FA094B28431B68202B06D1760055
:10409000B60E074BB600F55800022843FFF77CFE2A
:1040A0000137CBE7F00F0020590600002000002068
:1040B000B4D500000200086810B5C3070FD5401042
:1040C0001823012A03DD4A68042A00D10833054A6F
:1040D0001360FEF7BFFFFFF745FF002010BD012072
:1040E0004042EDE72000002010B50124044002D03A
:1040F0004410200010BD042810D90F23026813407B
:10410000042B07D1FFF720FA21000A2207F062FFF3
:104110000400EEE7032B01D10430F5E70D20FDF795
:10412000F7F8E6E70868F8B5C3071AD5FFF7DCFF2C
:104130000300203B5E2B25D80520434301221D1898
:104140000020114E9D4219D005211024F75C3C42FD
:1041500000D080180139520064100029F7D10133D2
:10416000F0E704280ED90F2203681A40042A09D167
:104170001B099BB2002B05D00379DAE7012340002D
:104180001843F8BD0120FCE7D9D3000070B50868DA
:104190000D00FFF7A9FF04006868FFF7A5FF621E86
:1041A0000100042A14D8451E042D11D805236B43A1
:1041B0009B18012215009D402B00064805682B43E3
:1041C0000360054B1B68002B02D0200002F023FB8C
:1041D000002070BDF80F0020E41A002070B50868B8
:1041E0000D00FFF781FF04006868FFF77DFF621E86
:1041F0000100042A13D8451E042D10D805236B4353
:104200009B1801229A400748036893430360064BBA
:104210001B68002B03D00022200002F0FCFA0020D3
:1042200070BDC046F80F0020E41A0020F0B505006C
:1042300089B008680C00FFF757FF0690022D36DDA5
:104240006068FFF751FF0190A068FFF74DFF040081
:104250000127231D661E0793731C0293079B9E4232
:1042600035D0052373430593019B019D05330493CA
:10427000049BAB421ED0042E16D86B1E042B13D801
:104280000122059B2349013B5B199A409446224A2F
:104290000B681068069A3A4003920DD062461A43A2
:1042A0000A60012200280DD17F000135E0E70124DA
:1042B0000194CDE7029ECFE7624693430B6000284E
:1042C000F2D0039A0299280002F0A5FAECE7019BCC
:1042D0001E1D042E1AD8012C18D1002505273B00DD
:1042E00021006B439B1999400B000A4A0135116864
:1042F0009943094B11601B68002B05D0019B0022DC
:10430000581D290002F087FA052DE8D1002009B0D8
:10431000F0BDC046F80F0020E41A0020086810B570
:10432000C30703D5FFF7E0FE054B1860054B1B687C
:10433000002B03D0024B186802F06EFA002010BD6B
:10434000F80F0020E41A00207FB5A04C2368002B52
:104350000AD19F4A1268002A06D19E4B1B68002B87
:1043600001D0FFF767FD7FBD9B4D2A68002A26D14B
:10437000984A1268002A1BD0FFF75CFD0028F2D093
:10438000FFF744FD924B24681A681C60002A16D07F
:10439000002C14D101AD0C229049280007F0ACF993
:1043A000285D00210134FEF731FE0C2CF8D1DAE74C
:1043B000874A1268002AE5D1002BE3D0E0E700210C
:1043C0000D2003F0DBFB00210E2003F0D7FB0021C2
:1043D0000F2003F0D3FB2E68012E5DD0022E00D1FA
:1043E000A2E0002E51D101363100794C042023681F
:1043F000994303F0C3FB04212368052019404B4275
:10440000594103F0BBFB10212368062019404B42A1
:10441000594103F0B3FB80212368090119404B4245
:1044200059410C2003F0AAFB80212368090219409E
:104430004B4259410B2003F0A1FB80212368490224
:1044400019404B4259410A2003F098FB8021236810
:10445000890219404B425941092003F08FFB80210A
:104460002368C90219404B425941082003F086FBDA
:10447000802321681B0319404B425941072003F058
:104480007DFB31000D2003F079FB2B680321581CC4
:1044900005F0F0F8296066E702214D4C07202368FB
:1044A00019404B42594103F069FB08202168014043
:1044B0004B42594103F062FB80212368C900194037
:1044C0004B425941052003F059FB802123684901E3
:1044D00019404B425941062003F050FB80212368CC
:1044E000C90119404B425941042003F047FB802188
:1044F0002368890319404B4259410A2003F03EFBCF
:10450000802321681B0419404B425941092003F0C4
:1045100035FB31000C2003F031FB31000B2003F0A0
:104520002DFB31000E20AEE72021294C0720236807
:1045300019404B42594103F021FB402123680820D8
:1045400019404B42594103F019FB8021236809208F
:1045500019404B42594103F011FB80212368490067
:1045600019404B4259410A2003F008FB802123687F
:10457000890019404B4259410B2003F0FFFA80217A
:104580002368890119404B4259410C2003F0F6FA87
:1045900080212368490319404B425941062003F00A
:1045A000EDFA80212368C90319404B425941042088
:1045B00003F0E4FA802321685B0419404B4259411F
:1045C000052003F0DBFA01210F205CE7F80F002043
:1045D000EC0F0020FC0F0020E00F0020CDD30000E6
:1045E000012010B54042FFF7BDFC0020FFF7D4FBCF
:1045F00010BD000010B5034A0921034800F062FF16
:1046000010BDC046B4D60000FCD600008023F0B533
:1046100002255B051A690A4C0A4BA1261D51032786
:104620008025F600ED00BA43884202D300221A51D9
:10463000F0BD5F59002FFCD098518018F4E7C046B8
:104640000405000000E0014010B5002806D1C0209C
:10465000B02140028902FFF7D9FF10BDB0208021B0
:104660008002C902F7E7000043425841064B40422E
:104670001840B0239B02C018036800201A0E532A6A
:1046800001D11B02180A704700C0FEFF30B501249B
:104690008025054B054AED009C505C59002CFCD050
:1046A00001600021995030BD00E001400405000088
:1046B00043425841074B40421840B0239B02C01868
:1046C000A62310B50902DB05090A1943FFF7DEFF2F
:1046D00010BDC04600C0FEFFF0B5012480260D4B82
:1046E0000D4DF6005C51002902DC00225A51F0BD4C
:1046F000577814783F022743947824042743D478CA
:10470000043224063C439F59002FFCD010C00139CD
:10471000E9E7C04600E001400405000070B505006F
:104720004B680A009C1C2100A400FFF7D5FF281944
:1047300070BD0000134B1B68002B0CD08022B023EF
:10474000D2029B0200280BD11A1D5B681B0E522B54
:1047500000D110007047B022C02392025B02F1E743
:1047600082420DD903681B0E522B09D143680233D4
:104770009B00C018824203D903681B0E522BE9D05C
:104780000020E7E700110020F0B50020B7B00024BA
:10479000FFF7D0FF270005002600002D2ED1284D61
:1047A0002868FFF761FF32003B0001900094254923
:1047B00004A807F001FB04A801F086F8224B64204E
:1047C0001C682B68A0215A425341204A5B42134087
:1047D000B02292029B18E41A6043490204F064FE7E
:1047E000A0225202030000921949220004A807F0F7
:1047F000E3FA04A801F068F837B0F0BDFF226B6857
:1048000029689C460233FF180B12013613409C4264
:1048100000DA1C00FF200A140240039262460140A5
:1048200001920091039A0B4904A807F0C5FA04A865
:1048300001F04AF82800FFF77DFF0500ADE7C0460C
:104840000011002006D800000411002000C0FEFF67
:10485000B0D70000F2D7000070B50020FFF704FFCA
:1048600004000120FFF700FF844200DA04000A4B35
:104870001D686A42554128001D60FFF7E5FEA02231
:104880006B4252021340054A28009B18044A611CDF
:104890001360FFF70DFF70BD0011002004800100C0
:1048A00004110020F8B50020FFF7DEFE070001200C
:1048B000FFF7DAFE3E00204D0643204C0DD180214B
:1048C000C020C9024002FFF7A1FE01213000FFF71E
:1048D000EFFE1B4B2E6023601DE0874209DD0023A5
:1048E000B0212B60164B890223602368002001252C
:1048F00017E0012380212B60124BC9022360F4E7EB
:10490000120E522A08D0002800D023600E4800F072
:10491000DBFFFFF7A1FFF8BD28005A6802329200C2
:104920009B188B4205D21A68561CE9D10028F2D098
:10493000D1E72160EFE7C0460011002004110020FC
:104940000480010004C00200CBD7000070B5002035
:10495000FFF7F0FEFF260500002801D1280070BDFA
:1049600003681C143440FFF7E5FEDA2CF4D105008F
:10497000F2E700008022F0B55200A1B000216748A4
:1049800006F0D6FE802200215200654806F0D0FED7
:10499000644BFF271B681A00049353425A411000CE
:1049A0000592FFF751FE049C0020631E9C415E4B64
:1049B00064421C405D4BE418FFF7C8FF0600002E60
:1049C0002DD10498FFF750FE411C0598FFF770FEAB
:1049D000059A574D534B2C601A60FEF73FFD514B23
:1049E00064201B68A0215A4253414F4A5B42134046
:1049F000B0222C6892029B18E41A6043490204F02A
:104A000053FDA0225202030000924A49220007A847
:104A100007F0D2F907A800F057FF21B0F0BD3268C7
:104A2000131412123A403B4003921A000A3A092A20
:104A300049D83A4B039A995C002931D110223E485B
:104A400006F076FE35002B6803991A123A4091421F
:104A500009D11A143A400B2A27D0132A2DD00A2A3A
:104A600001D1354B1D602800FFF764FE051EEAD119
:104A7000314B196800290FD02000FFF74FFE0400CA
:104A80002D4B5B195968002903D02000FFF746FE23
:104A9000040004350C2DF3D1204B0121039A9954C5
:104AA0003000FFF747FE060089E73B40022BDADCC7
:104AB000214A9B00D3185D60D5E7102200211E48D3
:104AC00006F036FECFE71A00153A082AE8D8144A4D
:104AD0000399525C002AE3D13500152B00D0150054
:104AE000300003681A143A40152A0FD01D2A00D14D
:104AF0000025FFF71FFE0028F3D1002D04D0200071
:104B00002900FFF70BFE0400054BC6E7039A1B12B2
:104B10003B409A42EDD10500EBE7C0460010002073
:104B2000081100200011002000C0FEFF04C0020098
:104B30000411002095D70000202F002010B5FFF7AA
:104B400019FF10BDF0B585B0039203220333DC17C3
:104B5000294D1440E4182B68284F5A4253418022B3
:104B60005B42D202A4103B409B18A21C0291244E2F
:104B7000910000910190316800980A18934215D273
:104B8000FFF7F8FE2B685A42534180225B421F40D8
:104B9000D202BF183368009A9B189F4206D2194868
:104BA00000F092FE0025280005B0F0BD029B35689C
:104BB00019066B461A7BA423DB051343FF222F0043
:104BC000090C1943019B12041B04134019432800CC
:104BD000FFF75CFD0837281D21003760FFF756FD01
:104BE000002C04D00A9A21003800FFF775FD009BC5
:104BF000083BFF183760D6E70011002000C0FEFF19
:104C0000041100206FD7000070B59AB0FFF74AFE7C
:104C1000FF221E4CD2000021200006F089FDFF2556
:104C2000FFF794FE0026002814D10200C300E358C9
:104C30000130591E8B41D218FF28F7D1144901A821
:104C400007F0BAF801A800F03FFE124800F03CFE61
:104C50001AB070BD03681A142A400A2A0AD11A121F
:104C60002A40FF2A03D0D200A1180B71A050FFF7F1
:104C700061FDD8E7132AFAD11B122B40FF2BF6D087
:104C8000DB00E2181671E650F1E7C04698250020D7
:104C90003BD800004FD800000021094B094A596059
:104CA0000131516059680029FCD0002119610123AC
:104CB00093600222044B8131FF315A501A607047D1
:104CC000FC1000400010004000E100E00222064B12
:104CD0000121DA670022054B5A61054A11615A69C0
:104CE000002AFCD07047C04604E100E0FC10004000
:104CF0000010004010B5044C2378002B01D0FFF7C2
:104D0000E5FF0020207010BD091200208023012043
:104D10005B055B6E5B001843704700000120024B8F
:104D20001B685B00184370478C1200200120024B67
:104D30001B685B0018437047240000200120024BD1
:104D40001B685B00184370479012002070B5040088
:104D50000D001600FEF74CF9802301215B055A6E09
:104D60002670002653006170E1706272010A5A0ACF
:104D70006071A171A272010C5A0C000E5B0EA6703C
:104D80002571E1712072E272237370BD10B5044C7D
:104D9000200007F057F801002000FEF7F5FD10BDD8
:104DA000951200200E4B10B51B680E4C5A1C0FD0EC
:104DB0000D4C002B0CD00D4C012B09D00C4C022BB0
:104DC00006D0094C042B03D00A4C052B00D1074C0C
:104DD000200007F037F801002000FEF7D5FD10BDD8
:104DE00028000020E0D8000060D10000EBD80000CF
:104DF00067D10000E5D8000070B5214C2278002A68
:104E00003DD1204B01215A608022D20511605A68A1
:104E1000002AFCD0002207201B4B1C4901255A50B8
:104E20000439585008315A5019481A4958501A49EB
:104E30001A485A501A495A50A622D2009D500822A8
:104E400018495A50043158500220174958501749F0
:104E500017485850174804395850182016495850C8
:104E6000C12189005A500539FF3958589218024318
:104E70005A501249124A9950FFF70EFF257070BD23
:104E800009120020FC000040001000400C0500004A
:104E9000746962751C0500002405000020000402EE
:104EA0002C05000014050000340500003C0500003E
:104EB000FFFF000021100100540500000A1200202D
:104EC0000405000070B50E4B06001B78002B01D1C5
:104ED000FFF792FF00200B4D2C7884420ED00A4B36
:104EE000202219780323091B1940084B4901C918CE
:104EF000300006F001FC0120013C2C7070BDC04662
:104F00000912002094120020081200200A1200202A
:104F1000002370B588B0984235DD0D6801262C005D
:104F200034409C422FD12300042D2CD90F222B6812
:104F30001A402300092A26D16A683F2A23DD6846E1
:104F4000FFF7C0FF230000281DD06B4619783300FF
:104F5000A14203DB6B461B5D5B003343A200AA1832
:104F600001349360202CF2D1092169444A780B78EE
:104F700012021A438B781B041A43CB781B06134387
:104F8000024A13600423180008B070BD901200207C
:104F900070B5454B8AB01B78002B01D1FFF72CFF71
:104FA00002AC2000FFF78EFF002802D100200AB0DB
:104FB00070BD23780B2BF9D96378012BF6D1E378F8
:104FC000012BF3D100231120384E394D33602B7063
:104FD00068442379374A4178136002780902114303
:104FE000827812041143C27812060A4332490A60D9
:104FF000002B0ED1152169444A780B7812021A430E
:105000008B781B041A43CB781B06134333600023B1
:1050100018E0012B1AD1152169444A780B78120245
:105020001A438B781B041A43CB781A211B061343AF
:1050300033600E23627C6944934200DD130000223A
:105040009A422CD100220420EA54B0E7022B03D16B
:10505000627B10331621EEE7042B0DD115210822B7
:105060006944684606F048FB0098019902F0D2FDB9
:1050700006F0F4F93060CAE7052BC8D115210822E3
:105080006944684606F038FB0098019902F0C2FDB9
:1050900006F0E4F93060627D0A231E21CBE7885CCC
:1050A000A8540132CCE7C046091200208C1200201F
:1050B00095120020280000209012002010B5134BFC
:1050C00004001B78002B01D1FFF796FEFFF7FEFDD1
:1050D00000200F4A0F49104B5450586001301060A7
:1050E00058680028FCD000201861013090601869D1
:1050F0000028FCD0094B0A481B785B011B18535051
:10510000FFF7E4FDFFF7C8FD10BDC04609120020FF
:105110000010004004050000FC10004008120020B0
:105120000A12002010B588B000281DDD0A68012190
:1051300013000B4018D1042A16D90F201468204000
:10514000092811D150683F280EDD9800101880689A
:105150000024084201D04010C4B26846C454013350
:10516000202BF2D1FFF7AAFF002008B010BD0000ED
:1051700010B5002813DD0C68E30710D56410532C1C
:105180000DD8084B1B78002B01D1FFF735FEFFF738
:105190009DFDA123044ADB00D450FFF77DFD0020D4
:1051A00010BDC046091200200010004010B50028B4
:1051B0000EDD0C68E3070BD56410FF2C08D8054BF7
:1051C0001B78002B01D1FFF717FE034A034BD45085
:1051D000002010BD0912002000100040240500002E
:1051E00013B5002814DD0C68E30711D5094B6410D2
:1051F0000093094B0193072C0AD8084B1B78002B0E
:1052000001D1FFF7F9FD6B46054A1957054BD150FF
:10521000002016BDE2ECF0F4F8FC000409120020B6
:10522000001000400C05000070B588B0002820DD9B
:105230000124086804401CD104281AD90F230268ED
:105240001340042B15D1FEF77FF9060006F0FAFD96
:105250000500122800D912252A0002210D326846C5
:10526000FFF774FD6B465D73A54205DC6846FFF7EA
:1052700025FF002008B070BD2300325D6B449A7397
:105280000134F1E7F0B50D008BB0012832DD08687C
:105290000122040014402DD104282BD90F230168CA
:1052A0000B40042B26D16B68134223D0FEF74CF938
:1052B0006E6807007310019306F0C4FD05000E2808
:1052C00000D90E252A000121113202A8FFF73EFD68
:1052D0006A46127902AB5A7302AA73129373019B46
:1052E00076141B0ED67313745574A54205DC02A800
:1052F000FFF7E4FE00200BB0F0BD3A5D02A9631891
:105300009A740134F1E730B589B0002814DD0C68D7
:10531000E30711D5102268460021FFF717FD6B4601
:105320006A4665105D73684663122D0E64149373AC
:10533000D4731574FFF7C2FE002009B030BD000021
:10534000174B184A5968002903D0002159600131D0
:105350009160196900291FD0002018618023DB00AB
:10536000D3581149012B18D1A923DB00D3585B4234
:105370000B600E490B78032B01D801330B7003200F
:105380000B490B78013303400B700A495B015B1832
:10539000094953500123936070470860FAE7C046FB
:1053A000FC10004000100040240000209412002057
:1053B000081200200A1200200405000010B5034A5C
:1053C0001021034800F07EF810BDC04660D80000F0
:1053D00057D80000044A05491368C85401339B0597
:1053E0009B0D13607047C046C4160020C4120020F5
:1053F00070B5114C114A2368834202DC00232360FC
:1054000016E0155C411C2E00FA3E012E05D899428B
:105410000FDA555C013D1F2D01D90800ECE70100B2
:10542000151A565C6E5401318B42FADC181A206052
:1054300070BD1570FAE7C046D01A0020D0160020C3
:1054400010B5FDF7CBFD064B1A68824201D9002248
:105450001A601B68C31A034898428041404210BD3D
:10546000C0120020204E000010B5094C094A2368E4
:105470001268934200D110BD074AD05CFDF7E6FFE9
:105480000028F8D0236801339B059B0D2360ECE7CF
:10549000C8160020C4160020C412002010B5040055
:1054A000064B074A1B6812689B1ADB439B059B0D42
:1054B000A34200DB10BDFFF7D7FFF1E7C4160020C1
:1054C000C816002070B5074E33680B2B08DC0C257E
:1054D0005D43054C0133285164196160A26033605B
:1054E00070BDC046CC160020302F002010B5FBF751
:1054F00011FEFFF77FF8FBF735FEFDF73BFFFEF7E8
:10550000F3FBFEF731FCFFF759FF00F083FF01F0DA
:1055100085F901F0CFFB10BD962210B512010021D4
:10552000034806F005F90022024B1A6010BDC04680
:10553000381C0020CC050020064B074A1B68126867
:105540009B1ADB439B059B0D0122834200DC00225A
:1055500010007047C4160020C8160020F8B50500DA
:105560000C0016001F1E0ED10320FFF7E5FF0028D8
:1055700008D0FA20FFF72EFFE8B2FFF72BFFE0B2CA
:10558000FFF728FFF8BD501DFFF7D6FF0028F9D020
:10559000FB20FFF71FFFE8B2FFF71CFFE0B2FFF7A9
:1055A00019FFF0B2FFF716FF3012C0B2FFF712FF7B
:1055B0003C00E31B9E42E5DD2078FFF70BFF013442
:1055C000F7E7000070B50024F0250B4B1B68A342E1
:1055D00002DCFFF7A1FF70BD2B006343074A9B1855
:1055E0001A78002A05D05978002311201A00FFF7F5
:1055F000B5FF0134E9E7C046CC050020381C002087
:10560000F8B507000024F0252B0063430C4A013451
:105610009E18B74211D0317800290BD00133D15CEC
:10562000002311201A00FFF799FF2A000021300003
:1056300006F07EF80A2CE7D1F8BD024B1C60F9E7B2
:10564000381C0020CC050020F0B5150001222F00E9
:105650007A4C1740A54401900291002F11D005AB60
:105660001A706A105A70120E1A7105226912997016
:105670006D140299DD70FFF771FFCF239B009D44ED
:10568000F0BD042D2AD90F2428680440042C32D1FF
:10569000022304AA28001371FDF756FF050006F047
:1056A000D1FBC82302009B00984200DD1A007C1C3D
:1056B00097420DD1984206D9614804AB0322614953
:1056C000C01806F019F8220005AB02990198D2E73C
:1056D0002700611E695C05ACE155E8E7042D00D0A8
:1056E000A7E0032304AA043D13716B425D4105AB9F
:1056F00055710222E9E7092C7ED1042205AB1A700C
:105700006A68511000916946521209789A70009A9D
:1057100059701F2A01DD202200926A46127806ACD9
:10572000DA70009BBB4202DC05ABE21ACDE7012632
:10573000BB00EB189868064006D1042837D90F2122
:105740000368194002290CD10123237043106370B0
:1057500042121B0E4014A270E07023710534013711
:10576000DFE7042921D102232370FDF7EDFE03902A
:1057700006F068FBA31C0C2809D86070864201D192
:105780009C19ECE7039A925D9A550136F6E70C22D4
:105790006270039A925D9A550136092EF9D12E2333
:1057A000E372237363730E34D9E7012907D103230E
:1057B000043823704342584160700234CFE709290E
:1057C00009D10423237043685A1062705B12A370DE
:1057D000E6700434C3E703290BD105232370006866
:1057E000020992B2430F92000B40D31A63701B124E
:1057F000EDE726700134B2E7032C00D03DE7052227
:1058000005AB01091A7089B2420F890022408A1A39
:1058100011125A709970642A00DD64220421DA7032
:10582000081F824201DC04324FE7685C58540131A2
:10583000F6E7002D00D020E753E7C046C4FCFFFF89
:1058400022030000DCCD000070B502000024F0212E
:105850000D4E0800604380194578954203D001340D
:105860000A2CF6D170BDF022002105F061FF074A35
:105870001368013BA34200D11460002329001A00E1
:105880001120FFF76BFEEDE7381C0020CC0500204F
:1058900010B5B2B002236A460400137006F0D2FAC3
:1058A000C72800D9C7200023984207DC421C6B465A
:1058B000FE211420FFF752FE32B010BD69460133BD
:1058C0005A1EA25CCA54EFE730B5B3B002236A4651
:1058D0000500137006F0B6FA0400C72800D9C724E3
:1058E00000239C420BDC20003230FFF7D7FD621C06
:1058F0006B46FF211420FFF731FE33B030BD6946FF
:1059000001335A1EAA5CCA54EBE70000F0B5BBB0E5
:1059100004900C00012803DC1B20FBF7F9FC51E08C
:105920002A4B08680293C30709D4042807D90F2318
:1059300002681340042B02D1FDF706FE0290234BB0
:1059400060680393C30709D4042807D90F230268AA
:105950001340042B02D1FDF7F7FD039000271C4BE9
:105960001B680693069BBB420BDC039B194A009302
:10597000C821029B08A806F0EDF908A8FFF7A4FFCC
:10598000CAE70C267E43144B0299F618306806F0DD
:105990004FFA051E05D17368B6680793079B9D42B1
:1059A00001DB0137DEE730680399059606F040FA1F
:1059B0000836002808D121000498059B08310238D8
:1059C0005B6898473BB0F0BD0135E7E76BD200005C
:1059D000CC160020BCD90000302F0020F7B5234B97
:1059E00006001B68F02100930023009A9A4211DC04
:1059F0000024F0231A006243019201991C4A5518B1
:105A00002F78002F12D001340A2CF3D11948FFF758
:105A10005BFF29E00A005A43154882185078B042CB
:105A200002D11278002A1FD10133DEE7F0223900BB
:105A3000280005F07DFE02230D4A0199EB605354C6
:105A40000D4AF1008A58009B6E70AE70AA602F61FB
:105A50006F61A34202DC054B01341C60002331005E
:105A60001A001020FFF77AFDF7BDC046CC050020D4
:105A7000381C002005DE00009825002010B5FFF737
:105A8000A1FDFF24084AE3005B429B18074AD35C50
:105A9000043B012B03D8E043C0B2FFF79FFF013C5A
:105AA000002CEFD110BDC046FC0700009825002057
:105AB000F7B50F00FF247F2501901E4AE300D31A9B
:105AC0001D4A9A181278062A01D0032A20D1FF22F3
:105AD000D2009B18186883682B401C2B18D1C36810
:105AE0001A002A40042A13D102692A40192A0FD128
:105AF0001B0A01339B000C30C018FDF725FD03780D
:105B00000600002B10D006F09DF90023B84209D002
:105B1000013C002CD1D1F7BD019AF15CD25C9142DD
:105B2000F6D101339F42F7DCE043C0B2FFF756FFE6
:105B3000EEE7C04698250020FC07000070B5050080
:105B4000FF24084AE3005B429B18074AD35CAB4240
:105B500003D1E043C0B2FFF741FF013C002CF0D17C
:105B600070BDC046FC07000098250020F7B5FDF782
:105B700035FA574B1A68824201D900221A601A6816
:105B80005449821A8A420DD9FF2253491860D30022
:105B90005248CB1A1B181B78073B022B0CD9013A31
:105BA000002AF4D1F7BD0720FFF7C8FF4C4B27E0D0
:105BB0000820FFF7C3FF38E0FDF71AFA071E00D1EF
:105BC00001270020FDF70EFB01900020FDF71EFBD2
:105BD000019B0090434C444D002B12D02368002BB6
:105BE0006ED12B682760002B6ED0404B01261B78AE
:105BF000002BD8D10920FFF7A1FF394B1E703B4B7A
:105C00001E70009B002B12D02B68002B0FD1236835
:105C10002F60002B1ED0324B01261B78002BC7D1E2
:105C20000920FFF78BFF2E4B1E70304B1E70236830
:105C3000002B0FD02A4E3278002A0BD19F4200D27F
:105C400027602368FB1A312B04D90720FFF776FF62
:105C5000012333702B68002B0FD0244E3278002A9A
:105C60000BD1BB4200D92F602B68FF1A312F04D90A
:105C70000820FFF763FF012333702368002B0CD04B
:105C8000019B002B09D1164E3378002B02D107203F
:105C9000FFF754FF0023236033702B68002B00D1E3
:105CA00080E7009B002B00D07CE7104C2378002B72
:105CB00002D10820FFF742FF00232B60237071E719
:105CC000009A002AA0D1B5E7009B002B9FD1AEE738
:105CD000BC1200200F27000098250020FC070000C0
:105CE000B0120020AC120020B4120020B812002024
:105CF00037B500240500FFF765FC01A80194FDF706
:105D00005FFA21002000FEF71DF9FEF71DFBFDF7ED
:105D100091FAFDF70BFBFDF725FBFEF761FCFDF7A4
:105D200083F9A54204D0FDF7BBFB0248FFF7CCFD89
:105D300037BDC046F6DD0000002310B501001A0093
:105D40001120FFF70BFC10BD07B56B4619706946B3
:105D50005A7013128B701314120ECB700A716B46AB
:105D6000010005221320FFF7F9FB07BD10B50A005B
:105D700001001220FFF768FC10BD70B50500080097
:105D80000C003230FFF78AFB2B00220000211B2081
:105D9000FFF7E4FB70BD10B50C00030011001420E8
:105DA0002200FFF7DBFB10BD012370B5FF24084A7A
:105DB00041185B42884201D3D84370BD06781D0A62
:105DC000234073409B009B5801306B40F2E7C04674
:105DD000D8D9000013B50400FE2813D80A4BC2001E
:105DE000D05800280ED0436808309900FFF7DCFF38
:105DF00001900920FFF752FB01AB0422210017207C
:105E0000FFF7ACFB13BDC04698250020F7B5019005
:105E1000FEF79CFD01250400FF276D42002C01D1F7
:105E20002800FEBD266833143B40152B0DD1210000
:105E30000198083105F0FCFF002801D135123D40E2
:105E40002000FEF777FC0400E8E71D2BF8D10125C0
:105E50006D42F5E7F0B580279FB0FFF705FBB54C25
:105E6000B54D2068FF00391A4019FDF7D5FA2368AF
:105E70000600C3182360002B0ED11FB0F0BD2068B0
:105E8000391A2818FDF7C8FA236806001B18236082
:105E9000FDF7A4F8A94B1860002EF0DC2B78FA2B44
:105EA00000D00EE12368022B07DCFFF7C9FA0028B7
:105EB000E3D00120FFF79CFADFE76B78AC78981EFF
:105EC000182800D9F2E003F05BFA0D2024282B34C7
:105ED000F13E707A7E94CDDEF1F1F1F1F1F1F1F164
:105EE000F1F1EC00FF2C0ED02000FFF7ADFC0022FA
:105EF000934BE100CA505B181A7121000092130005
:105F00001320FEF71FFE0320D4E72000FFF766FDF5
:105F1000F9E72000FFF798FCF5E7FFF7AFFDF2E7A0
:105F2000FFF750FB0020FFF7E3FE8648FFF7CCFCAD
:105F3000E9E7632CE7D8844BA200D2582100152052
:105F4000FFF782FBDFE7FEF701FDFF270400002CCF
:105F5000D9D025682B143B40152B04D02000FEF728
:105F6000E9FB0400F3E72000083005F06BFF0600B2
:105F70000530FFF793FAFB20FFF72CFA2D121D20B6
:105F8000FFF728FAE8B2FFF725FAF0B2FFF722FA96
:105F90003012C0B2FFF71EFA25002B1B9E42DDDD3A
:105FA000287AFFF717FA0135F7E700211D20009145
:105FB0000B000A00FEF7C6FDFDF772FAA3E720000A
:105FC000FFF708FF9FE7FDF71BF805AC5F4A642168
:105FD00000905F4B200005F0BDFE022320002370DF
:105FE00005F030FF2300020000211620FFF7B6FA6B
:105FF00089E70026524AF3009B181C68002C28D021
:106000001B790393636808349F00B81D0293FFF760
:1060100045FAFB20FFF7DEF901207D1CFFF7DAF9D6
:10602000F0B2FFF7D7F9E8B22D12FFF7D3F9E8B2D3
:10603000FFF7D0F90398FFF7CDF9E719A7420CD87D
:10604000FFF712FA05230298584301F06DFBFFF7A2
:106050000BFA0136FF2ECDD155E72078FFF7BAF9BC
:106060000134EBE70024FFF7ADFA22002100009491
:106070002300DA20FEF766FDFF222100D20030481F
:1060800005F056FB98E7012C02D1FEF77DFB3AE7BD
:10609000022C02D1FEF752FD35E70120FFF728FE62
:1060A00031E7002321001A001A209FE71A00C83A9E
:1060B000052A00D927E7002218001100FBF75EF837
:1060C00021E7FB2B00D0F4E62268042A00DCECE692
:1060D0002E79E8781F4B360206439E4200DDE8E643
:1060E000331D9A4200DCE0E6EB5CFE2B00D0E0E6DC
:1060F0006878AC78771E1B2800D17DE02ED8072861
:1061000063D0082838D001282DD1FF2C10D02000D2
:10611000FFF79AFB6D79104AB31E009221002A0006
:106120000A20FEF70FFD064BE400E0501B191D711D
:10613000701DBFE6D01A0020D0160020C01200202B
:1061400098250020D8DD0000902D0020EFDD000014
:10615000EADD0000F6030000D61600201D285DD001
:106160004FD31E2871D00300C83B052BE0D8404A0E
:106170003900FBF703F8DBE7632CD9D86A79022AE8
:1061800013D0032A1BD0012AD2D1E979AB790902B5
:1061900019432B7AA4001B0419436B7A1B060B438B
:1061A0005B001343334AA350C2E7002FC0DDB11E8A
:1061B0003148FDF7E9FB2F4BA400E050B8E7AB797D
:1061C000A4005A1E93419B00ECE7632FB0DC05ADA1
:1061D0003A002749280005F08FFA00232800EB55E4
:1061E000FFF714FE0028A3DB224B8000C2582100D9
:1061F0001520FFF729FA9BE739001D48FFF758FCE7
:1062000096E7FF2C94D06A79022A91D81A490B207C
:1062100000912100B31EFEF795FC89E7632F00DD96
:106220006327002305A9BB420ADBFB430022DB17DF
:106230003B40CB181A70152000917B1C2100EAE727
:10624000EA185279CA540133EDE7012C00D06FE708
:10625000002F00DC6CE76B79002B03D01C00322B85
:1062600000DD322464235C43044B1C6060E7C046BD
:10627000D5160020902D0020D61600200400002006
:106280000120704710B5064C200000F043FE054980
:10629000200000F081FE0122034B1A6010BDC046B1
:1062A000081B0020801A0600D41A002010B5012116
:1062B0000D20FCF7ABFE01210E20FCF7A7FE00210C
:1062C0000F20FCF7A3FE044C200000F065FD102118
:1062D000200000F07DFD10BDE81A0020F8B5012572
:1062E0000C682C4203D10D20FBF712F8F8BD6410A6
:1062F0002DD4FCF789FEA04229DB00212000FCF709
:1063000085FEFA222900D200200001F03FFA002881
:106310001DD0002500270726FA2201219200200027
:1063200001F034FA002812D0282802DD0123B340FE
:106330001F43013EF0D20E4EAF550135052DE9D178
:10634000012206210920FDF7A1FA002801D1002031
:10635000CCE70B23012443600023F25C9900520038
:106360004118224301338A60052BF6D1BEE7C046AF
:10637000D81A002010B504680D20E30703D5641077
:10638000FF2C03D91720FAF7C3FF10BDFFF78EFFCC
:10639000E1B2024800F03EFD0020F6E7E81A0020D6
:1063A00010B5FFF783FF0021034800F033FD4300E1
:1063B0000120184310BDC046E81A0020A021012288
:1063C0000B4BC9005A500B480B4958500B491A60E7
:1063D0004A68002AFCD000224A60A121C90058580E
:1063E00001215960A021C9005A50054BC0187047BF
:1063F000007000406A10000004050000FC700040BE
:10640000FBFDFFFF10B5FFF7D9FF43000120184344
:1064100010BD000010B5034A0A210348FFF752F8E7
:1064200010BDC0461CDE00006CDE0000F8B5012384
:1064300006681E4205D045681D4202D084681C4291
:1064400003D10D20FAF764FFF8BD76101520802ED9
:10645000F8D86D101620FF2DF4D86410FF2C01D948
:106460001720EFE70B4B1B68002B01D1FFF70AFF4A
:10647000094FF1B2380000F026FEE9B2380000F012
:1064800015FDE1B2380000F011FD380000F086FE85
:106490000020D9E7D41A0020081B0020F7B50122FC
:1064A0001400904222DD0D682A421FD01D4B154179
:1064B0001B684C68002B01D1FFF7E4FEE9B201270D
:1064C0002500194E3D40300000F0FDFD002D0FD09D
:1064D0003C413000E1B200F0E9FC300000F05EFE2B
:1064E0000024A04202D02320FAF712FF2000FEBDB4
:1064F000042CF2D90F2322681340092BEDD16368D5
:106500005B100193019BAB42E7DDAB00E318996898
:10651000394204D04910C9B2300000F0C7FC01353F
:10652000F0E7C046D41A0020081B0020154B70B5B8
:106530001B6805000E00002B01D1FFF7A3FE124CD3
:10654000EDB22900200000F0BEFDF1B2200000F005
:10655000ADFC0021200000F0C1FD002801D0404228
:1065600070BD72B601222900200000F0A7FD62B6BE
:10657000200000F08CFC0028F2D0200000F08CFC01
:10658000EEE7C046D41A0020081B002010B50124F5
:106590000368234202D04168214203D10D20FAF75B
:1065A000B7FE10BD5810802801D91520F7E7491013
:1065B000FF2901D91620F2E7FFF7B8FF400020437A
:1065C000EFE710B50400012814D105211820FFF7CA
:1065D000ADFF7F282BDC03007F3301DA7F204042B0
:1065E000C8235B4258437F2102F05EFF052C00D197
:1065F000404210BD032811D101001820FFF796FF7B
:106600007F2814DC03007F3301DA7F204042C82357
:106610005B4258437F2102F047FFEAE70020052C48
:10662000F5D107211830FFF781FF7F2802DD0138FF
:10663000FF38D0E703007F3301DA7F204042C823D0
:106640005B4258437F2102F02FFFD1E710B50120B4
:10665000FFF7B7FF43000120184310BD10B503201A
:10666000FFF7AFFF43000120184310BD10B5052010
:10667000FFF7A7FF43000120184310BD10B5082104
:106680001820FFF753FF0300C00FC018012340106C
:1066900015304000184310BDF8B501231C00984286
:1066A0002BDD0F683B4228D04E6835001D4024D1B9
:1066B000042E22D90F2231680A40092A1DD173689D
:1066C0005C10202C00DD2024144B1B68002B01D112
:1066D000FFF7D8FD72B67F10F9B2114F22003800D3
:1066E00000F0ECFC62B6A54214DA380000F0CFFBF3
:1066F000002804D101246D002C432000F8BD38008F
:1067000000F0CAFB0122AB004000F3181043986070
:10671000AD18E8E764000125EEE7C046D41A002072
:10672000081B002070B52B4B86B01B68002B02D1D4
:106730000120FFF746FF01AD14220021280004F0DC
:10674000F7FF254E1821300000F0BDFC032130007A
:1067500000F0ACFB0021300000F0C0FC041E13D19F
:1067600072B605221821300000F0A8FC62B6300095
:1067700000F08DFB002802D0300000F08DFBA3005C
:106780000134E850052CF2D1019B7F2B01DD013B48
:10679000FF3BAA687F2A01DD013AFF3A29697F2978
:1067A00001DD0139FF39C820434342434843DB112F
:1067B000D2115243C0115B4340439B18181804F098
:1067C00083FE01F057FB04F049FE4300012018430B
:1067D00006B070BDE01A0020081B002000207047A2
:1067E000012070470020704700207047012070474B
:1067F000002070470020704700207047002070473D
:10680000002070470020704700207047002070472C
:1068100000207047704770477047000010B5034A6A
:106820000E210348FEF74EFE10BDC046D0DE00002C
:1068300040DF00000378013B1F2B00D97047013077
:10684000F8E710B5FFF7F6FF0378002B0BD0013007
:10685000222B11D10378002B03D0421C222B03D111
:106860001000FFF7E7FF10BD5C2B03D14378002B2E
:1068700000D0821C1000EDE73A2BF2D02C2BF0D088
:106880007B2B0BD1FFF7D6FF0378002BE9D07D2BB4
:1068900001D10130E5E7FFF7D4FFF5E720225B2BBC
:1068A00014D1FFF7C7FF0378002BDAD05D2BF0D0AF
:1068B000FFF7C7FFF7E7202BD3DD2C2BD3D0190030
:1068C00091435D29CFD0222BCDD001300378002B0E
:1068D000F1D1C6E7002210B5904216D0FFF7AAFF0B
:1068E00003780422222B10D0023A7B2B0DD0013AE0
:1068F0005B2B0AD0190030390232092905D92D2B1A
:1069000005D14178303909290AD8100010BD052277
:10691000742BFAD00132662BF7D001326E2BF4D0F3
:10692000581E83415A42F0E770B5FFF783FF0378A2
:1069300001222D2B01D18018023A00230A2502E002
:106940006B430130CB1801783039CCB2092CF7D920
:106950005A43100070BDF8B50C001500FFF76AFF30
:106960000378222B02D000232370F8BD0D236A1E6A
:10697000210008250C260A279C4601300378222B8B
:1069800002D100230B70F0E7002BFAD0441C5C2BE3
:106990000BD14378841C622B0ED0662B0ED06E2B4D
:1069A0000ED0722B0ED0742B0ED0002AE9DD0B70A6
:1069B000013A01312000E1E72B00F6E73300F4E76C
:1069C0003B00F2E76346F0E70923EEE710B5040069
:1069D000FFF737FFA04202D90378202B00D910BD62
:1069E0000138F7E710B5002815D00378002B13D035
:1069F000FFF720FF2021037802008B4300205D2B4E
:106A000009D01000FFF71DFF03782C3B5A42534179
:106A1000C018FFF70FFF10BD1800FCE703000020AF
:106A200070B50C0081420EDD1A785B2A0BD1581C20
:106A3000FFF700FF0125AC4205D0FFF7D3FF002888
:106A400001D00135F7E770BD70B50C0015000029C5
:106A500001D000230B70002820D00378002B1ED01B
:106A6000FFF7E8FE037806002C2B03D10130FFF777
:106A7000E1FE0600337800207D2B0FD0844204D045
:106A80002A0021003000FFF766FF3000FFF7D9FE33
:106A900003783A2B02D10130FFF7CCFE70BD18000D
:106AA000FCE7F0B50D0004009DB02E78002E35D027
:106AB0002E21280005F0AEF9071E14D0431B0193C8
:106AC000303E092E14D82800FFF72EFF01002000C9
:106AD000FFF7A4FF0400002C20D0002F1ED0019B44
:106AE0000133ED18E1E7280005F0ACF90190E7E784
:106AF00023787B2B11D1601C642203A9FFF7A4FF2C
:106B0000041E0BD0019A290003A805F0A2F9002861
:106B1000E1D02000FFF795FEEEE7002420001DB035
:106B2000F0BD70B5050000200C0081421DDD28007D
:106B3000FFF7D0FE0300681C012B14D00020022BAD
:106B400013D10022681C1100FFF77EFF012C0CD02E
:106B5000FFF748FF00221100FFF776FF013CF5E741
:106B6000FFF740FF013C012CFAD170BDF8B50500DC
:106B700000200C0016001F0081420DDD2800FFF7E9
:106B8000A9FE03000020022B06D1681C3A00310048
:106B9000FFF75AFF012C00D1F8BDFFF723FF3A00A1
:106BA0003100FFF751FF013CF4E710B50024A0428B
:106BB00018D0FFF73FFE03787B2B0AD1013000226B
:106BC0001100FFF741FF00280CD0FFF73AFE013417
:106BD000F5E75B2B06D10130FFF704FF002801D059
:106BE0000134F9E7200010BDF8B5002816DD0D6866
:106BF000EB0713D56D10013D0124FDF7A7FE00261C
:106C0000FF27644200280CD1002E21D0300005F06F
:106C100019F901003000FCF7B7FEF8BD01256D42FF
:106C2000EAE703681A143A40152A0BD11B123B40BD
:106C30009C4200DA1C009D4201D106000836FDF797
:106C400079FDDFE71D2AFAD1012400266442F6E728
:106C50000120013464002043DFE7000010B508681C
:106C60000C00FCF771FCFFF7D1F8002803DB626829
:106C7000024B8000C250002010BDC046902D002065
:106C800010B50868FCF760FCFFF7C0F80123002886
:106C900002DB024B8000C358180010BD902D00206D
:106CA00010B50868FCF750FCFFF7B0F8C043C00F00
:106CB000800010BD10B5034A04210348FEF702FC12
:106CC00010BDC046D0DF0000C9DF000010B5FCF7E2
:106CD0005DFBFCF70BFCFEF709FC0448FEF7F4FD36
:106CE000FDF792FFFEF7CAFE10BDC0461FE0000090
:106CF00010B5FCF74BF810BD70B5002504AC247836
:106D00000573A94205D10A4B0A4A23210A4804F017
:106D100085FC01600949920052589B0002715B5842
:106D2000A40083716358856043710223C37170BDF1
:106D300037E0000096E0000045E00000F4E00000CD
:106D4000037B002B04D1437383730361013303730B
:106D5000704700001FB50191A02100240068C90000
:106D6000D2B24450012A10D0A24209D0032A0AD03C
:106D7000074A8350074B019AC250012343501FBD5D
:106D800002221343F4E70422FBE70622F9E7C04698
:106D9000540500002405000010B50400FFF7D0FFE3
:106DA000A1222368A179D20099506179064A200076
:106DB0009950217904329950044B19685A689B689C
:106DC000FFF7C8FF10BDC0460C050000FC1A0020EC
:106DD0004BB2002B0FDB80233F290FD81F290FD880
:106DE0000F290FD807290FD803290FD81B060168D0
:106DF000074A8B50704780239B04F8E7DB04F6E7D3
:106E00001B05F4E75B05F2E79B05F0E7DB05EEE722
:106E1000240500000368074A99501A00FC32D16823
:106E20000029FCD0A321C90058580023C0B2D36068
:106E30007047C0461C05000007B58022074BD205ED
:106E40001A6000229A6002321A7111230E320093E6
:106E5000034905330348FFF74FFF07BDFC1A002025
:106E600000300040E81A0020F8B505000E001700B9
:106E70000024BC4208D02B68315D1B68280098476D
:106E8000002801D00134F4E72000F8BD704710B5A8
:106E90001C3000F0BDF910BD10B51C3000F0AAF98F
:106EA00010BD10B51C3000F0B9F910BD70B5437EAF
:106EB0000D00002B01D1002070BD6430040000F0F3
:106EC000B6F90028F7D12000290000F084F901204C
:106ED000F2E70000F7B50193FA23002504009B00B8
:106EE00083600B4B4560083303601C300F001600B5
:106EF00000F066F92000643000F062F96B461B79FF
:106F0000276166756576A5762000A375FEBDC0462F
:106F1000D4E000000123827DC3751B4B9200F0B5C5
:106F2000D4582022210011404D1EA941457DC02684
:106F3000AD005D59A0272A40531E9A4153421F229B
:106F400014402A402500B6004942C135FF053140B2
:106F50003340FF350D4EC919AD006E501100C131DF
:106F6000FF31DB198900CE50CC210569084B49045B
:106F7000E95005210569243BE95001690833CC50EB
:106F80000169044BCA50F0BDF4E000000C0600009B
:106F9000240500000C050000A022002310B50469A0
:106FA000D200A3500A4CA1420FD90A4C8C425B413B
:106FB00009495B420B40CD21C9045B1804690749AC
:106FC000635005210369995010BDCC235B04F5E79C
:106FD000A086010090D00300000098FD2405000069
:106FE000F7B5040000200D000193824265D0160021
:106FF000402A00D9402627001C37380000F0F6F858
:10700000B1232269DB00D55080220123216992003F
:107010008B50A27E002A03D1226913622269136079
:107020000025731EAB4207D1019B002B04D08022A8
:107030000221236992009950012223691A6223696F
:10704000FC33DA68002A02D19A6A002AF9D09A6AD7
:10705000002A0BD1DA60A3232269DB00D158380063
:10706000C9B2013500F0B7F8B542DAD3019B226905
:10707000002B0FD11300FC339B6A002B0AD1013384
:10708000A376D3612369FC33DA6C002AFCD000229A
:10709000DA640AE000230121A37651611A00236912
:1070A000FC3399680029FCD09A602369FC339A6A02
:1070B000002A01D000229A62E8B2FEBD10B5012379
:1070C000FFF78EFF10BD0300AC3310B5040019703C
:1070D000643000F08BF80123637610BD00230200BA
:1070E00070B5AC3243760D001178B122040000690E
:1070F000D20081508022216992008B502269013395
:1071000013622269936026006436300000F080F834
:10711000002812D0300000F06DF81E4B2269D050CC
:107120002369FC331A6A002A02D19A6A002AF9D02C
:107130009A6A002A01D11A62E5E723690122002D2B
:107140000DD11900FC31896A002908D1DA6123695F
:10715000FC33DA6C002AFCD00022DA6407E05A61C2
:107160002369FC339A68002AFCD000229A60002030
:107170002369FC339A6A82420BD098622169064ADD
:107180008B588B501800022B03D0181F431E9841B8
:10719000033070BD1C050000C404000010B50121BF
:1071A000FFF79CFF10BD000010B513231222024907
:1071B0000248FFF78FFE10BD00400040081B002072
:1071C00010B540220021040004F0B2FA0023200090
:1071D0002364636410BD10B53F24026C531C23402C
:1071E000446C9C4201D08154036410BD00230364AD
:1071F00043647047436C026C934206D03F21C25CEB
:1072000001330B4043641000704701204042FBE70C
:10721000036C406C181A00D540307047436C026C08
:10722000934201D0C05C704701204042FBE73F22FF
:10723000036C406C01331340181A43425841C0B2EA
:107240007047000003210A4802680A4302600948A7
:1072500002680A4302600849084A094B9B1A03DD89
:10726000043BC858D050FBDC00F012F8F8F74CFF94
:1072700024050040540500403CE6000000000020CA
:1072800064020020FEE7FEE7FEE7FEE7FEE7FEE71A
:107290002D4B10B51A68D2B2012A0FD12B4A1268B1
:1072A00012070BD12A4AE0241168F022080010408E
:1072B00021422DD12749096811422CD01A68D2B237
:1072C000012A12D12149096809070ED1F02020496D
:1072D00009680140402908D11E490968014204D1CA
:1072E0008020C121C005C90042501B68DBB2012BC0
:1072F0000DD1164B1B681B0709D1154B1A68F023DB
:107300001A40A02A0FD1134A12681A420ED010BD9B
:107310003028CFD0D2E7104A104911608021104A9E
:1073200009021160CAE7D02AF1D1ECE70D4B1A68C7
:10733000012A04D00C4A1A601A68012AFCD1C02222
:107340000A4B1A60E3E7C046E00F00F0E40F00F0DC
:10735000E80F00F0EC0F00F004050040DFFF07C06D
:10736000186C004000EC06407593000014EC0640D9
:107370000120704710B503681322DB69984710BDE0
:1073800070470000054B0269D1500369FC331A6A4B
:10739000002AFCD0002201201A6270471C05000060
:1073A000030010B55C331A781F231A401E3B1900E6
:1073B0009140114AD167C222042104699200A15070
:1073C000026953600269D360A02300220169DB00D7
:1073D000CA5001230169094A5B428B500169084A7E
:1073E0008B5001690C3A8B50016908328B50143074
:1073F000FFF7FCFE10BDC04604E100E00C050000F4
:107400001405000010B51430FFF702FF10BD10B5D1
:107410001430FFF703FF10BD10B51430FFF7EAFE7C
:1074200010BD0000030070B55E331A780469724B1A
:10743000E25003005D331A780469704BE250030098
:1074400061331C7802696E4B012C00D09EE0050070
:107450005F352E78A225ED00565102006032157876
:10746000A1220669D200B5500269D4509623DB00F0
:10747000994200D88CE096231B01994200D88AE0FB
:1074800096235B01994200D888E096239B0199429C
:1074900000D885E0E1239B01994200D882E0962341
:1074A000DB01994200D880E0E123DB01994200D85A
:1074B0007DE096231B02994200D87AE0E1231B026B
:1074C000994200D877E096235B02994200D874E095
:1074D000E1235B02994200D871E0E1239B029942CB
:1074E00000D86EE0474B994200D86CE0E123DB0204
:1074F000994200D86AE0E122002312038A425B41EC
:10750000414A5B421340802252059B1801693F4A61
:107510008B50A02304220169DB00CA5000210369BB
:10752000FC33D9600369FC331962012301690B60E4
:1075300001698B60C1210469890062501F215C30A0
:1075400002780A4093406231314AFF3153500021A2
:10755000415600293CDA0F230B40083B2D4C9B0879
:107560009B001B1903242140A140FC348C40DD69A1
:10757000A5432C00C0258D4029002143D9611F233C
:10758000017819401E3B8B40136070BD00246CE7EE
:107590009E23DB02BAE79D231B03B7E71E4BB5E72B
:1075A0001E4BB3E7EC239B03B0E71D4BAEE71D4B2F
:1075B000ACE71D4BAAE71D4BA8E71D4BA6E71D4BEB
:1075C000A4E71D4BA2E78023DB049FE71B4B9DE74D
:1075D0008C080F4BA400E41803230B40FF21C025A7
:1075E000DB009940AD0066598E433100C0269E40B5
:1075F00033000B436351C2E70C0500001405000083
:107600006C05000090D0030000D0BEFE24050000F1
:1076100000E100E000ED00E000B0130000502700A2
:1076200000A04E0000F0750000509D0000F0EB003F
:1076300000903A0100E0D70100B0AF0300705F078F
:10764000F7B5009308AB1B7800250193FA230400DB
:107650009B0083600E4B45600833036014300F00BD
:107660001600FFF7ADFD23005C3327611E70009B01
:10767000084A9B00995823005D331970019B200034
:107680009B009A5823005E33DD701A70FEBDC04621
:1076900070E10000F4E00000036910B51A00FC324C
:1076A000D2680400002A0AD0A322D20099581430CC
:1076B000C9B2FFF790FD00222369FC33DA6010BDE8
:1076C00010B50248FFF7E8FF10BDC046C01B002000
:1076D0001D2307B502220093024901330248FFF738
:1076E000AFFF07BD00200040C01B002010B50028E0
:1076F00001D004F0D9FA10BD0849094A094B10B568
:107700001B688858FA22190A1B06184392000023A6
:1077100002F002F84904C00B084310BD00100140FC
:1077200004050000241C002070B5041E09D0FFF7DA
:10773000E3FF050000F014F8FFF7DEFF401BA04256
:10774000F8D370BD0022044B9A60044A13680133D9
:10775000DBB213607047C046FC100140241C0020BF
:107760007047704710B500F061F8FFF7FAFF01208D
:10777000FFF7DAFFFFF7AAFAFFF7BAFA024B002B7E
:10778000FAD000E000BFF7E700000000F8B51600EF
:107790004C1EA1411F220125104B8000104FC358E1
:1077A0004C42134038680F499D4001F0F3FD0A2117
:1077B000704301F0EFFD2C400300220029000A482D
:1077C00000F016F8FA21094C89004443386801F0AA
:1077D000E1FD0100200001F0DDFDF8BDF4E0000056
:1077E0002C00002040420F00100500501027000020
:1077F00030B504680C40944206D1013B002BF8D10F
:1078000012E0013B002B0FD004680C409442F8D1E9
:10781000002405680D40954204D101349C42F8D102
:10782000002002E0201C00E0181C30BDC420114BD9
:1078300080001A5810491140C02212020A431A50FF
:10784000C0218022490092025A501A608023A3224C
:107850000021DB05D20099500122F9309A60074BD4
:10786000FF301950C12002318000195040301950AA
:107870001A60704700E100E0FF00FFFF00100140C8
:10788000014B18607047C04678000020F7B5002310
:107890001E285AD8384B8000C258042A5BD007D81B
:1078A000022A54D055D80423012A09D000234CE0E1
:1078B000062A54D051D31A2A53D002231B2AF5D1B9
:1078C0002E4A116808294ED909294FD00A240226C8
:1078D000A02001252A4AC00015502A482A4D0768D1
:1078E0001C20BF00074029480197006857590090A5
:1078F00027481B0207401F43C02300989B020340F8
:10790000FF2057515759000207401F43019B1F4357
:10791000009B58016023184007433E435651012500
:107920001C4B156058680028FCD000205860A1232B
:107930000125DB00D3585560A025ED0050511BB246
:10794000A14202D015D2611ACB401800FEBD082317
:10795000B6E71023B4E72023B2E74023B0E7802343
:10796000AEE70123ACE708240026B1E70C000126AE
:10797000AEE7091B8B40E8E7F4E00000740000204C
:10798000007000403000002004050000340000209A
:10799000FF00FFFFFC700040F0B51E285BD8364B9F
:1079A0008000C258354B1E68002E30D1C227344BA0
:1079B000BF00D859334C03250440C02000022043A7
:1079C000D851C02480206400800018512E4F1860C8
:1079D0002E4B803CD859FF3CA043D8510437D8598E
:1079E000A8432043D8510837D8590C35A8438446BA
:1079F000072065462843D851A820C0001E50C1204A
:107A00008026800076021E501C601C4B1C601425D2
:107A100000202B001E4C2E0046433659771C1BD1EC
:107A20004343E250A0230325C132FF329200DB051D
:107A3000D550184B1A68082A14D114234343E3186D
:107A40009A6812485132FF32920059601150DA6838
:107A5000C1239B00C250F0BD9642E1D00130032803
:107A6000D9D1F8E7082A02D9083AD140E5E7082336
:107A70009A1A9140E1E7C046F4E00000281C00207B
:107A800000E100E0FF00FFFF04050000009000405F
:107A900038000020780000202149F0B54A6C2148C8
:107AA000002A14D0A025A12600230124ED05F6000C
:107AB000C258571C06D0C7187F68002F02D0270075
:107AC0009740AF5114333C2BF2D100234B64A023D9
:107AD0000121DB0500260F009C4614234B43C318ED
:107AE0001A1F1268104C0E4D920014195219526C44
:107AF000002A10D01A00143A1268551C09D0103B05
:107B00001B68FF2B05D03B00934065461A00074BCE
:107B1000EA50FC34666401310429DED1F0BDC04670
:107B2000FC90004038000020009000400C05000050
:107B300000B51E2818D8104A80008358C0209A0625
:107B40008000D2170240A020C00512181F20034059
:107B5000032909D80800C133FF339B0001F010FC52
:107B6000020905070021995000BD0C21FBE7042103
:107B7000F9E70321F7E7C046F4E000001E2812D819
:107B80000B4B8000C258C02093068000DB170340D7
:107B9000A020C0051B181F20104001228240002990
:107BA00002D104495A507047A121C900FAE7C046E2
:107BB000F4E000000C050000030000201E2B12D88A
:107BC000C021094A9B009A5889009306DB170B4095
:107BD000A021C9055B18A221C90058581F231A40CB
:107BE000D0401E3B18407047F4E00000F7B5060097
:107BF0000D000C008B180193019B671B9C4207D062
:107C0000336821781B683000984701340028F3D18D
:107C10003800FEBDF0B5C64600B5CB0F9846404AC9
:107C20004B005B0D9A1882B00D000400132A2FDC64
:107C3000002A49DB3B4F17413E000E40064323D04C
:107C40007F08390029400C430AD03749BD438C4690
:107C500063445C425C418023DB021341E4071D4323
:107C60004146CE0031492B008E19220034687568D8
:107C70002000290001F0F6FE009001910098019982
:107C800022002B0003F086F802B004BC9046F0BD41
:107C9000332A08DD8023DB009A42F5D102000B0075
:107CA00001F0E0FEF0E7224A94460122634452428A
:107CB000DA400242E8D052080242D1D094438022F6
:107CC000D2051A411443CBE74B005B080343DBD0DA
:107CD0000B031B0B1C436342234380244D0C2403E2
:107CE0001B0B23406D042B4319004346DA000F4B56
:107CF0009B181C685D6802000B002000290001F041
:107D0000B1FE009001910098019922002B0003F030
:107D100041F842464B005B08D60733431900B3E7EE
:107D200001FCFFFFFFFF0F00EEFBFFFFA0E10000E3
:107D3000EDFBFFFFF8B5274A4B005B0D9A180C00CE
:107D40000700132A10DC002A36DB234B13410B42B9
:107D50003AD0802424031441002064189C43060078
:107D6000250030002900F8BD332A0EDD80230600EF
:107D7000DB000D009A42F4D102000B003800210014
:107D800001F070FE06000D00EBE7144D0600AC4656
:107D9000012563446D42DD40AC4663460D0003425D
:107DA000DFD033239A1A323B93401818874200D908
:107DB0004C1C63469843D2E7C90FCC070020531CE4
:107DC000CDD1074B1C43CAE706000D000028C0D1E7
:107DD000C7E7C04601FCFFFFFFFF0F00EDFBFFFF01
:107DE0000000F03F30B5214A4B0087B05B0893425A
:107DF0001EDD1F4A934205DD02000B0002F0CAFFA0
:107E000007B030BD02AA00F095F803231840049A89
:107E1000059B012813D002281DD0002814D00298F9
:107E2000039900F06FFB80231B069C466144E7E743
:107E3000002300220093002301F0DEF8E0E702981F
:107E4000039900F05FFBDBE701240298039900949B
:107E500001F0D2F8D4E7012402980399009401F0CC
:107E6000CBF880231B069C466144C9E7FB21E93F10
:107E7000FFFFEF7FF0B54746CE4680B58DB00400DA
:107E80000D0000F067FA294B06001B780F005BB26B
:107E90009846013310D022002B002000290003F067
:107EA000C1FA8146002807D10022002320002900C2
:107EB00001F00AFC002806D1300039000DB00CBCDE
:107EC00090469946F0BD01230293194B06940795FD
:107ED00003934B460A93434604940595002B15D013
:107EE000002300221900100002F0D8F84346089041
:107EF0000991022B0ED103F0AFFB212303600A9BF3
:107F00000193002B0CD1089E099FD5E70023002484
:107F10000893099402A801F0C1F90028EFD1EAE71B
:107F200003F09AFB0A9B01930360ECE77C000020BE
:107F3000B0E10000F0B54E464546DE465746E0B596
:107F4000E14B4C008FB09046894664089C4200DCAF
:107F500087E0DE4B9C4222DCDD4A002900DC92E017
:107F6000DC4B02F017FFDB4B06000F009C4200D1F8
:107F70007EE1D94AD94B02F00DFF02000B004146C9
:107F800030000A604B60390002F004FFD34BD24A44
:107F900002F000FF434601259860D9606BE0D04BAA
:107FA0009C4200DC8FE0CF4B9C4200DD55E1CE4A85
:107FB000231592469A4451460905631A19001D007B
:107FC000040003F04BFA03F07FFA02000B002000DC
:107FD00029000892099302F0DDFE0022C34B02F053
:107FE00067FC0F00060003F039FA03F06DFA040095
:107FF0000D0002000B00300039000A940B9502F0CE
:10800000C9FE0022B94B02F053FC002200230C9061
:108010000D9101F053FB002800D192E100230022D2
:108020002000290001F04AFB434243410133B04A9A
:1080300041460192022208A80092524600F07CFBC1
:108040004B460500002B16DA802243461206944662
:1080500042465B68454263445360D3686344D360DF
:1080600009E00B00020041460A604B600022002339
:1080700000258A60CB6028000FB03CBC9046994632
:10808000A246AB46F0BD934B01F0ECFC914B0600D1
:108090000F009C4200D13DE18F4A904B01F0E2FC81
:1080A00002000B00414630000A604B60390002F0CC
:1080B00071FE894A894B01F0D5FC012543466D428A
:1080C0009860D960D7E701F049F88A4A8A4B0600E0
:1080D0000F0002F0EDFB0022884B01F0C3FC03F01F
:1080E000BDF9050003F0F0F9794A7A4B0490059147
:1080F00002F0DEFB02000B003000390002F04AFE05
:10810000754A06000F0004980599744B02F0D0FBE5
:10811000029003911F2D00DCC7E0029A039B300000
:10812000390002F037FE83468A4653465B00241529
:108130005B0DE31A102B6CDD04980599D322674B75
:10814000520502F0B5FB02000B003000390002922C
:10815000039302F01FFE0A0001001300069107922C
:1081600002003900300002F015FE029A039B02F073
:1081700011FE06000F0004980599614A614B02F058
:1081800097FB32003B0002F005FE069E079F0B00A6
:108190000200390030000292039302F0FBFD4B0015
:1081A0005B0D83468A46E41A312C32DD049805992A
:1081B000B822544B920502F07BFB03000C00020036
:1081C000029303940B000698079902F0E3FD020066
:1081D0000B0006000F000698079902F0DBFD029ADB
:1081E000039B02F0D7FD484A029003910498059939
:1081F000464B02F05DFB029A039B02F0CBFD0200AE
:108200000B00300039000292039302F0C3FD834655
:108210008A465A465346414630000A604B60390050
:1082200002F0B8FD029A039B02F0B4FD44460B0035
:108230000200A260E3604B46002B00DB1BE75B46BD
:10824000236080231B065344636080231B069C46E7
:108250006144A060E1606D420DE70B00020002F096
:1082600099FD434600259860D9601860596002E77F
:10827000D3221A4B520502F08DFD214A214B0D00ED
:10828000040002F087FD02000B00414620000A6056
:108290004B60290002F07EFD1A4B194A02F07AFD6C
:1082A000434601259860D960E5E602000B003000E6
:1082B000390002F06FFD6B1E154A9B009B588346E8
:1082C0008A46A342A5D130E7FB21E93F7BD9024092
:1082D00000004054FB21F93F3163621A61B4D03D84
:1082E000FB213941FFFFEF7FEAFBFFFF00007041F8
:1082F00038E2000083C8C96D305FE43F0000E03F12
:108300007370032E8A19A33BC14920259A837B39B8
:10831000B8E10000D3220C4B520501F0A3FB0B4A3D
:108320000B4B04000D0001F09DFB02000B004146C9
:1083300020000A604B60290002F02CFD034A044B28
:10834000B9E6032373E6C04661B4D03D7370032ED3
:108350008A19A33BF8B54746CE46674B80B50A005D
:108360000F00190005003940994200D19BE004003C
:108370000100002F69DD3F1500D1B4E05F4B12030F
:108380009C468023120B5B0313435B00CA0F6744B8
:108390009B184A00F80703D5D20F5B009B188A0090
:1083A00079108C46002180201624894680030D1800
:1083B0009D4202DC29185B1B8144D50F5B00013C08
:1083C0005B1952004008002CF1D10020804680202B
:1083D00020250027000609E08B425CD0D40F5B000B
:1083E000013DE31852004008002D16D0C4198B42FD
:1083F000F2DD27180E00002C49DB5B1AA2428941EE
:1084000049425B1A121BD40F5B00013D80443100CE
:10841000E31852004008002DE8D113434ED14346E3
:108420005B0837494A468846494652104244C907C4
:1084300002D5802109060B4361460F05BD181800BF
:1084400029000CBC90469946F8BD7B005B080343AD
:108450003900002BF5D0002F3CD1E30A153A640512
:10846000002BFAD08020400303423FD1002700E0D8
:108470000F005B00791C0342FAD0250020208D40BC
:10848000401A2900D71B2200C2401A4376E7FE4358
:10849000F60F8E19B1E79442A0D82718002CF6DB0E
:1084A0001E000023AEE702003B002800390002F066
:1084B000FFF92A003B0001F0D5FAC2E74346013339
:1084C00003D0434601335B08ABE701239846002302
:1084D000C144A6E73B00020002F05CFC02000B0076
:1084E00001F0DCFDADE713000022BBE7012721000E
:1084F00020207F42C6E7C0460000F07F01FCFFFF5E
:108500000000E03FF0B54746CE4680B587B0009208
:108510000193754B4F00814688467F089F4263DC7C
:1085200002F09CFF002800D1D4E04A46434648466A
:10853000414602F0BDF904000D006C4A6C4B02F09C
:10854000B7F96C4A6C4B01F08DFA22002B0002F057
:10855000AFF96A4A6A4B02F01DFC22002B0002F0C0
:10856000A7F9684A684B01F07DFA22002B0002F05F
:108570009FF9664A664B02F00DFC22002B0002F0C8
:1085800097F9644A644B01F06DFA22002B0002F067
:108590008FF9029003910022604B2000290002F025
:1085A00087F9029A039B06000F002000290002F0C1
:1085B0007FF9009A019B04000D004846414602F0F5
:1085C00077F902000B002000290002F0E3FB020013
:1085D0000B003000390002F0DDFB02000B00002030
:1085E0004F4902F0D7FB70E002000B0002F060F987
:1085F00004000D003D4A3E4B02F05AF93D4A3E4B05
:1086000001F030FA22002B0002F052F93B4A3C4BB9
:1086100002F0C0FB22002B0002F04AF9394A3A4B23
:1086200001F020FA22002B0002F042F9374A384BC1
:1086300002F0B0FB22002B0002F03AF9354A364B2B
:1086400001F010FA2B00220002F032F9354B0290B3
:1086500003919F429FDD344B00229F423DDC334912
:1086600000207B182E4916001F0002F093FB049097
:1086700005910022294B2000290002F019F932004F
:108680003B0002F087FB029A039B06000F002000CC
:10869000290002F00DF9009A019B04000D004846E4
:1086A000414602F005F902000B002000290002F00B
:1086B00071FB02000B003000390002F06BFB02007E
:1086C0000B000498059902F065FB07B00CBC9046BE
:1086D0009946F0BD00201249F7E7154B0026049299
:1086E0000593144FC5E7C046FFFF3F3ED43888BE10
:1086F000E9FAA8BDC4B1B4BD9EEE213EAD529C8046
:108700004F7E923E9015CB19A001FA3E7751C116CB
:108710006CC1563F4C5555555555A53F0000E03F9F
:108720000000F03F3233D33F0000E93F0000E0FF9C
:108730000000E73F0000D23FF0B5DE464E4645461A
:108740005746E0B5DC4CA5440D9114001900A49ADD
:108750000993DA4B9200D6584D1E03901821E01E63
:108760000696029500F0A0FEC3430100DB171940F6
:108770004B1C9A009B1ADB001B190B9105934C1B99
:10878000771918D4A59BA5009C463F1922AE6544D5
:10879000013707E0286802F097FE013403C604356C
:1087A000BC4208D0002CF5DA00200021013403C6B9
:1087B0000435BC42F6D1069B002B01DA00F0FDFB2C
:1087C000069B03990133DB009A46099BDA00944625
:1087D00000920022914672AA0492B94A61449346DB
:1087E00088469AAB63449B44029B002B00DABCE1B1
:1087F0005D4600260027039C4D442A686B6803CC25
:1088000002F056F802000B003000390001F02AF99E
:10881000083D06000F004445EFD1049B4B441E6009
:108820005F6008239C46E144D145DDD10EA80421B8
:108830008446494261448C46069A93009C446146B2
:1088400084460A910399083B63448C460C93009B31
:10885000009263449B46009A0498D10003008C4622
:10886000634408911E685F68002A33DD954980469D
:108870008C466244D300984470AB9A460EAB99463E
:108880000022914B3000390002F012F802F0E6FDB0
:1088900002F01AFE00228D4B04000D0002F008F8D1
:1088A00002000B003000390002F074FA02F0D6FD2D
:1088B0004B4601C39946434620001A685B6829006D
:1088C00001F0D0F808235B429C46E04406000F000C
:1088D000D045D5D1059B30001A003900984600F0EC
:1088E000DFFCFF2300229B0504000D0001F0E0FFE8
:1088F00000F038FC0022764B01F0DAFF02000B009A
:108900002000290002F046FA0D00040002F0A6FD46
:10891000814602F0D9FD02000B002000290002F080
:1089200039FA060040460F00002800DCEEE0009B0C
:1089300018215A1E92000EAB9B58091A1D000D41BA
:10894000A9448D405D1B0EAB9D5017231B1A1D4182
:10895000002D2DDD01239C46009BE144002B00DC13
:108960001CE20E9C0123002C00D0B5E0009A012AE5
:1089700009D099000EAA54580133002C00D0ACE065
:10898000009A9A42F5D1059B002B0EDD012B00D1F8
:10899000A8E1022B09D1009B0EA95A1E92000EAB32
:1089A0009B5807939B029B0A8B50022D00D1C1E07C
:1089B000002300223000390000F080FE009B0028D8
:1089C00000D194E2069A591E8A4210DC414A0A9864
:1089D00094460EAA6344944600229B0063441C689C
:1089E000043B22438342FAD1002A00D0C0E0069B18
:1089F0000EAA013B9B00D358002B00D0B3E001220C
:108A00000C9B043B596801320029FAD0009B9C461C
:108A10006244110007921A0001338B4246DC0B9826
:108A200063468046A59C4344A046099C9B00A14602
:108A30004A449844D30022AA9146049A9944944601
:108A4000089BA59A63448446614494469A468B00E9
:108A5000634400934346586802F036FD4B46186065
:108A60005960029B002B24DB4D46039C0026002707
:108A700001E0286869680CCC01F01AFF02000B00C5
:108A80003000390000F0EEFF083D06000F005C45A5
:108A9000EFD153469E60DF6004239C460433E044DC
:108AA0009C46009BE144E2449845D3D1079B009348
:108AB000D1E600260027ECE794FDFFFF80E30000ED
:108AC00018FEFFFFFFFFFF1F0000703E0000704117
:108AD00000002040FFFFFF3F002180225204141BB2
:108AE0000EAA5450009999420EDD0EA884469B00B0
:108AF0000EAA8900D25861446344CF4800E01A6846
:108B0000821A04C38B42FAD101243CE7059B002B57
:108B100006D1009B0EAA013B9B00D558ED1517E727
:108B20000022C64B300000F0EDFD002800D024E10B
:108B300000253DE732003B000020C14902F02AF940
:108B400006000F00002C00D132E7059A0020BC4936
:108B500000F0A6FB02000B003000390002F01AF909
:108B600006000F0024E7012250E70026002754E604
:108B70004B46059A079388468B000EA9CB58183AA6
:108B800008950592002B0DD18C464146AD4B4344D0
:108B90009B006344043B58680139183A0028F9D017
:108BA00088460592059A0020A54900F079FB4346C6
:108BB00004000D00002B00DA05E29E000EAB9C467F
:108BC0004346DB0066449C46059370AB9946049F80
:108BD00067440097306802F077FC22002B0001F018
:108BE00067FE002238607960974B2000290001F071
:108BF0005FFE083F04000D00043EB945EAD14AABD0
:108C000003939B4600239A46069B42469946434659
:108C10000132029204934B46002B00DAAAE0802036
:108C20008A4B009D9846C0058949002600270024EC
:108C300008E008239C460835E044544511DC4346CF
:108C4000186859682A686B6801F032FE02000B0050
:108C50003000390000F006FF013406000F00A14586
:108C6000E7DA5B46C0C39B4601239C46009BE24477
:108C7000083B0093029B9A45CDD1049B9846A49B48
:108C8000022B00DD8EE0002B37DC1FD1059B002777
:108C90001D00039B00249C461E006544083E2A6874
:108CA0006B683800210000F0DDFE083D07000C0075
:108CB000AE42F4D1089B002B03D080231B069C46B8
:108CC00064443A0023000D990A604B600720079B1B
:108CD00018409B239B009D443CBC90469946A2466D
:108CE000AB46F0BD009B0EA95A1E92000EAB9B58DE
:108CF00007935B025B0A8B5057E64346002B00DA72
:108D000070E100200021DB004AAAD61848AF326883
:108D10007368083E00F0A6FEB742F8D1089B002B0E
:108D200000D025E10B0002004A984B990D9C22606F
:108D3000636002F02FF8434607000C00002B13DDA0
:108D400001254CAEB14638002E0021004C460136BC
:108D50000CCC00F087FEA146B045F7DA089B07006F
:108D60000C00002B00D015E13A0023000D998A6019
:108D7000CB60ABE70026002773E701239C46009BEE
:108D8000E1440225002B00DDEBE532003B00002032
:108D90002B4901F0FFFF06000F0009E60024F2E571
:108DA0004AAB0393A49B032B00D08FE74346002BD1
:108DB00000DC14E1039ADB009B46130091465B4400
:108DC0001E685F68234B43440293DB00994448AB21
:108DD0009A464B465C681B681800210032003B0035
:108DE0000090019100F03EFE04000D0002000B0017
:108DF0000098019901F0CEFF3B00320000F032FEF6
:108E00004B469860D9601C605D6008235B429C46BD
:108E1000E14426002F00CA45DBD14346012B00DC8C
:108E2000E3E0039A13005B441E685F68029BDB006B
:108E300099464A44904610E0FFFFFF000000E03FE3
:108E40000000F03FFFFFFF3F0000703E40E30000E6
:108E5000FB21F93FFFFFFF1F984643465C681B68F4
:108E60001800210032003B000090019100F0FAFD53
:108E700004000D0002000B000098019901F08AFF28
:108E800032003B0000F0EEFD4346039A9860D96043
:108E90001C605D60083B26002F009A42DCD14D46E5
:108EA0009446002600244746083565442A686B68C6
:108EB0003000210000F0D6FD083D06000C00AF4256
:108EC000F4D1039B4A9F5D689968D868089B002B82
:108ED00065D08022120694460D9B6544604464442C
:108EE0001F605D609960D8601E615C61EEE69A4625
:108EF0004B460793059B30005A423900089500F015
:108F0000CFF900223A4B06000F0000F0FBFB0028CF
:108F100024D0384B00223000390001F0C9FC02F0A7
:108F20009DFA52460400950002F0CEFA0022304B22
:108F300001F0BEFC02000B003000390001F02AFFF6
:108F400002F08CFA0EAA50510122059B52441833AC
:108F50009046059393000EAAD45023E65346300062
:108F600039009C0002F07AFA0EAB1851D04619E68F
:108F700080230D9A1B06CB18106053600B00020073
:108F80004A984B9901F006FF434607000C00002B5E
:108F900000DDD5E680231B069C466444E4E62B00F6
:108FA0003A000D9D2A606B600A000300AA60EB6026
:108FB000320023002A616B6188E6099BDB00009385
:108FC00072AB049332E4A49B022B00DDE8E6002B95
:108FD00000DD92E600D079E6002700246AE600264C
:108FE00000246EE70020002198E60026340068E7A0
:108FF000000070410000703EF0B5CE46474680B597
:1090000087B000920193474A4B00814688465B082F
:10901000934207DC4146484602F020FA4146031ECF
:10902000484666D04A4643464846414601F040FC21
:1090300004000D0002000B004846414601F038FCD8
:10904000394A3A4B06000F002000290001F030FC9D
:10905000374A384B01F09EFE22002B0001F028FC1D
:10906000354A364B00F0FEFC22002B0001F020FCBC
:10907000334A344B01F08EFE22002B0001F018FC25
:10908000314B324A00F0EEFC0E9B02900391002B14
:1090900034D00098019900222D4B01F009FC029A6E
:1090A000039B049005913000390001F001FC02009F
:1090B0000B000498059901F06DFE22002B0001F0D1
:1090C000F7FB009A019B01F065FE224A04000D00A7
:1090D000214B3000390001F0EBFB02000B002000B7
:1090E000290000F0BFFC02000B004846414601F099
:1090F00051FE07B00CBC90469946F0BD02000B0033
:109100002000290001F0D4FB124A134B01F042FE6B
:1091100032003B0001F0CCFB4A46434600F0A2FC83
:10912000E7E7C046FFFF3F3E7CD5CF5A3AD9E53D41
:10913000EB9C2B8AE6E55A3E7DFEB157E31DC73E08
:10914000D561C119A0012A3F1111813FA6F8101164
:109150000000E03F495555555555C53F49004B085E
:1091600019007047474AF0B54F4691464B005B0DDA
:1091700099444646D6464A46C0B505000C000E0046
:1091800088460700132A27DC002A4BDB3E4B13419D
:109190009A460B0052461340034318D03B4A3C4BBF
:1091A0002800210000F05EFC0022002300F0A0FA5D
:1091B000002847D0002C04DA80234A465B03134181
:1091C00098444646534600279E43380031001CBC55
:1091D00090469946A246F0BD332A08DD8023DB0085
:1091E0009945F4D102000B0000F03CFCEFE7294A5E
:1091F0009446012263445242DA4092460242E6D04B
:10920000224A234B2800210000F02CFC00220023DE
:1092100000F06EFA002815D0002C1EDB534646469F
:109220009F430FE0194A1A4B2800210000F01AFC56
:109230000022002300F05CFA002803D0002C04DB9D
:109240000027002638003100C1E764006408254388
:109250000027002DF6D0104EF4E74B46142B0BD010
:109260003422D21A012393405D19BD4208D2012352
:109270009C462F00E044D1E7133B9C46E044CDE7F9
:109280002F00CBE701FCFFFFFFFF0F009C7500885C
:109290003CE4377EEDFBFFFF0000F0BF002070478D
:1092A0004B0070B55B0D14000A00002B1AD14B0067
:1092B0005B08034315D0234B002201F0F9FA224B3F
:1092C0009C422DDB0A004B005B0D363B1F4DE31823
:1092D000AB422ADC002B0DDD1D4C1B0522401A433E
:1092E000110070BD1B4DAB42F0D102000B0000F02D
:1092F000B9FBF6E71D00353519DA174B02009C4221
:1093000009DD0B001548164900F032F8134A144BDA
:1093100001F0CEFAE5E70B001248134900F028F8F7
:10932000104A114B01F0C4FADBE70200E9E7084CF0
:10933000363322401B051343190000220B4B01F06A
:10934000B7FACEE700005043B03CFFFFFE07000035
:10935000FFFF0F80FF07000050C300009C750088CE
:109360003CE4377E59F3F8C21F6EA5010000903C23
:1093700030B54A00DB0FDB0752081A43110030BD3D
:1093800002B4714649084900095C49008E4402BC98
:109390007047C046002243088B4274D303098B42B6
:1093A0005FD3030A8B4244D3030B8B4228D3030CB5
:1093B0008B420DD3FF22090212BA030C8B4202D357
:1093C0001212090265D0030B8B4219D300E0090A7F
:1093D000C30B8B4201D3CB03C01A5241830B8B4288
:1093E00001D38B03C01A5241430B8B4201D34B0371
:1093F000C01A5241030B8B4201D30B03C01A5241D6
:10940000C30A8B4201D3CB02C01A5241830A8B425A
:1094100001D38B02C01A5241430A8B4201D34B0243
:10942000C01A5241030A8B4201D30B02C01A5241A7
:10943000CDD2C3098B4201D3CB01C01A524183095B
:109440008B4201D38B01C01A524143098B4201D395
:109450004B01C01A524103098B4201D30B01C01AC0
:109460005241C3088B4201D3CB00C01A524183083A
:109470008B4201D38B00C01A524143088B4201D367
:109480004B00C01A5241411A00D2014652411046C7
:109490007047FFE701B5002000F0F0F802BDC046BC
:1094A0000029F7D076E7704703460B437FD40022AC
:1094B00043088B4274D303098B425FD3030A8B4268
:1094C00044D3030B8B4228D3030C8B420DD3FF22D2
:1094D000090212BA030C8B4202D31212090265D0A0
:1094E000030B8B4219D300E0090AC30B8B4201D353
:1094F000CB03C01A5241830B8B4201D38B03C01A9A
:109500005241430B8B4201D34B03C01A5241030B10
:109510008B4201D30B03C01A5241C30A8B4201D3C1
:10952000CB02C01A5241830A8B4201D38B02C01A6C
:109530005241430A8B4201D34B02C01A5241030AE3
:109540008B4201D30B02C01A5241CDD2C3098B42C8
:1095500001D3CB01C01A524183098B4201D38B0145
:10956000C01A524143098B4201D34B01C01A5241E8
:1095700003098B4201D30B01C01A5241C3088B422D
:1095800001D3CB00C01A524183088B4201D38B0018
:10959000C01A524143088B4201D34B00C01A5241BA
:1095A000411A00D201465241104670475DE0CA0F91
:1095B00000D04942031000D34042534000229C4651
:1095C00003098B422DD3030A8B4212D3FC2289015B
:1095D00012BA030A8B420CD3890192118B4208D331
:1095E000890192118B4204D389013AD0921100E093
:1095F0008909C3098B4201D3CB01C01A52418309A7
:109600008B4201D38B01C01A524143098B4201D3D3
:109610004B01C01A524103098B4201D30B01C01AFE
:109620005241C3088B4201D3CB00C01A5241830878
:109630008B4201D38B00C01A5241D9D243088B42CE
:1096400001D34B00C01A5241411A00D20146634671
:1096500052415B10104601D34042002B00D54942D5
:10966000704763465B1000D3404201B5002000F014
:1096700005F802BD0029F8D016E770477047C046CC
:10968000D0400B1C1141203A03D49C46134118438F
:1096900063465242934018437047C0468446101CAC
:1096A00062468C46191C634600E0C0461FB501F0B7
:1096B00097F8002801D40021C8421FBD10B500F062
:1096C000EFFF4042013010BD10B501F089F80028CD
:1096D00001DB002010BD012010BDC04610B501F017
:1096E0007FF8002801DD002010BD012010BDC0461C
:1096F00010B501F011F8002801DC002010BD012098
:1097000010BDC04610B501F007F8002801DA0020AE
:1097100010BD012010BDC046F0B5CE464746150429
:109720002D0C2E0080B50704140C3F0C9946030C39
:109730007E435D43674363437F19340CE4199C46C1
:10974000A54203D980235B029846C4444B46434359
:109750005143250C36046544360C2404A4195B19C6
:10976000591820000CBC90469946F0BDF0B54E4605
:1097700057464546DE46E0B543025B0A450083B0E6
:109780000F1C99462D0EC60F002D57D0FF2D24D04B
:109790008020DB00C0041843002381469A469B4684
:1097A0007F3D7C027A00FB0F640A120E984623D09C
:1097B000FF2A4BD0E30080240020E4047F3A1C43BE
:1097C000AD186B1C47460193534677403A000F2B68
:1097D00048D87D499B00CB589F46002B00D085E0A0
:1097E00008339A46063B9B467C027A00FB0FFF2516
:1097F000640A120E9846DBD1002C00D090E052464D
:1098000001231A4392460120DBE74C4658461700D5
:10981000022824D0032800D1CFE000220023012811
:109820004DD15802D205400AFF071043384303B018
:109830003CBC90469946A246AB46F0BD002B5BD19E
:1098400004239A46033B00259B46AAE7FF35002CDC
:1098500060D1524602231A4392460220B1E7FF220A
:109860000023DEE74B461B0C9C464B462604360C79
:10987000180461463300220C6446000C43434E43F7
:109880005043544380191A0C1218964203D9802170
:1098900049028C4664441B041B0C1004C01883014D
:1098A0005E1EB341800E1843130C1B199B0103432A
:1098B0001C00230179D5012362081C401443019A3E
:1098C0007F32002A4DDD630704D00F232340042B91
:1098D00000D00434230103D53C4B019A1C40803254
:1098E000FE2ABCDCA3015B0AD2B29AE70C239A469B
:1098F000093BFF259B4654E7180001F071FE4A46DC
:10990000431F76259A4000236D4291462D1A9A46B0
:109910009B4646E7524603231A439246032050E7EC
:10992000200001F05DFE431F2D1A9C40763D002073
:1099300047E780230027DB03FF2272E7424666E702
:109940004C463200584662E780234A46DB031A42FF
:1099500022D01C4220D123435B025B0A4746FF22F0
:109960005FE701239A1A1B2A21DC23000199D340C7
:109970009E318C401A0023005C1EA34113435A07FA
:1099800004D00F221A40042A00D004335A0111D403
:109990009B015B0A002244E780234A46DB03134312
:1099A0005B025B0A3700FF223BE7019587E7002255
:1099B000002336E70122002333E78023DB03234320
:1099C0005B025B0AFF222CE790E30000FFFFFFF73A
:1099D00070B500283DD0C317C5185D40C40F2800DE
:1099E00001F0FEFD9E22121A962A07DCD2B2082848
:1099F00033DD083885406802400A23E0992A0BDDF0
:109A0000052329001B1AD94003001B339D402B005E
:109A10005D1EAB4119430D00052801DD431F9D402C
:109A20002B000F490B406E0709D00F263540042D3F
:109A300005D004335D0102D59F220B40121A9B0111
:109A4000580AD2B24002D205400AE407104320432C
:109A500070BD002400220020F4E76802400AF1E70C
:109A6000FFFFFFFBF0B54F464646D6460C00090304
:109A7000C0B5490A470F5E0039431F03DB0F9C4600
:109A800065007B0A570F1F436D0DE40F760DA1464D
:109A9000C000B846D200AB1B64457BD0002B5FDD15
:109AA000002E00D0A4E03E00164300D112E15E1E5D
:109AB000002E00D09EE1871A4346B842804101251E
:109AC000C91A4042091A0B0200D431E149024E0A78
:109AD000002E00D16EE1300001F082FD0300083B52
:109AE0001F2B00DD61E120223900D21A9E40D140B7
:109AF0009F400E439D4200DD51E15D1B6B1C1F2BFF
:109B000000DD7CE12021C91A3D0030008F408840F3
:109B1000DD40791E8F41310007222843D9400025BE
:109B200007433A40002A09D00F233B40042B05D0BD
:109B30003B1DBB42BF417F42C9191F000B0200D42D
:109B400026E26A1CC64B55056D0D9A4200D106E10E
:109B5000C44AFF080A40530752023B43120B8EE0EF
:109B6000002B00D0B8E06B1C5B055B0D012B00DC0B
:109B700030E1871A4346B842B641CB1A76429E1B63
:109B8000330200D54CE13B003343A1D10022002435
:109B9000002570E0002B00DCE5E0002E00D183E022
:109BA000AF4EB54260D0802636043743B846382BD6
:109BB00000DC3EE1434613431F007A1E97413F18E5
:109BC00087428041404209180B0200D4B0E0A44B08
:109BD00001359D4200D1C3E0A24A7B080A40012121
:109BE0000F401F435108D30707221F433A4099E70C
:109BF0009B4EB54238D0802636043743B846382BC2
:109C000000DDDCE01F2B00DC30E11E004746203E7B
:109C1000F740BC46202B04D04026F31A46469E400F
:109C20003243170063467A1E97411F43CCE0002B56
:109C300000D104E24346134300D159E14B07C00869
:109C400018438023C9081B03194208D04546ED0874
:109C50001D4204D14346D008590708432900420F4A
:109C6000C9007F4D1143C0004B07CA087C49C0089A
:109C700003438D4268D012036D05120B6D0D002158
:109C800012031800130B0A0D12051A43764B2D050B
:109C900013402B435B00E4075B08234319001CBC03
:109CA00090469946A246F0BD3E00164312D05E1E75
:109CB000002E00D000E18718874280414144404295
:109CC000091801250B0233D5022585E764463300C8
:109CD000414610001D00C7E7002D00D0DAE00C005F
:109CE0000443F3D05C1C00D19FE15D4CA64200D13F
:109CF0002FE1DB43382B00DD66E11F2B00DD83E124
:109D000020240500E41A0F00DD40D940A04043465E
:109D1000A7405B1A441EA04198462F433843171AA8
:109D2000BA42924143465242991A64463500CAE605
:109D300007223A40002A00D0F6E64B07CA084849F5
:109D4000FF083B438D4296D11900114300D19EE19B
:109D5000802109030A431203120B414D8FE71500BE
:109D6000002200238BE7002B00D0C7E06B1C5F05AF
:109D70007F0D012F00DCF1E0394DAB4200D1B9E09D
:109D800085180A00854289414244494251180722F8
:109D9000CF076D082F4349083A401D00C2E607224D
:109DA0003049ED1A31403A40BCE63E002838864042
:109DB00000279FE6380001F013FC20308EE6434672
:109DC00013431F007A1E9741C71BB842804140428F
:109DD000091A78E60E003B0006431343002D61D1BB
:109DE000002E00D0F4E0002B00D11BE164463900C6
:109DF000100039E71A4FBB427AD03300FFE630003B
:109E00001F3DE840202B03D04021CB1A9E40374312
:109E10007B1E9F41072207433A400021002589E726
:109E2000171A4346BA42B641591A76428E1B644607
:109E30004EE61F2B00DDADE020264746F61AB74060
:109E4000B9461700B246DF404E463E4337005646FD
:109E5000B240561EB24117434246DA408918AEE678
:109E6000FF070000FFFF7FFFFFFF0F802026474610
:109E7000F61AB740B9461700B246DF404E463E4399
:109E800037005646B240561EB24117434246DA40AA
:109E9000891A99E77F4CA6425BD0802424045B4258
:109EA000214327E7002E0CD1002B00D1CBE06446E4
:109EB00039001000774DD7E6764FBB4218D03300FB
:109EC00075E6002B14D04B07C00818438023C9083F
:109ED0001B03194207D0FC081C4204D17907D008A3
:109EE0000843E14621004C46420FC9001143C0001F
:109EF000684DB9E61D0000220023C0E6002D5BD1AD
:109F00000D00054300D1E2E65D1C00D1B0E0614DDB
:109F1000AE421FD0DB43382B71DC1F2B00DD96E0F7
:109F200020250F00ED1AAF40B9460700AA46DF40D2
:109F30004D463D432F005546A840D940451EA841F7
:109F400088440743BF18974292415142414435002B
:109F50003AE6644635004146100085E60B000343AF
:109F6000002D00D063E6002BF5D04346134300D10B
:109F70007AE6871887428041072241444042091807
:109F80003A400B0200D4D5E6434B01351940C9E5F0
:109F9000380069E61E004746203EF740BC46202BAD
:109FA00004D04026F31A46469E40324317006346CB
:109FB0007A1E97411F4302E6364DAE42CAD0802535
:109FC0002D045B422943A6E70843411E8841A6E6CB
:109FD000002B00D148E6871A4346B842B641CB1A57
:109FE00076429E1B33024BD5171A4346BA42924122
:109FF000591A5242891A072264463A4092E50143AF
:10A000000F00791E8F419DE71C000F00203CE740A8
:10A01000202B03D04024E31A99400843411E884175
:10A0200038437CE60022002425E6171A4346BA424C
:10A030009241591A5242891A6446350043E5414615
:10A040001000144D10E680220024120380E61D004B
:10A050000F00203DEF40BC46202B03D04025EB1ADB
:10A060009940084307006346781E87411F4369E70C
:10A07000871897429B4141445B42C9183500A3E5CC
:10A080003B003343CED0072231003A4052E6002352
:10A090001A00F4E5FF070000FFFF7FFFF0B5574609
:10A0A000DE464E464546E0B5834607000E034800AF
:10A0B00085B092461C00360B400DCD0F002800D114
:10A0C0009DE0954B984239D08023F6001B041E4337
:10A0D000924A7B0F334399469446030063440093AE
:10A0E00000230026FF00029323031B0B9846630006
:10A0F000E40F52465B0D019400D1B3E086498B42D8
:10A1000000D19EE04246D100802212040A4351460B
:10A11000490F11438B46814952468C46009963444E
:10A12000CB1A0021D20000932B0063409A460F2ED9
:10A1300000D905E17A4BB6009B599F465B463343F5
:10A14000994600D0B8E00223082600270090029329
:10A15000CAE7CB463A0002990195019B9A4602292B
:10A1600027D0032900D180E2012944D06D49009B0A
:10A170008C4663441C00002C38DD530700D013E2EA
:10A18000D2085B46DB0109D55946674B19408B461F
:10A190008021C9008C46009B63441C00634B9C4299
:10A1A00007DC5B4664055F075B0217431B0B620D10
:10A1B00002E000230027584A00211B031C0B0B0D53
:10A1C0001B05234314055A4A380013401C435346C9
:10A1D0006400DB0764081C43210005B03CBC9046CA
:10A1E0009946A246AB46F0BD0122524201231B1BF9
:10A1F000382B00DCADE1002200230027DCE75B46C2
:10A20000334399465ED0002E00D18AE1300001F040
:10A21000E7F903000B3B1C2B00DD7BE11D22D31A69
:10A220005A460100DA4008398E4013005F46334336
:10A2300099468F403F4B00261B1A00930023029340
:10A2400052E7414653460B433B499B468C46009B95
:10A25000634400935B46002B3BD1022300221E4344
:10A26000022161E7434613439B4637D04346002B08
:10A2700000D162E1404601F0B3F903000B3B1C2B17
:10A2800000DD53E102004146083A914088461D2115
:10A29000CB1A5146D9400B0041460B439B465346CF
:10A2A00093401A00009B25499C46604403008C465D
:10A2B00063440093002137E70323B14600900C2646
:10A2C000029311E700230093013304260027029331
:10A2D0000AE70323C3461E43032125E701331E4338
:10A2E0000022012120E700239A46802300271B0338
:10A2F000094A61E7802349461B03194200D1E2E085
:10A300005946194200D0DEE00B431B0317001B0B1C
:10A31000A246014A50E7C046FF07000001FCFFFFCC
:10A32000D0E30000FF030000FFFFFFFEFE07000078
:10A33000FFFF0F800DFCFFFF01F8FFFFF30300009C
:10A34000D94500D9CBE000D1C6E03C004846002703
:10A35000009B013B00935B46160E1B021E4313023B
:10A36000984633041B0C9946310C0191FFF798F87D
:10A370004A4642430B04210C050019438A4207D97F
:10A380008919013D8E4203D88A4201D9851E891957
:10A39000881A0199FFF784F809048C464A4621047B
:10A3A00064464243090C030021438A4204D98919B7
:10A3B000013B8E4200D8F1E02D041D43AB464346DD
:10A3C000891A4246280C12041D0C5B46140C22000C
:10A3D0001B041B0C5A4303946B434443029568438C
:10A3E0001B19150CEB189C4203D980246402A44667
:10A3F00060441C0C15041B042D0C20185D198142AF
:10A4000077D373D00C1AA24A7D1BAF42BF4194464A
:10A41000009B7F426344E01B1C00864200D1DBE0CE
:10A420000199FFF73DF84A4642430B04290C070007
:10A4300019438A4207D98919013F8E4203D88A42BB
:10A4400001D9871E8919881A0199FFF729F809048B
:10A450004A46894629044D464243090C03002943D4
:10A460008A4207D98919013B8E4203D88A4201D911
:10A47000831E89193F04891A3A00039F1A43380042
:10A4800013041B0C584381460298150C6F43434339
:10A4900045434846000C8446DB1963449F4203D978
:10A4A000802040028446654448461F0C00041B047B
:10A4B000000C7D191818A94200D284E000D17FE079
:10A4C00001231A4357E680234A461B0313431B0309
:10A4D0001B0BAA466F4A6FE6BA4200D935E74B46D6
:10A4E000DC0758087B081C43FF0734E70024AF4211
:10A4F00089D247444745A4415B466442A419641885
:10A50000013BA6421ED2A0426DD800D1B6E0241A6B
:10A510009B4678E703005A46283B9A40002791461D
:10A5200088E6584601F05CF8203072E60300524697
:10A53000283B9A4093460022B4E6504601F050F87A
:10A5400020309AE6A642E2D1B845DCD9341A9B46BF
:10A5500059E71F2B65DC504C0099A4465C466144CA
:10A5600008008C4011008240D940501E82410C43AB
:10A5700014435A46DA401300620709D00F222240E2
:10A58000042A05D02200141D9442894149425B18D7
:10A590001A0262D50122002300270DE68A4200D864
:10A5A0000AE7831E891907E70F231340042B00D104
:10A5B000E6E5171D9742924153429B44FA08E0E5B5
:10A5C000002800D1D7E57118531EB14227D3A94204
:10A5D00015D358D01A0073E7002B00DC04E60123E2
:10A5E00000229B44CDE502234744474589415B4215
:10A5F0009C46494289190C19E344241A03E743464F
:10A600005F0047459B41B8465B429E19023A891953
:10A61000A94200D054E7404500D051E7ABE51A000D
:10A62000F6E71F215F4649420C1BE740202B07D06D
:10A630001A49009B8C46634418005B4683401A43CA
:10A64000501E82413A4307270023174009D00F21AB
:10A65000002311401400042995D122005F075B02FA
:10A660001B0BD20817430022A6E5802359461B0383
:10A670000B431B0317001B0B064A9DE5BD42B2D8D6
:10A680009B460024BFE68045B9D31A00C3E7C04605
:10A69000FF030000FF0700001E0400003E0400004E
:10A6A000F0B54F464646D6468446C0B58046194E5C
:10A6B00018030F034D00000B5C0082463F0B6D0D2D
:10A6C000C90F9146640DDB0F0120B5420AD0B44298
:10A6D00003D0A54201D157450CD01CBC90469946E9
:10A6E000A246F0BD66463E43F7D1AC42F5D1544692
:10A6F0001443F2D10120C845EFD1994207D0002D73
:10A70000EBD163461F433800471EB841E5E7002000
:10A71000E3E7C046FF070000F0B54F464646D64681
:10A720004D00C0B50E03C90F8A462C491F035C00BB
:10A730008046360B6D0D91463F0B640DDB0F8D424D
:10A740001ED08C4216D0002D1ED130438446002CE2
:10A7500001D13A4323D06246002A1AD09A4529D023
:10A76000514602200139084001381CBC90469946E8
:10A77000A246F0BD39001143E5D002204042F4E783
:10A780003043FAD1AC420FD0002C0FD13A43E7D07E
:10A790000CE00122013B934318000130E5E76346DA
:10A7A0000020002BE1D0DBE73A43E6D19A45D7D130
:10A7B000A542D5DCA54205DBBE42D1D808D0002099
:10A7C000BE42D2D250460123013898430130CCE733
:10A7D000C845C5D80020C845F4D3C6E7FF07000028
:10A7E000F0B54F464646D6464D00C0B50E03C90FDC
:10A7F0008A462E491F035C008046360B6D0D91463C
:10A800003F0B640DDB0F8D4218D08C4211D0002D10
:10A8100018D130438446002C1ED13A431CD16346E4
:10A820000020002B30D05146022001390840013869
:10A830002AE039001143EAD0022025E03043FBD161
:10A84000AC4226D0002C26D13A4324D151460220D6
:10A8500001390840013817E06246002A0FD09A45B6
:10A86000E1D1A54205DBBE42DDD819D00020BE42B1
:10A870000AD25046012301389843013004E00122F6
:10A88000013B9343180001301CBC90469946A246F8
:10A89000F0BD3A43D0D19A45C5D1A542C3DCE0E72B
:10A8A000C845C0D80020C845E3D3EDE7FF07000046
:10A8B000F0B55746DE464E464546E0B583460600AF
:10A8C0000F03480087B092461D003F0B400DCC0F90
:10A8D000002800D16FE0DE4B984238D08023FF0083
:10A8E0001B041F43730F3B430193DA4B0027994628
:10A8F00000239B46F60081442B0369001B0B524644
:10A900009846490DED0F002900D185E0D04B9942C2
:10A9100000D173E04346DA0080231B041343524600
:10A92000CC48520F84461343524600206144D20063
:10A9300089442100694000918C46012149448A469E
:10A940000F2F00D990E0C449BF00CF59BF465B46E6
:10A950003B43019300D06AE1022308270026814689
:10A960009B46C9E732005846019B61460091022888
:10A9700000D175E0032800D1FEE1012800D02CE1D0
:10A9800000230027002600253F032A0D3F0BB34874
:10A9900012053A4302401B051343009A5B00D1079E
:10A9A0005B080B433000190007B03CBC9046994649
:10A9B000A246AB46F0BD5B463B43019300D12FE17D
:10A9C000002F00D1A5E1380000F00AFE03000B3B88
:10A9D0001C2B00DD96E11D22D31A5A460100DA40F5
:10A9E0005E4608398F4013008E403B4301939C4BD9
:10A9F00000271B1A994600239B467DE74146534694
:10AA00000B4393498C46E144002B00D01AE102220B
:10AA10000220174300228CE7134300D10DE1434687
:10AA2000002B00D181E1404600F0DAFD02000B3A34
:10AA30001C2A00DD72E10100434608398B4098462C
:10AA40001D239A1A5346D3401A00434613435246D5
:10AA50008A404946081A824989468144002068E7AD
:10AA60007B4B002700268EE7140C1204120C1100F9
:10AA7000370C3604350C794328008C462E00604391
:10AA80006044834656432100300C80465846794343
:10AA900040440291844506D98846802149028C466B
:10AAA000E044414602913604010C360C00048B460A
:10AAB00081191E0C1B041B0C0391190079438C4651
:10AAC000280075436544A8465843050C4544774320
:10AAD000A94203D9802149028C466744290C8C463F
:10AAE00039000004000C2D042D186144AB4405917D
:10AAF0005946049101990F043F0C080C3900514349
:10AB00004243904602008C46090C8B4662437C43CC
:10AB100044445C44A04503D980214902884642440C
:10AB2000210C884661460904090C8C4639005943BA
:10AB3000434370437E430F0CF6182404BE1964444B
:10AB400042448C46B34203D980235B02984640447A
:10AB5000029B61469846049B370443449B46AB45A1
:10AB6000AD416B420D0405992D0C8C467F1967444D
:10AB7000FD18A8465D462D19A542A441934664429E
:10AB8000A446C344DC448F42BF4198459B41934552
:10AB90009241A445A4415B427F421F43360C52427E
:10ABA0006442BF192243BF18624638184302D20DCF
:10ABB000039913436A020A43501E82416146ED0D18
:10ABC0002A434E023243D90100D4B3E00126500893
:10ABD00032400243DE0732435B08224C5444002CCF
:10ABE00062DD510709D00F201040042805D0101D48
:10ABF0009042924152429B180200D90104D5802410
:10AC00001948E400034054441848844200DD27E713
:10AC10005E075B02D2081F0B630516435B0DB2E6AD
:10AC2000002399460133042700269B4664E603234C
:10AC3000019781460C279B465EE6012201201743BF
:10AC4000002276E6032303201F43434671E6C046F5
:10AC5000FF07000001FCFFFF10E40000FFFF0F8072
:10AC60000DFCFFFFFF030000FFFFFFFEFE070000DB
:10AC70000023802700933F030026434B83E6019B7C
:10AC80003200A446584670E6AC466EE6802701992D
:10AC90003F0339422DD03B422BD11F433F033F0B93
:10ACA00000951600384B6EE601252D1B382D00DD72
:10ACB00066E61F2D40DC35481C00504416008240DB
:10ACC0008440EE40501E824134431443EB406207FF
:10ACD00009D00F222240042A05D02200141D9442DC
:10ACE000804140421B181A023ED50123002700264E
:10ACF00049E68027019B3F031F433F033F0B00941E
:10AD0000214B40E603005A46283B9A400026019218
:10AD10006DE6584600F064FC203057E603005246CA
:10AD2000283B9A401300002293E6504600F058FC5E
:10AD300020307BE6CA4650E71F201E004042041B1D
:10AD4000E640202D03D0124C5444A3401A43501E19
:10AD50008241324307260027164009D00F200023E6
:10AD6000104014000428B9D122005E075B021F0BBB
:10AD7000D2081643002306E680273F031F433F0304
:10AD80003F0B1600004BFEE5FF0700001E0400000D
:10AD90003E040000F8B557464E464546DE460C00D8
:10ADA0000903E0B5490A460F5F0031431E03DB0F7C
:10ADB000760A9B46530F3343C84E6500C000E40F2C
:10ADC000D2006D0DA24681467F0D9C469046B7424B
:10ADD00000D1B9E05B46012673409B46EE1BA345BC
:10ADE00000D183E0002E63DD002F00D0B1E0634688
:10ADF000134300D123E1731E002B00D0BAE1861A61
:10AE00006346B04280410125C91A4042091A0B022B
:10AE100000D447E149024B0A98464346002B00D133
:10AE200089E1404600F0DCFB0300083B1F2B00DDFE
:10AE30007CE120223000D21A4146D04099400200E5
:10AE40009E400A439D4200DD6AE15D1B6B1C1F2B87
:10AE500000DD94E1202110003500C91A8E40DA404F
:10AE60008840DD40711E8E411100072228430025D5
:10AE700006433240002A09D00F233340042B05D06B
:10AE8000331DB342B641764289191E000B0200D42D
:10AE90003DE26A1C914B55056D0D9A4200D119E1B6
:10AEA0008F4AF6080A40570752023743120B9BE0BD
:10AEB000002E00D0C5E06E1C7605760D012E00DC5C
:10AEC00048E16746861ACB1BB042BF417F42B84675
:10AED0001F004346FF1A3B00B8461B0200D55FE146
:10AEE00037439AD100220024002579E0002E00DCAF
:10AEF000FAE0002F00D18DE0784B9D4267D080238F
:10AF000067461B041F43BC46382E00DC52E16346F3
:10AF100013435A1E93411E1886428041404209182D
:10AF20000B0200D4BEE06D4B01359D4200D1D2E052
:10AF30006B4A73080A4001210E401E435108D30793
:10AF400007221E43324095E71E00164300D045E716
:10AF500040E7624B9D423AD0802367461B041F4363
:10AF6000BC46382E00DDEBE01F2E00DC3AE133005A
:10AF70006746203BDF403B00202E05D04027BF1B0B
:10AF80006646BE40324390464646721E9641334363
:10AF9000DAE0002B00D114E26346134300D168E1EC
:10AFA00080234E07C008C9081B030643194208D076
:10AFB0006046C008184204D163460100D2085E070B
:10AFC0001643F3009946C900720F444D11434B4696
:10AFD000DE08424B4F073743CA089D4200D16EE05E
:10AFE00012036D05120B6D0D00211203130B0A0DD8
:10AFF00012051A433B4B2D0513402B435B00E4071E
:10B000005B082343380019003CBC90469946A24691
:10B01000AB46F8BD6346134311D0731E002B00D01E
:10B0200007E18618864280416144404209180125A3
:10B030000B0237D502257BE73E006146914635007D
:10B04000C5E75C46002D00D0E1E00B000343F3D0E0
:10B05000731C00D1ACE1214B9F4200D13AE1F34394
:10B06000382B00DD6FE11F2B00DD8CE120250E0069
:10B07000ED1AAE40B0460600AA46DE4045463543CE
:10B080002E005546D940A8406346451EA8415B1A8C
:10B090009C463043161AB242924163465242991A74
:10B0A0003D00B4E607223240002A00D0E4E60B4B14
:10B0B000F6084F073743CA089D4200D090E73B008F
:10B0C000134300D1A6E180231B031A431203120B82
:10B0D000024D89E715000022002785E7FF070000E1
:10B0E000FFFF7FFFFFFF0F80002E00D0C7E06B1C2B
:10B0F0005E05760D012E00DCF0E0C84DAB4200D1BC
:10B10000B9E085180A0085428941624449425118D4
:10B110000722CE076D082E43490832401D00A9E6DC
:10B12000BF49ED1A114007223240A3E63200283809
:10B130008240002686E6300000F052FA203073E6A6
:10B14000634613435A1E9341C61AB042804140429F
:10B15000091A5CE60E00674606431743002D5ED1D0
:10B16000002E00D0F3E0002F00D11EE15C466146C6
:10B1700091462CE7A94FBE427BD01E00F1E610009D
:10B180001F3DE840202B03D04021CB1A9A401643A4
:10B19000731E9E410722064332400021002583E7AB
:10B1A000161A6346B2428041591A40420B1A984619
:10B1B0005C4632E61F2E00DDABE02027BB1B9A4623
:10B1C00063465746BB40994613004F46F3401F4322
:10B1D0003B005746BA40571EBA4113436246F240FD
:10B1E000891898E62027BB1B9A4663465746BB4002
:10B1F000994613004F46F3401F433B005746BA4061
:10B20000571EBA4113436246F240891A9CE7834BAA
:10B210009F425FD080252D047342294320E7002EF2
:10B220000CD1002F00D1D0E05C46614691467B4DA9
:10B23000CDE67A4FBE421CD01E0065E6002F18D026
:10B24000C0084E0706438020C9080003014208D009
:10B250006346DC08044204D12100DA46D2085E07C6
:10B260001643F300994601245346C900720F114357
:10B270001C406A4DABE61D0000220027B4E6002DFD
:10B2800059D10B00034300D1D6E6731C00D1B2E0C4
:10B29000624B9F421ED0F343382B6FDC1F2B00DD27
:10B2A00097E020250E00ED1AAE40B0460600AA46F3
:10B2B000DE40454635432E005546A840D940451E40
:10B2C000A8418C440643B6189642924151426144CB
:10B2D0003D0025E63D006146914678E60B000343BC
:10B2E000002D00D055E6002BF5D06346134300D166
:10B2F0006DE686188642804161444042091800226A
:10B300000B0200D4D0E6464B01351940B2E5B146F8
:10B310005DE633006746203BDF403B00202E05D032
:10B320004027BF1B6646BE40324390464646721ECB
:10B3300096413343EFE5394B9F42CBD080252D0416
:10B3400073422943A8E70843411E8841A2E6002F23
:10B3500000D13CE66346861ACF1AB0429B415B425D
:10B36000FB1A98461B024ED5161A6346B24292410A
:10B37000591A5242891A5C4600227BE501430E00AD
:10B38000711E8E419FE71D000E00203DEE40B0462D
:10B39000202B04D04025EB1A9940084381464846AB
:10B3A0004346411E8841184374E60022002417E6F4
:10B3B000161A6346B2429241591A5242891A3D0006
:10B3C00025E561469146154D01E6802200241203D1
:10B3D00079E61D000E00203DEE40B046202B04D043
:10B3E0004025EB1A9940084381464E464346711E5C
:10B3F0008E411E4367E7861896429B4161445B423B
:10B40000C9183D008CE547463743CED00722414658
:10B41000324049E600273A00E6E5C046FF07000053
:10B42000FFFF7FFF70B50C4E0D031C0349005B004E
:10B430002D0B490D240B5B0DB14208D006490020AD
:10B440008B4203D114432000441EA04170BD05432C
:10B450000120002DFAD1F1E7FF07000030B5144DAF
:10B460000A034B00120B5B0DC90F0024AB4211DD28
:10B47000104CA34210DC8024640322430E4CE41AD7
:10B480001F2C0CDD0D48C31ADA4013005C42002962
:10B4900000D11C00200030BD094BCC18FAE7094D43
:10B4A000E040AC4663449A4013000343EEE7C046D5
:10B4B000FE0300001D04000033040000130400001C
:10B4C000FFFFFF7FEDFBFFFF70B500282DD0C317F6
:10B4D000C5185D40C40F280000F082F8154B1B1AF8
:10B4E0005B055B0D0A2815DD0B38854000222D0316
:10B4F0002D0B002110002D030A0D2D0B12052A43E0
:10B500000D4D1B052A4013435B00E4075B082343F2
:10B51000190070BD02002900153291400A000B216C
:10B52000081AC5402D032D0BE3E700240023002556
:10B530000022DEE71E040000FFFF0F804100090E1D
:10B540004B1C70B5DBB24602750AC40F012B14DD2B
:10B55000E0239B006D07360BCB1800210A0D280055
:10B5600012051C4D32435B052A405B0813435B0008
:10B57000E4075B082343190070BD002914D1002D96
:10B580001ED0280000F02CF80A281CDC0B232A000F
:10B590001B1ADA40030015339D400F4B12031B1A90
:10B5A0005B05160B5B0DD8E7002D06D0320B80260D
:10B5B00036036D071643094BCFE7084B0026CCE74F
:10B5C00000230026C9E703002A000B3B9A40002510
:10B5D000E3E7C046FFFF0F8089030000FF0700007C
:10B5E0001C2101231B04984201D3000C10391B0AB3
:10B5F000984201D3000A08391B09984201D3000977
:10B60000043902A2105C40187047C04604030202CD
:10B6100001010101000000000000000030B51C0025
:10B62000094B05001B6885B0D868084B002A01D17A
:10B63000074B1A000292019300912B00220005494A
:10B6400000F026F800F0A6FD8000002050E4000085
:10B650006BD200005DE40000014B18687047C046E3
:10B6600080000020084B10B50400002B02D0002100
:10B6700000E000BF054B1868836A002B00D0984794
:10B68000200001F05DFBC046000000008CE40000DB
:10B690000EB403B5010003AB044804CB006801936A
:10B6A00000F076F802B008BC03B018478000002014
:10B6B00070B500260C4D0D4C641BA410A64209D198
:10B6C000002601F03FFB0A4D0A4C641BA410A64261
:10B6D00005D170BDB300EB5898470136EEE7B300D3
:10B6E000EB5898470136F2E7500200205002002044
:10B6F0005002002060020020002310B59A4200D1C1
:10B7000010BDCC5CC4540133F8E710B5884202D9AF
:10B710008B18984203D3002307E08B5C8354013AD3
:10B72000FBD210BDCC5CC45401339A42FAD1F8E785
:10B7300003001218934200D1704719700133F9E7E2
:10B74000936810B5013B9360002B04DA9469A3421F
:10B7500007DB0A2905D01368581C1060197008000F
:10B7600010BD00F04BFC0100F9E7F8B506000F0032
:10B770001400D518AC4201D1002007E021783A002E
:10B780003000FFF7DDFF0134431CF3D1F8BD0000AA
:10B79000F0B59FB002900F0016000593002805D069
:10B7A00083690493002B01D100F0F4FD7B4B9F4291
:10B7B0005BD1029B5F68BB891B0762D53B69002B8D
:10B7C0005FD0002306AC6361203363761033A37629
:10B7D00035002B78002B01D0252B5CD1AB1B0493BB
:10B7E0000CD0320039000298FFF7BFFF431C00D194
:10B7F000C4E06269049B9446634463612B78002B28
:10B8000000D1BBE0012200235242626002A95432FF
:10B8100052186E1C2360E360A3601370A365317837
:10B8200005225F4800F0D4FE751C002835D122683F
:10B83000D30604D5532302A95B18202119701307DE
:10B8400004D5532302A95B182B21197033782A2BB6
:10B850002CD0350000210A20E3682A786E1C303A8B
:10B86000092A64D900292ED026E04E4B9F4202D1EE
:10B87000029B9F689FE74C4B9F429CD1029BDF68D5
:10B8800099E73900029800F00FFC002899D00120B8
:10B8900040421FB0F0BD01359BE7414B2268C01A02
:10B8A00001238340134323602E00B8E7059B191D35
:10B8B0001B680591002B01DB099304E05B42E36008
:10B8C0000223134323602B782E2B0AD16B782A2B6B
:10B8D00035D1059B02351A1D1B680592002B2BDB09
:10B8E0000793324E29780322300000F071FE0028C1
:10B8F00006D04023801B8340226801351343236018
:10B90000297806222A486E1C217600F061FE002864
:10B910003AD0284B002B25D10722059B07339343B0
:10B92000083305936369039A9B18636150E74343A7
:10B9300001219B18350090E701235B42D0E70023EB
:10B940000A201A000135636029786E1C30390929F4
:10B9500003D9002BC5D00792C3E7424301235218F5
:10B960003500F1E705AB00933A00134B2100029834
:10B9700000E000BF0390039B0133D3D1BB895B067A
:10B9800000D584E70B9884E705AB00933A000A4B97
:10B990002100029800F080F8ECE7C046E4E40000E3
:10B9A00090E4000004E50000C4E4000096E4000018
:10B9B0009AE40000000000006BB70000F7B5150026
:10B9C00001938A680B6900900C00934200DA13001F
:10B9D00022002B6043321278002A01D001332B6001
:10B9E00023689B0602D52B6802332B600627236849
:10B9F0001F4027D0230043331B785A1E93412268EF
:10BA0000920630D42200019943320098089EB04734
:10BA1000431C25D0062320682A68E16803400025DE
:10BA2000042B03D18D1AEB43DB171D40A368226959
:10BA3000934201DD9B1AED180027BD4220D1002062
:10BA400010E00137E3682A689B1ABB42D2DD22006E
:10BA50000123193201990098089EB047431CF0D188
:10BA600001204042FEBD3020E11843310870210022
:10BA70005A1C45310978A218433202331170C1E7CC
:10BA8000220001231A3201990098089EB047431CF6
:10BA9000E6D00137D1E70000F0B589B004920A0082
:10BAA00043320593039002920A7E0C000E9B6E2A8D
:10BAB00000D186E01FD8632A33D008D8002A00D1ED
:10BAC0008CE0582A4DD0250042352A7030E0642A97
:10BAD00001D0692AF7D1196825680A1D280629D5D9
:10BAE00008681A60002803DA2D23029A4042137076
:10BAF0006B4E0A274FE0732A74D008D86F2A1FD0E4
:10BB0000702AE0D1202209680A43226003E0752AE6
:10BB100016D0782AD7D12200782145321170614E93
:10BB200022E025001A684235111D196013682B7038
:10BB3000012365E008681A606906D3D500B2D1E731
:10BB400019682568081D186008682E0605D5544E2A
:10BB500008276F2A1BD00A2719E06D06F7D580B297
:10BB6000F5E745314E4E0A7018682268011D0068DD
:10BB70001960150621D5D30702D520231A43226068
:10BB80001027002803D1202322689A432260230033
:10BB9000002243331A706368A360002B58DB042231
:10BBA000216891432160002854D1029D002B5AD076
:10BBB0002500337842352B7055E05506DBD580B231
:10BBC000D9E71A680D68101D4969186013682E06B8
:10BBD00001D5196002E06D06FBD519800023029D96
:10BBE00023614FE01A68111D196015680021626811
:10BBF000280000F0EDFC002801D0401B6060636865
:10BC000023610023029A13703CE023692A000499FF
:10BC10000398059DA847431C3ED023689B0715D475
:10BC2000079BE068984239DA180037E022000123C8
:10BC3000193204990398059EB047431C2CD0013556
:10BC4000E368079A9B1AAB42F0DCE9E70025F7E7C7
:10BC50000028ADD0029D3900FDF722FC735C013D48
:10BC60002B700028F7D1082F09D12368DB0706D5F0
:10BC700063682269934202DC3023013D2B70029BF2
:10BC80005B1B2361059B07AA00932100049B03987B
:10BC9000FFF794FE431CB8D10120404209B0F0BD2B
:10BCA000A1E40000B2E400000D4B70B51C68050073
:10BCB000A36B002B0FD1182000F06EFC094BA06382
:10BCC0000360094B01224360084B83600B2383818F
:10BCD0000023026143610022A36B1D615A6170BDA4
:10BCE000800000200E33CDAB34126DE6ECDE050093
:10BCF000124B10B51C68A36B002B0FD1182000F05D
:10BD00004BFC0F4BA06303600E4B012243600E4BB4
:10BD100083600B238381002302614361A46B0B4A80
:10BD2000206961690A4BFDF7F7FC012200238018A6
:10BD30005941206161614800400810BD8000002029
:10BD40000E33CDAB34126DE6ECDE05002D7F954C45
:10BD50002DF451580CB430B5164B9DB00C1E1D6817
:10BD600008DA8B2301202B6040421DB030BC08BC98
:10BD700002B01847822302A99B008B810023029006
:10BD800008619C4200D0631E8B604B6101235B42C3
:10BD9000CB81209A21AB2800019300F055FD431C74
:10BDA00001DA8B232B60002CDFD00023029A137062
:10BDB000DBE7C046800000200EB400B50B499CB004
:10BDC0001DAB02900690079104910948094904CBE4
:10BDD0000591006802A9019300F036FD0023029A44
:10BDE00013701CB008BC03B01847C046FFFFFF7FAC
:10BDF000800000200802FFFF020010B51378541CD9
:10BE0000002B05D1CC5CD4540133002CFAD110BDE9
:10BE10002200F3E7C9B20378002B04D08B4200D193
:10BE200070470130F7E74B42594149420840F7E774
:10BE300002780B78002A03D0013001319A42F7D002
:10BE4000D01A70470023C25C0133002AFBD1581E70
:10BE50007047002330B59A420AD0013AC45CCD5CE9
:10BE6000AC4204D1934202D00133002CF6D1631BC3
:10BE7000180030BD30B50500002A00D130BD0C7867
:10BE8000013A6B1C2C700131002C05D19A189A4292
:10BE9000F4D01C700133FAE71D00EDE710B503780C
:10BEA000002B0FD10B785A4253415B42184010BD12
:10BEB0000023CA5C002AFAD0C45C944201D1013349
:10BEC000F7E701300378002BF2D11800EFE700000C
:10BED000F0B51F000E0087B00590019102920C98FA
:10BEE000347800F0EAFA082200194378751C1340F0
:10BEF00036D12D2C36D1B51C74780126002F62D096
:10BF0000102F09D1302C07D120222B789343582BA6
:10BF100054D110276C7802352D4B3900F3181800D6
:10BF20000393FDF7BDFA0491012100234942020069
:10BF30008C4618002100303909291AD80C00A74274
:10BF400023DD591C09D06346824206D302D10499ED
:10BF5000A14202DB0123784320182C780135E9E760
:10BF60002E00BCE72B2C01D01E00C7E7B51C74784F
:10BF7000FAE721004139192901D8373CDFE72100D0
:10BF80006139192901D8573CD9E75A1C08D1059ABB
:10BF900023331360029B0398002B09D107B0F0BD37
:10BFA000002E00D04042029A002AF7D0002B01D088
:10BFB0006B1E0193029B019A1A60EFE73024002F59
:10BFC000AAD10827A8E7302C9ED00A27A4E7C046AC
:10BFD000FFFFFF7F37B51300064A05001068046AAB
:10BFE000002C00D1044C0A0000942900FFF770FFD8
:10BFF0003EBDC04680000020E4000020F8B50500EA
:10C000000E001400002804D08369002B01D100F039
:10C01000C1F9224B9C422DD16C68A369A360A3890E
:10C020001B0731D52369002B2ED023682269F7B274
:10C03000981A6369F6B2834205DC2100280000F0FB
:10C040003BF9002826D1A3680130013BA360236897
:10C050005A1C22601F706369834204D0A389DB07E6
:10C060001AD50A2E18D12100280000F025F9002841
:10C0700012D00FE00A4B9C4201D1AC68CDE7094BCE
:10C080009C42CAD1EC68C8E72100280000F00CF8F7
:10C090000028CAD0012676423000F8BDE4E4000052
:10C0A00004E50000C4E40000364B70B51D680600CE
:10C0B0000C00002D05D0AB69002B02D1280000F048
:10C0C00069F9314B9C420FD16C680C23E25E93B24C
:10C0D00019072DD4D90611D4092301203360373331
:10C0E0001343A381404270BD284B9C4201D1AC68F0
:10C0F000EBE7274B9C42E8D1EC68E6E75B0713D5FA
:10C10000616B002908D023004433994202D03000EB
:10C1100000F06AFA002363632422A3899343A38176
:10C1200000236360236923600823A2891343A3814A
:10C130002369002B0BD1A0218022A38989009200C2
:10C140000B40934203D02100300000F0E1F90123BD
:10C15000A289134011D00023A36063695B42A361ED
:10C16000002023698342BED10C23E25E1306BAD5B8
:10C1700040231343A3810138B5E7920700D46369D4
:10C18000A360EDE780000020E4E4000004E5000087
:10C19000C4E4000010B5062000F090FC012000F07F
:10C1A000CFFD0000F7B58A8905000C00130760D4A5
:10C1B0004B68002B04DC0B6C002B01DC0020FEBD67
:10C1C000E76A002FFAD000232E682B6080235B01E2
:10C1D000216A1A4034D0606DA3895B0706D5636875
:10C1E000C01A636B002B01D0236CC01A0200216AB5
:10C1F00000232800E76AB847A189431C06D12B68B1
:10C200001D2B30D82B4ADA40D3072CD5002363608E
:10C2100023692360CB0405D5431C02D12B68002B76
:10C2200000D16065616B2E600029C7D023004433C4
:10C23000994202D0280000F0D7F900206063BEE7E1
:10C2400001232800B847431CC6D12B68002BC3D05C
:10C250001D2B01D0162B01D12E60AFE74023A28900
:10C260001343A381ABE740230B430120A38140424A
:10C27000A5E70F69002FA1D00B680F60DB1B0193AE
:10C280000023920700D14B69A360019B002B00DCC7
:10C2900094E7019B3A00216A2800A66AB04700286B
:10C2A00003DC4023A2891343DFE7019B3F181B1ADD
:10C2B0000193EAE7010040200B6970B505000C000E
:10C2C000002B01D1002070BD002804D08369002B11
:10C2D00001D100F05FF80B4B9C4209D16C680C2235
:10C2E000A35E002BEED021002800FFF75BFFEAE7FA
:10C2F000054B9C4201D1AC68F1E7044B9C42EED166
:10C30000EC68ECE7E4E4000004E50000C4E40000AD
:10C31000002310B50400036043608360818143669D
:10C32000C281036143618361190008225C30FFF719
:10C33000FFF9054B24626362044BA362044BE36282
:10C34000044B236310BDC046FDCA000025CB00008E
:10C350005DCB000089CB000010B5024900F08CF8DD
:10C3600010BDC046B9C2000070B568254A1E5543CD
:10C370000E002900743100F081F9041E08D000215C
:10C380002A00016046600C30A0606832FFF7D0F9E7
:10C39000200070BD836913B50400002B28D183648D
:10C3A000C3640365134B144A1B688262019398426D
:10C3B00001D101238361200000F020F8606020009B
:10C3C00000F01CF8A060200000F018F80022E060E7
:10C3D00004216068FFF79CFF01220921A068FFF794
:10C3E00097FF02221221E068FFF792FF0123A36169
:10C3F00013BDC0468CE4000059C30000F8B51C4BC7
:10C4000007001E68B369002B02D13000FFF7C2FF9E
:10C410004836B4687368013B04D53368002B07D0F5
:10C420003668F6E70C22A55E002D0DD06834F2E7E1
:10C4300004213800FFF798FF30600028F0D10C236A
:10C4400004003B602000F8BD20000A4B65662560B3
:10C450006560A560E36025616561A561082229002A
:10C460005C30FFF765F96563A563A564E564E9E7FA
:10C470008CE400000100FFFFF7B504000700002670
:10C4800001914834002C01D13000FEBD6368A568DD
:10C490000093009B013B009301D52468F2E7AB8930
:10C4A000012B08D90E22AB5E013304D029003800DD
:10C4B000019B984706436835EBE7EC30006870470E
:10C4C00070B50E001D000E23C95E96B01400002941
:10C4D00007DA00232B60B3891B0611D48023DB000D
:10C4E0000FE06A4600F088FB0028F2DBF022019B97
:10C4F00012021340054A9B185A4253412B60EDE744
:10C5000040230020236016B070BDC04600E0FFFF4E
:10C51000F7B502268B8905000C00334206D02300B4
:10C5200047332360236101236361F7BD01AB6A4692
:10C53000FFF7C6FF00990700280000F09FF80028C9
:10C5400008D10C22A35E9A05EFD4032293431E4325
:10C55000A681E4E70F4BAB628023A28920601343DE
:10C56000A381009B20616361019B002B0DD00E23F2
:10C57000E15E280000F052FB002806D00322A389C8
:10C5800093431A0001231343A381A0893843A08158
:10C59000CBE7C04659C3000010B5034B0100186833
:10C5A00000F06CF810BDC0468000002082B0002969
:10C5B00000D101A9101E06D0002B06D013780B6005
:10C5C0001078431E984102B0704702204042FAE7BB
:10C5D000C9B28218904201D10020704703788B4283
:10C5E000FBD00130F6E7000070B50500002910D03F
:10C5F0000C1F2368002B00DAE418280000F034FB3D
:10C600001D4A1368002B05D163601460280000F0F8
:10C610002CFB70BDA34209D9216860188342F3D175
:10C6200018685B6841182160EEE713005A68002A19
:10C6300001D0A242F9D919685818A0420BD120683C
:10C640000918581819608242E0D1106852684118E0
:10C6500019605A60DAE7A04202D90C232B60D5E7B3
:10C6600021686018824203D1106852684118216025
:10C6700062605C60CAE7C0462C1C0020032370B5D2
:10C68000CD1C9D43083506000C2D1ED20C25A94259
:10C690001DD8300000F0E8FA254A1468210000296E
:10C6A00019D1244C2368002B03D1300000F0CAF9C3
:10C6B00020602900300000F0C5F9431C2BD10C2369
:10C6C0003000336000F0D1FA03E0002DDFDA0C23F4
:10C6D0003360002070BD0B685B1B19D40B2B03D992
:10C6E0000B60CC18256003E04B688C420DD11360C1
:10C6F000300000F0BAFA200007220B30231D9043CF
:10C70000C31AE7D05A42E250E4E763600C00EFE757
:10C710000C004968C3E70323C41C9C43A042E1D03A
:10C72000211A300000F08EF9431CDBD1C7E7C04668
:10C730002C1C0020301C0020F8B507000D0016004E
:10C74000002905D11100FFF799FF04002000F8BD72
:10C75000002A03D1FFF748FF3400F7E700F086FA1C
:10C760002C00B042F2D231003800FFF787FF041EE0
:10C77000ECD029003200FEF7BFFF29003800FFF798
:10C7800033FFE3E7F0B58E6885B007000C00039235
:10C7900001939E423CD890238A89DB001A4234D010
:10C7A0000325096923685B1A0293636902985D4354
:10C7B000EB0F5D19019B6D1001331B18AB4200D9C3
:10C7C0001D00530532D529003800FFF757FF061E1C
:10C7D00009D10C233B6040230120A289404213432E
:10C7E000A38105B0F0BD029A2169FEF785FFA389F8
:10C7F000144A1A4080231343A381029B2661F61832
:10C8000026606561019EED1AA560019B9E4200D9DC
:10C81000019E320003992068FEF777FFA36800208D
:10C820009B1BA36023689E192660DAE72A00380064
:10C83000FFF782FF061EE0D121693800FFF7D4FE22
:10C84000C7E7C0467FFBFFFFF0B59FB0029005939E
:10C850008B890F0016001B0611D50B69002B0ED11A
:10C860004021FFF70BFF38603861002805D10C2309
:10C87000029A013813601FB0F0BD40237B61002392
:10C8800006AC6361203363761033A37635002B78D2
:10C89000002B01D0252B46D1AB1B04930CD03200CA
:10C8A00039000298FFF76EFF431C00D1AEE06269C9
:10C8B000049B9446634463612B78002B00D1A5E070
:10C8C000012200235242626002A9543252186E1CA7
:10C8D0002360E360A3601370A36531780522544898
:10C8E000FFF776FE751C00281FD12268D30604D5F9
:10C8F000532302A95B1820211970130704D5532371
:10C9000002A95B182B21197033782A2B16D0350019
:10C9100000210A20E3682A786E1C303A092A4ED991
:10C92000002918D010E00135B1E7414B2268C01A48
:10C9300001238340134323602E00CEE7059B191D7E
:10C940001B680591002B01DB099304E05B42E36067
:10C950000223134323602B782E2B0AD16B782A2BCA
:10C9600035D1059B02351A1D1B680592002B2BDB68
:10C970000793304E297803223000FFF729FE002864
:10C9800006D04023801B8340226801351343236077
:10C990002978062228486E1C2176FFF719FE002808
:10C9A0003CD0264B002B25D10722059B0733934310
:10C9B000083305936369039A9B18636166E74343F1
:10C9C00001219B183500A6E701235B42D0E7002335
:10C9D0000A201A000135636029786E1C3039092954
:10C9E00003D9002BC5D00792C3E742430123521855
:10C9F0003500F1E705AB00933A00114B2100029896
:10CA000000E000BF0390039B0133D3D1BB890B9897
:10CA10005B0600D42FE7012040422CE705AB0093D2
:10CA20003A00074B21000298FFF736F8EAE7C046C4
:10CA300090E4000096E400009AE40000000000008A
:10CA400085C70000002370B5064C05000800236070
:10CA500000F060F9431C03D12368002B00D02B6049
:10CA600070BDC046C02F002070B504000D001F2906
:10CA700004D9162303600120404270BD436C002B93
:10CA800004D08A009B181A68002A08D1200000F000
:10CA900031F82A000100200000F01AF8EDE700202C
:10CAA000012AEAD0511C03D1162301302360E4E7A8
:10CAB000002428001C6090472000DEE710B5034BDF
:10CAC00001001868FFF7D0FF10BDC04680000020AD
:10CAD000002370B5064C050008001100236000F02B
:10CAE00001F9431C03D12368002B00D02B6070BDDB
:10CAF000C02F002010B500F0E5F810BD70B50C0097
:10CB00000E25495F00F0BAF8002803DB636D1B189F
:10CB1000636570BDA389024A1340A381F9E7C0464B
:10CB2000FFEFFFFFF8B51F008B8905000C00160012
:10CB3000DB0505D50E23C95E0022022300F080F834
:10CB4000A389054A28001340A38132000E23E15E29
:10CB50003B0000F02BF8F8BDFFEFFFFF70B50C00B5
:10CB60000E25495F00F06CF8A389421C03D1054AE9
:10CB70001340A38170BD802252011343A3816065DD
:10CB8000F8E7C046FFEFFFFF10B50E23C95E00F0C7
:10CB900021F810BD0B1E04D0FF2A04D98A2303609C
:10CBA0008B3B180070470A700123FAE770B5050047
:10CBB000080011000022064C22601A0000F0B8F8AC
:10CBC000431C03D12368002B00D02B6070BDC046EE
:10CBD000C02F0020002370B5064C0500080023601C
:10CBE00000F060F8431C03D12368002B00D02B60B9
:10CBF00070BDC046C02F0020002370B5064C050054
:10CC000008001100236000F055F8431C03D123688D
:10CC1000002B00D02B6070BDC02F0020002370B50A
:10CC2000064C05000800236000F054F8431C03D1B3
:10CC30002368002B00D02B6070BDC046C02F0020A1
:10CC400070B50500080011000022064C22601A0091
:10CC500000F050F8431C03D12368002B00D02B6058
:10CC600070BDC046C02F0020704770470B1F1B6867
:10CC7000181F002B01DA0B58C018704770B505005B
:10CC8000080011000022064C22601A0000F03AF859
:10CC9000431C03D12368002B00D02B6070BDC0461D
:10CCA000C02F002058220120014B40421A607047DB
:10CCB000C02F002058220120014B40421A607047CB
:10CCC000C02F002058220120014B40421A607047BB
:10CCD000C02F00205822024B00201A607047C04627
:10CCE000C02F002058220120014B40421A6070479B
:10CCF000C02F002058220120014B40421A6070478B
:10CD0000C02F002058220120014B40421A6070477A
:10CD1000C02F0020044A1368002B00D1034B1818C1
:10CD2000106018007047C046341C0020C82F002037
:10CD300058220120014B40421A607047C02F00204A
:10CD4000FEE7C046F8B5C046F8BC08BC9E46704732
:10CD5000F8B5C046F8BC08BC9E4670476461746173
:10CD600000000000E0CD0000EF010000E9CD000070
:10CD7000E3020000F1CD000019090000F8CD000029
:10CD8000290A0000FDCD00004105000008CE00008A
:10CD9000530300000DCE0000810C000019CE0000EE
:10CDA0001F02000023CE00002108000031CE000049
:10CDB000CD0600003ECE00000305000072616E64E7
:10CDC0006F6D00616C6C006C6173740066616C73F4
:10CDD00065007472756500252E3135732E2E2E0078
:10CDE0006D616B654C697374006164644C6173744C
:10CDF0000064656C657465006A6F696E00636F70CE
:10CE00007946726F6D546F0066696E64006A6F696F
:10CE10006E537472696E677300756E69636F6465D3
:10CE2000417400756E69636F6465537472696E67EF
:10CE3000006E65774279746541727261790066723D
:10CE400065654D656D6F727900000000B1CE000020
:10CE50002D110000B6CE00004B110000F1CD0000F6
:10CE60004F110000BCCE000031110000C6CE000002
:10CE700053110000CFCE000057110000D9CE0000A2
:10CE80005B110000E4CE00005F110000F0CE000056
:10CE900035110000F9CE00004311000003CF00005F
:10CEA000391100000ECF00004711000066696C6563
:10CEB000006F70656E00636C6F736500656E644F24
:10CEC0006646696C6500726561644C696E650072E6
:10CED000656164427974657300617070656E644C5D
:10CEE000696E6500617070656E6442797465730087
:10CEF00066696C6553697A650073746172744C6914
:10CF00007374006E657874496E4C6973740073793C
:10CF10007374656D496E666F000000009013000029
:10CF2000A0130000BA1300003814000070140000B1
:10CF3000A6140000DE1400000415000040150000D7
:10CF400082150000D81500001C160000881600008D
:10CF5000D0160000F61600002E170000741700000F
:10CF60009A170000C8170000F617000038180000D4
:10CF7000BC1800008E190000181A00006E1A00007C
:10CF8000BA1A0000DA1A0000FC1A0000AE1B0000FA
:10CF9000F41B00006C1C00009A1C0000CA1C00005E
:10CFA000001D0000841D0000EC1D0000321E00006A
:10CFB0007A1E0000F01E0000661F0000AE1F000079
:10CFC000F41F00002A20000070200000B62000009E
:10CFD000082100005C210000B0210000EE210000CB
:10CFE000582200008E220000D62200001E230000DE
:10CFF00066230000A0230000E82300003024000086
:10D000009C250000C81700002E170000982400007F
:10D0100090130000D8240000042500003A250000E9
:10D02000662500009013000090130000901300008C
:10D030009013000016260000582600009E260000CF
:10D04000EE2600001A2700006A2700009027000043
:10D05000BE2700009013000090130000E22700009C
:10D060001228000042280000AC280000D62800004A
:10D070000C290000362900005E29000086290000E6
:10D08000B6290000E6290000102A00003A2A000014
:10D090006A2A0000942A00009013000090130000F8
:10D0A000901300009013000090130000C42A0000A9
:10D0B000F02A00001C2B0000482B0000742B0000FD
:10D0C000AA2B0000E02B0000162C00004C2C0000C6
:10D0D000782C0000AC2C0000E22C00009013000023
:10D0E00090130000901300009013000090130000B4
:10D0F00090130000901300009013000090130000A4
:10D100009013000090130000901300009013000093
:10D11000901300000E2D0000442D00005B256420BC
:10D120006974656D206C6973745D002825642062E4
:10D13000797465732900286F626A65637420747955
:10D1400070653A2025642900537461636B20756E05
:10D15000646572666C6F7700626F6F6C65616E00FC
:10D160006E756D62657200737472696E67006C69CA
:10D1700073740062797465206172726179000000D5
:10D180000700000003000000E1D10000652E000050
:10D19000E9D10000152F0000F2D10000BF2F0000E0
:10D1A000FBD10000692E000004D20000C32F000054
:10D1B0000CD20000AD2F00001C0000000100000098
:10D1C000020000000400000005000000060000004E
:10D1D000100000001100000043616C6C696F706505
:10D1E00000686173546F6E6500706C6179546F6E86
:10D1F0006500686173536572766F0073657453657B
:10D2000072766F00646163496E697400646163578C
:10D210007269746500474320746F6F6B202564202A
:10D2200075736563733B206672656520256420779E
:10D230006F726473003C496E74656765723E003CB2
:10D240004C6973743E003C4F626A6563743E003CF7
:10D250004279746541727261793E000D0A564D2023
:10D2600050616E69633A2025730D0A006D6973631E
:10D2700000000000A9D20000953C0000B2D20000DE
:10D28000253C0000B6D20000793B0000BED2000071
:10D290001F3B0000C8D20000B53A0000D4D2000005
:10D2A000B73900006E756C6C00686578546F496E14
:10D2B000740073696E006A736F6E476574006A73F9
:10D2C0006F6E436F756E74006A736F6E56616C7526
:10D2D000654174006A736F6E4B657941740000009C
:10D2E0003CD30000013D000044D30000053D000098
:10D2F0004ED30000233D000057D300002D3D000019
:10D3000062D30000373D00006ED30000413D0000B5
:10D3100083D300004B3D000098D30000553D000032
:10D32000A4D300005F3D0000B4D300000F3D000017
:10D33000C0D30000193D00006E657400686173572A
:10D340006946690073746172745769466900737441
:10D350006F705769466900776966695374617475BF
:10D3600073006D7949504164647265737300687429
:10D370007470536572766572476574526571756530
:10D38000737400726573706F6E64546F4874747058
:10D39000526571756573740068747470436F6E6E56
:10D3A00065637400687474704973436F6E6E65636F
:10D3B0007465640068747470526571756573740087
:10D3C00068747470526573706F6E7365000D0E0F24
:10D3D00004050C0B0A0607080900000000000808F5
:10D3E0000800080A4A4000000A5FEA5FEA0ED92EE8
:10D3F000D36E19324489330C924C924D08080000C8
:10D400000004880808040804848488000A448A40C8
:10D4100000048EC480000000048800000EC00000DC
:10D420000000080001224488100C9252524C048CD7
:10D4300084848E1C824C901E1EC244924C06CA529A
:10D440005FE21FF01EC13E02448ED12E1FE24488CF
:10D45000100ED12ED12E0ED12EC488000800080047
:10D4600000048004880244880482000EC00EC008B4
:10D47000048244880ED126C0040ED135B36C0C92C0
:10D480005ED2521C925C925C0ED010100E1C925216
:10D49000525C1ED01C901E1ED01C90100ED013711A
:10D4A0002E12525ED2521C8808081C1FE242524CB7
:10D4B0001254981492101010101E113B75B13111B6
:10D4C0003935B3710C9252524C1C925C90100C92F4
:10D4D000524C861C925C92510ED00C825C1FE484EC
:10D4E0008484125252524C1131312A44113135BBCD
:10D4F0007112524C9252112A4484841EC488101E08
:10D500000EC808080E10080482410EC242424E04A2
:10D510008A400000000000001F0804800000000E88
:10D52000D2524F10101C925C000ED0100E02424ED0
:10D53000D24E0C925C900E06C81C88080ED24EC2C9
:10D540004C10101C92520800080808024002424C7D
:10D5500010149814920808080806001B75B13100D1
:10D560001C925252000C92524C001C925C90000E85
:10D57000D24EC2000ED010100006C8049808080E43
:10D58000C807001252524F0011312A4400113135A0
:10D59000BB00124C8C9200112A4498001EC4881EB5
:10D5A00006C48C8486080808080818080C88180027
:10D5B000000C836000000000010000000200000079
:10D5C0000300000004000000050000000600000049
:10D5D0000700000008000000090000000A00000029
:10D5E0000B0000000C0000000D0000000E00000009
:10D5F0000F000000100000001200000014000000E6
:10D6000016000000180000001A0000001C000000B6
:10D610001E00000020000000230000002600000083
:10D62000290000002C0000002F0000003200000044
:10D63000360000003A0000003E00000042000000FA
:10D64000460000004B0000005000000055000000A4
:10D650005A00000061000000680000006F00000038
:10D66000760000007D000000840000008B000000B8
:10D670009200000099000000A0000000A700000038
:10D68000AE000000B5000000BC000000C3000000B8
:10D69000CA000000D1000000D8000000DF00000038
:10D6A000E6000000ED000000F4000000FB000000B8
:10D6B000FF00000004D70000813D00000FD70000EC
:10D6C0001D43000019D70000453F000026D7000089
:10D6D0008D4100002DD70000DD41000036D700004D
:10D6E0002D42000042D700002541000053D7000022
:10D6F000B53F000060D70000B5400000646973705A
:10D700006C6179006C696768744C6576656C006D56
:10D7100062446973706C6179006D62446973706C06
:10D7200061794F6666006D62506C6F74006D625572
:10D730006E706C6F74006D624472617753686170D3
:10D7400065006D625368617065466F724C657474F4
:10D750006572006E656F506978656C53656E640024
:10D760006E656F506978656C53657450696E004ED4
:10D770006F7420656E6F75676820726F6F6D2065BE
:10D7800076656E20616674657220636F6D7061638B
:10D7900074696F6E00436F6D7061637465642046D9
:10D7A0006C61736820636F64652073746F72650ABF
:10D7B000256420627974657320757365642028255B
:10D7C00064252529206F662025640042616420724B
:10D7D00065636F726420666F756E6420647572692C
:10D7E0006E6720696E697469616C697A6174696FCA
:10D7F0006E00256420256420256420282564207778
:10D800006F72647329002564207265636F7264739C
:10D810002C20256420776F7264732C206D61784909
:10D82000442025642C20636F6D70616374696F6E92
:10D83000206379636C657320256400526573746F8F
:10D840007265642025642073637269707473005379
:10D8500074617274656400726164696F0000000035
:10D86000F0D80000F54C0000FDD80000914F0000FA
:10D870000DD90000114F00001BD9000025510000F8
:10D8800026D900001D4D000036D90000A54D00002E
:10D890004AD900008D4D000059D9000007530000FF
:10D8A00065D90000855200006ED9000029520000A1
:10D8B00079D900007151000084D90000AD510000F9
:10D8C0008DD90000E151000096D900002D4D0000D7
:10D8D000A5D900000D4D0000AED900003D4D00005F
:10D8E0006E6F6E65006F74686572007061697200BA
:10D8F00064697361626C65526164696F006D657320
:10D90000736167655265636569766564007061631C
:10D910006B657452656365697665007061636B65FC
:10D920007453656E64007265636569766564496EFB
:10D9300074656765720072656365697665644D65D7
:10D9400073736167655479706500726563656976A4
:10D950006564537472696E670073656E64496E74B2
:10D96000656765720073656E645061697200736506
:10D970006E64537472696E67007365744368616E98
:10D980006E656C0073657447726F757000736574B3
:10D99000506F776572007369676E616C537472655E
:10D9A0006E677468006465766963654944006C61FC
:10D9B00073744D657373616765494400556E6B6E92
:10D9C0006F776E207072696D6974697665205B256A
:10D9D000733A25735D000000000000009630077761
:10D9E0002C610EEEBA51099919C46D078FF46A7053
:10D9F00035A563E9A395649E3288DB0EA4B8DC7973
:10DA00001EE9D5E088D9D2972B4CB609BD7CB17EF2
:10DA1000072DB8E7911DBF906410B71DF220B06AC2
:10DA20004871B9F3DE41BE847DD4DA1AEBE4DD6DD2
:10DA300051B5D4F4C785D38356986C13C0A86B64D2
:10DA40007AF962FDECC9658A4F5C0114D96C0663F2
:10DA5000633D0FFAF50D088DC8206E3B5E10694CD2
:10DA6000E44160D5727167A2D1E4033C47D4044B12
:10DA7000FD850DD26BB50AA5FAA8B5356C98B242F2
:10DA8000D6C9BBDB40F9BCACE36CD832755CDF4572
:10DA9000CF0DD6DC593DD1ABAC30D9263A00DE51A2
:10DAA0008051D7C81661D0BFB5F4B42123C4B35692
:10DAB0009995BACF0FA5BDB89EB802280888055F12
:10DAC000B2D90CC624E90BB1877C6F2F114C685872
:10DAD000AB1D61C13D2D66B69041DC760671DB0160
:10DAE000BC20D2982A10D5EF8985B1711FB5B60632
:10DAF000A5E4BF9F33D4B8E8A2C9077834F9000F72
:10DB00008EA8099618980EE1BB0D6A7F2D3D6D0811
:10DB1000976C6491015C63E6F4516B6B62616C1C01
:10DB2000D83065854E0062F2ED95066C7BA5011B31
:10DB3000C1F4088257C40FF5C6D9B06550E9B712D1
:10DB4000EAB8BE8B7C88B9FCDF1DDD62492DDA1591
:10DB5000F37CD38C654CD4FB5861B24DCE51B53AB1
:10DB60007400BCA3E230BBD441A5DF4AD795D83DB1
:10DB70006DC4D1A4FBF4D6D36AE96943FCD96E34F1
:10DB8000468867ADD0B860DA732D0444E51D0333D1
:10DB90005F4C0AAAC97C0DDD3C710550AA410227E1
:10DBA00010100BBE86200CC925B56857B3856F20B1
:10DBB00009D466B99FE461CE0EF9DE5E98C9D92911
:10DBC0002298D0B0B4A8D7C7173DB359810DB42E51
:10DBD0003B5CBDB7AD6CBAC02083B8EDB6B3BF9A9D
:10DBE0000CE2B6039AD2B1743947D5EAAF77D29D29
:10DBF0001526DB048316DC73120B63E3843B649409
:10DC00003E6A6D0DA85A6A7A0BCF0EE49DFF099308
:10DC100027AE000AB19E077D44930FF0D2A3088778
:10DC200068F2011EFEC206695D5762F7CB67658028
:10DC300071366C19E7066B6E761BD4FEE02BD38928
:10DC40005A7ADA10CC4ADD676FDFB9F9F9EFBE8E88
:10DC500043BEB717D58EB060E8A3D6D67E93D1A1C8
:10DC6000C4C2D83852F2DF4FF167BBD16757BCA6A8
:10DC7000DD06B53F4B36B248DA2B0DD84C1B0AAF48
:10DC8000F64A0336607A0441C3EF60DF55DF67A8C8
:10DC9000EF8E6E3179BE69468CB361CB1A8366BC58
:10DCA000A0D26F2536E2685295770CCC03470BBBA8
:10DCB000B91602222F260555BE3BBAC5280BBDB2A8
:10DCC000925AB42B046AB35CA7FFD7C231CFD0B548
:10DCD0008B9ED92C1DAEDE5BB0C2649B26F263EC3A
:10DCE0009CA36A750A936D02A906099C3F360EEB48
:10DCF0008567077213570005824ABF95147AB8E208
:10DD0000AE2BB17B381BB60C9B8ED2920DBED5E5E7
:10DD1000B7EFDC7C21DFDB0BD4D2D38642E2D4F137
:10DD2000F8B3DD686E83DA1FCD16BE815B26B9F6C7
:10DD3000E177B06F7747B718E65A0888706A0FFF27
:10DD4000CA3B06665C0B0111FF9E658F69AE62F8E7
:10DD5000D3FF6B6145CF6C1678E20AA0EED20DD7E7
:10DD60005483044EC2B30339612667A7F71660D007
:10DD70004D476949DB776E3E4A6AD1AEDC5AD6D947
:10DD8000660BDF40F03BD83753AEBCA9C59EBBDE67
:10DD90007FCFB247E9FFB5301CF2BDBD8AC2BACA17
:10DDA0003093B353A6A3B4240536D0BA9306D7CD87
:10DDB0002957DE54BF67D9232E7A66B3B84A61C4A7
:10DDC000021B685D942B6F2A37BE0BB4A18E0CC367
:10DDD0001BDF055A8DEF022D416C6C207461736B53
:10DDE000732073746F707065640076313037002073
:10DDF0002573202573004D656D6F727920636C6506
:10DE000061726564004E6F2066726565207461738F
:10DE10006B20656E747269657300000074DE00002B
:10DE20002567000081DE00007D6600008DDE0000B9
:10DE30004D66000093DE00005D66000099DE000084
:10DE40006D6600009FDE000081620000A9DE000018
:10DE500099660000B1DE00009D640000BADE00009B
:10DE6000DD620000C2DE00000564000073656E73B1
:10DE70006F727300616363656C65726174696F6E64
:10DE80000074656D70657261747572650074696C9B
:10DE900074580074696C74590074696C745A007415
:10DEA0006F756368526561640069326352656164CD
:10DEB0000069326357726974650072656164444831
:10DEC00054006D6963726F70686F6E6500000000CA
:10DED00044DF0000DD67000052DF0000E167000062
:10DEE0005BDF0000ED67000065DF0000F167000008
:10DEF0006EDF0000F567000073DF0000F9670000C7
:10DF000078DF0000FD67000084DF0000016800008A
:10DF10008BDF00000568000094DF00000968000046
:10DF200099DF00000D680000A4DF00001168000008
:10DF3000AEDF0000E5670000B8DF0000E967000021
:10DF400074667400656E61626C65446973706C61BF
:10DF5000790067657457696474680067657448651B
:10DF60006967687400736574506978656C006C69E2
:10DF70006E65007265637400726F756E64656452DD
:10DF800065637400636972636C6500747269616EC5
:10DF9000676C65007465787400746674546F75639B
:10DFA00068656400746674546F75636858007466BD
:10DFB00074546F7563685900746674546F75636840
:10DFC000507265737375726500766172730000003C
:10DFD000F0DF0000A16C0000FADF0000816C00009F
:10DFE00003E000005D6C00000FE00000E96B000042
:10DFF000766172457869737473007661724E616DF3
:10E000006564007365745661724E616D6564007677
:10E0100061724E616D65466F72496E646578005736
:10E02000656C636F6D6520746F204D6963726F421C
:10E030006C6F636B732100705F73706920213D20EA
:10E040004E554C4C002F686F6D652F6769742F2EED
:10E05000706C6174666F726D696F2F7061636B6154
:10E060006765732F6672616D65776F726B2D617274
:10E070006475696E6F6E6F726469636E7266352F58
:10E080006C69627261726965732F5350492F5350E6
:10E09000492E63707000535049436C6173733A3A70
:10E0A000535049436C617373284E52465F53504935
:10E0B0005F547970652A2C2075696E74385F742CF2
:10E0C0002075696E74385F742C2075696E74385FC2
:10E0D000742900000000000000000000AD6E000088
:10E0E000696E00008F6E0000996E0000A36E000044
:10E0F0008D6E000000000000010000000200000022
:10E1000016000000040000000500000006000000EA
:10E110000700000008000000090000000A000000DD
:10E120000B0000000C0000000D0000000E000000BD
:10E130000F0000001A0000001B0000001400000087
:10E140001300000011000000170000001000000084
:10E150001C0000001D0000001E0000001200000056
:10E160001500000003000000180000001900000066
:10E17000000000000000000085730000ED7B00003F
:10E1800005740000197400000F7400008173000012
:10E190007573000025740000A17300007173000006
:10E1A000000000000000304300000000000030C309
:10E1B0007371727400000000FB21F93FFB210940DC
:10E1C0007CD91240FB2119407A6A1F407CD9224039
:10E1D000BBFD2540FB2129403A462C407A6A2F405E
:10E1E0005C4731407CD932409C6B3440BBFD3540AC
:10E1F000DB8F3740FB2139401BB43A403A463C4064
:10E200005AD83D407A6A3F404C7E40405C4741408E
:10E210006C1042407CD942408CA243409C6B4440ED
:10E22000AC344540BBFD4540CBC64640DB8F474044
:10E23000EB584840FB21494083F9A200444E6E0050
:10E24000FC291500D1572700DD34F50062DBC00042
:10E250003C999500419043006351FE00BBDEAB004A
:10E26000B761C5003A6E2400D24D42004906E00075
:10E2700009EA2E001C92D100EB1DFE0029B11C0002
:10E28000E83EA700F535820044BB2E009CE98400DF
:10E29000B4267000417E5F00D69139005383390067
:10E2A0009CF439008B5F840028F9BD00F81F3B0007
:10E2B000DEFF97000F980500112FEF000A5A8B0020
:10E2C0006D1F6D00CF7E360009CB2700464FB7008B
:10E2D0009E663F002DEA5F00BA277500E5EBC70098
:10E2E0003D7BF100F739070092528A00FB6BEA0090
:10E2F0001FB15F00085D8D00300356007BFC4600B7
:10E30000F0AB6B0020BCCF0036F49A00E3A91D00EF
:10E310005E619100081BE60085996500A0145F000E
:10E320008D40680080D8FF0027734D00060631003D
:10E33000CA561500C9A873007BE260006B8CC00050
:10E3400000000040FB21F93F000000002D44743E16
:10E35000000000809846F83C0000006051CC783BFB
:10E3600000000080831BF0390000004020257A382F
:10E37000000000802282E336000000001DF36935B2
:10E38000020000000300000004000000060000007E
:10E39000649800000E9800000E9800003C99000060
:10E3A0000A9800000A980000329900003C99000089
:10E3B0000A980000329900000A9800003C99000079
:10E3C00040990000409900004099000048990000E1
:10E3D00040A30000B2A10000F6A100005AA1000075
:10E3E000F6A10000E6A20000F6A100005AA100007C
:10E3F000B2A10000B2A10000E6A200005AA10000F4
:10E4000052A1000052A1000052A10000F4A200009D
:10E4100068AA00006AA900006AA9000088AC000090
:10E4200064A9000064A9000070AC000088AC000082
:10E4300064A9000070AC000064A9000088AC000072
:10E440007EAC00007EAC00007EAC00008CAC000016
:10E450002C2066756E6374696F6E3A200061737369
:10E46000657274696F6E2022257322206661696C63
:10E4700065643A2066696C6520222573222C206C25
:10E48000696E65202564257325730A0084000020C9
:10E49000232D302B2000686C4C006566674546478D
:10E4A0000030313233343536373839414243444510
:10E4B000460030313233343536373839616263647F
:10E4C0006566000000000000000000000000000081
:10E4D000000000000000000000000000000000003C
:10E4E000000000000000000000000000000000002C
:10E4F000000000000000000000000000000000001C
:10E50000000000000000000000000000000000000B
:10E5100000000000000000000000000000000000FB
:10E52000000000004300504F5349580000202020B5
:10E5300020202020202028282828282020202020B3
:10E540002020202020202020202020202088101083
:10E5500010101010101010101010101010040404DF
:10E56000040404040404041010101010101041419D
:10E57000414141410101010101010101010101018B
:10E58000010101010101010110101010101042429F
:10E59000424242420202020202020202020202025B
:10E5A00002020202020202021010101020000000FB
:10E5B000000000000000000000000000000000005B
:10E5C000000000000000000000000000000000004B
:10E5D000000000000000000000000000000000003B
:10E5E000000000000000000000000000000000002B
:10E5F000000000000000000000000000000000001B
:10E60000000000000000000000000000000000000A
:10E6100000000000000000000000000000000000FA
:10E6200000000000000000000000000000000000EA
:04E6300000000000E6
:08E63400D41AFF7F0100000071
:10E63C00FFFFFFFFD007000001000000E803DC052E
:10E64C00DC05DC05DC050000FFFFFFFFFFFFFFFF23
:10E65C001800000019FCFFFFFFFFFFFF0024F4006F
:10E66C000200000003000000FFFFFFFF000000009D
:10E67C00010000000000020001000000FFFFFFFF8E
:10E68C000000000002000000000004000200000076
:10E69C00FFFFFFFF00000000030000000000080067
:10E6AC00030000000A000000080000000100000048
:10E6BC008400002000000000E4E4000004E50000F9
:10E6CC00C4E4000000000000000000000000000096
:10E6DC00000000000000000000000000000000002E
:10E6EC00000000000000000000000000000000001E
:10E6FC00000000000000000000000000000000000E
:10E70C0000000000000000000000000000000000FD
:10E71C0000000000430000000000000000000000AA
:10E72C0000000000000000000000000000000000DD
:10E73C00000000004300000000000000000000008A
:10E74C0000000000000000000000000000000000BD
:10E75C00000000004300000000000000000000006A
:10E76C00000000000000000000000000000000009D
:10E77C00000000004300000000000000000000004A
:10E78C00000000000000000000000000000000007D
:10E79C00000000004300000000000000000000002A
:10E7AC00000000000000000000000000000000005D
:10E7BC00000000004300000000000000000000000A
:10E7CC00000000000000000000000000000000003D
:10E7DC0000000000430000000000000000000000EA
:10E7EC00000000000000000000000000000000001D
:10E7FC000000000095CB0000ADC50000000000003B
:10E80C002CE50000DECD00006BD200006BD20000C6
:10E81C006BD200006BD200006BD200006BD20000F8
:10E82C006BD200006BD200006BD20000FFFFFFFF29
:10E83C00FFFFFFFFFFFFFFFFFFFF00000100415341
:10E84C0043494900000000000000000000000000E7
:10E85C000000000000000000000000000000415318
:10E86C0043494900000000000000000000000000C7
:10E87C00000000000000000000000000000000008C
:10E88C00E9000000396E0000A9710000D17600008B
:04E89C00C1000000B7
:040000030000724542
:00000001FF
